:20000000003A0120D1F8010039FB021039FB021039FB021039FB021039FB021039FB021017
:1C00200039FB021039FB021039FB021039FB021039FB021039FB021011FB021002
:20004000BA492DE9F04F0446B74ADFF8E8920E68A578507800279046ADF1540D29460C29B1
:2000600007D9DFF8CCB2DFF8D0A2203933290FD953E3DFE811F06D055E0543052D050D0506
:20008000F704F304DD04C7045203BA04B6049604DFE811F083047F047B046B046704EC0242
:2000A00051042F04B10287024303430343034303430343030B04F003D303B80359029D034A
:2000C0003402FC01430343034303430343034303E801B5019C0143038C03790183037703BE
:2000E0006A0354012A01E500660362035803C000480382004503670046003400E1788DF871
:200100002A7031F07F0006D011F07F0F0CBF381C0120CA49087053210DF12A0300F004BD25
:2001200008F1110332203946012226F039F808F1120333203946012226F032F8C84898F894
:2001400011100078012905D04FF400611EF0EAFC00F001BD4FF40061642226F0ADFB00F0E9
:20016000FABC8DF82B7078B9E41C204626F058FA0546A01C0446083026F052FA0246214610
:20018000284624F0C0F900E012208DF82B0051210DF12B0300F0C8BCE01C26F041FAE51C02
:2001A000AE784FF6FF748DF80A600546ADF80850AC4218D0E01EA84215D0A01EA84212D0FD
:2001C00002208DF80C00ADF80E5003A81BF040FE012818BF4FF001090CD1BDF80E00ADF8E7
:2001E0000800012000E038468DF80B0002A81DF0E1FC8146E41EAC4204DC012088F82A00F2
:2002000088F82B6021F096FD8DF82C904F210BAB00F08ABC20798DF82E00E078012814D0E1
:20022000022809D0032805D052200DF12E0124F027FB0FE03C4600E0012452200DF12E01D1
:2002400021F0B8FD88F8004004E052200DF12E0121F0B0FD4D210DF12E0300F065BCE178D0
:2002600038465EB13279914205D1F2880DEB4003401CC0B21A813668002EF3D18DF830003A
:200280009DF83000012404EB4000C0B2054619F097FE5FEA000806D18DF8307049212246CB
:2002A0000CAB00F042BC02469DF8300002F8010B38469DF8301081420ADC652049212A462B
:2002C000434622F0A5F8404621F0D4FB00F043BC0DEB400108310B7813700988401CC0B2BA
:2002E00009125170921CE4E7301CE4788DF8317013D03E4601798C420BD11EB905680B49B8
:200300000D6002E001683160056821F0B3FB284601E0064600680028ECD121F06BFD0DF109
:200320003103472100F000BCE404012064F20020671B0120280401208A010120E01C10F856
:20034000014B26F06DF90146C7480068224650B13E4603799A4202D1C388994205D00646B8
:2003600000680028F5D1012008E006B9BE4E0168316021F07FFB21F03DFD38468DF832004E
:200380000DF13203CDE739460DF12200062207911BF024FDE01C07A924F09EFF8DF82200E7
:2003A000079870B101888DF8231046888DF8256009128DF8241031128DF8261000798DF894
:2003C0002700432106220DF12203AEE364788DF8377048B1012805D002281CBF01208DF80C
:2003E000370004D1022000E004200DF0BFFE24F01F04202C40F0AF830DF13703EEE22046BE
:2004000090F80180C01C26F00BF959460A7849468E6856B13C4633799A4202D1F3889842FE
:2004200005D034463668002EF5D101200EE03CB9346804B93C468C6004E0C046DC01012028
:2004400030682060304621F015FB384628F01F088DF83800B8F1200F40F07D830EABBDE213
:200460005001012020464478C01C26F0D9F80146584600781FF042FF24F01F048DF8390083
:20048000202C40F068830DF13903A7E2E41C204626F0C6F8A41CADF8080014F8010B04214E
:2004A0008DF81000204625F015F80646201D10F8019B10F8018B26F0B3F8044631464A464C
:2004C000434602A800941DF031FA8DF83A009DF810000F280FD1022053468DF810001888B2
:2004E00031464A46ADF80800434602A800941DF01DFA8DF83A000DF13A036FE2207826460E
:20050000042806F1030614BF16F8010B02208DF81000304626F084F8D54CADF80800B01C69
:2005200010F8018B012626700278414602A81EF047FE8DF83B002770404625F0CBFB0DF1B6
:200540003B0332464BE20220E41C8DF81000204626F066F84E46A11CADF808000C7A7068CB
:2005600026F0CEF97168C4F3400804F00104B8F1010F0F7204D17268107A40F04000107268
:20058000012C03D1087A40F080000872484602A9342209231DF080FD0DF13D038DF83D0069
:2005A000C1E20226E41C8DF81060204626F038F8A41CADF80800204626F032F8A2788046DC
:2005C00002A84146144625F023F98DF845009DF810000F280CD1504600888DF81060414642
:2005E0002246ADF8080002A825F012F98DF845000DF14503F2E10226E41C8DF810602046B6
:2006000026F00EF8A41CADF8080014F8010B8DF84700204626F004F8A41C14F8019B8046C7
:2006200002A90DF14700424600944B46019721F011F88DF846009DF810000F2811D150464C
:2006400000888DF810603E4602A94246ADF808004B4600940DF14700019620F0FBFF8DF829
:2006600046000DF14603B9E164F20020A946E51CA878B846FE280BD1E878FF2808D12078D5
:20068000082805DB284625F0CBFF294624F0BFF9284608A925F09CF9041C0ED1182019F0B9
:2006A0008FFC5FEA000807D0BDF8200039461822434625F075FD00B1C824192019F080FC8E
:2006C000061C20D05CB9701C2946082225F066FA06F109004146102225F060FA04E0701CC1
:2006E000FF2118221BF07AFB3470652049461922334621F08DFE3046394619221BF06EFB74
:20070000304621F0B7F9B8F1000F00F024824046394618221BF062FBD5E502271BE21BF0C2
:200720008DFF18E2E01C25F07BFFE51C0246A81C10F8011B1CF074FA4E210DF12D038DF8DB
:200740002D00F1E18DF82F7025F0DCFA0DF12F034C218DF82F00E7E120461BF035FFFAE1F2
:2007600020461EF08CF8F6E1E01C25F059FF6179A2791DF054FA46210DF133038DF833009E
:20078000D2E1E01C25F04CFF6179A27911F032FE45210DAB8DF83400C6E1E01C11F04CFB62
:2007A00044210DF135038DF83500BDE1E01C25F037FFE51CA91C0B4608310A4619461FF0F1
:2007C0005BF842210DF136038DF83600ACE10220E41C8DF81000204625F022FF4E46A11C40
:2007E000ADF808000C7A706826F08AF8706802A935220923047248461DF04EFC0FAB8DF8B6
:200800003C00EBE00220E41C8DF81000204625F007FFADF80800A0780DF13F0602A9332291
:200820008DF83F00012300964846019720F012FF0DF13E038DF83E00D0E00220E41C8DF89A
:200840001000204625F0ECFEADF80800A0780DF1410602A932228DF841000123009648460C
:20086000019720F0F7FE10AB8DF840005BE1C0468C0A01200220E41C8DF81000204625F030
:20088000CFFEADF80800A0780DF1430602A931228DF84300012300964846019720F0DAFEF1
:2008A0000DF142038DF842003DE10220E41C8DF81000204625F0B4FEA41CADF8080004219A
:2008C000204624F007FE4E46221D014612F8018B7068137825F056F902A900F8018B3022A1
:2008E0000370484606231DF0D7FB11AB8DF8440019E10126E41C8DF84860601C25F090FEFD
:20090000814604F10B0025F08BFE804694F800A0637BA07B22F036FC0093E01C494652468D
:20092000434613F06BFC12AB8D498DF84800042025F0A0FE05E60126E41C04218DF8496028
:20094000204624F0C7FD21791EF08CF885498DF84900022025F08EFE83490DF14903032095
:20096000E6E7204619F0E6FDF5E0E41C204625F057FEA11C0B4608310A4619461EF07CFF34
:200980000DF14A038DF84A00CDE020461AF089F9E1E020461AF042F9DDE020460FF0A4FE6E
:2009A000D9E0E01C25F03CFE4E464FF6FD740F22ADF8084071688DF81020022304121522CB
:2009C00001F8010B48460C7002A9F7701DF064FB39468DF84B000DF14B03F17001222946FC
:2009E000A3E0204618F0D8FDB5E0E41C204625F017FEA11C0A7A3B4622F028F813AB8DF8D5
:200A00004C0090E00220E41C8DF81000204625F007FEADF80800A01C25F002FE01461122EB
:200A200002A824F0F5FE0DF14D038DF84D007AE00220E41C8DF81000204625F0F1FDADF8C6
:200A40000800A01C25F0ECFD0146102202A824F0DFFE0DF14E038DF84E0064E020460FF0F5
:200A6000A3F978E00220E41C8DF81000204625F0D7FDADF80800A01C25F0D2FD01460522C1
:200A800002A824F0C5FE0DF14F038DF84F004AE00220E41C8DF81000204625F0C1FDA41CD7
:200AA000ADF80800204625F0BBFD4E467268A1781070726803125370706803230422817088
:200AC00002A948461DF0E8FA14AB8DF850002AE00220E41C8DF81000204625F0A1FDADF8DB
:200AE0000800A01C25F09CFD0146032202A824F08FFE0DF151038DF8510014E00226E41C89
:200B00008DF81060204625F08BFDADF80800A01C25F086FD0146324602A824F079FE0DF1EA
:200B200052038DF8520029460122652021F070FC11E0E41C204625F073FDA41C14F8011B31
:200B4000227822F053FB0DF153038DF85300EAE7204617F0FFF9384615B0BDE8F08FC046CC
:200B60006D290200CD4A0200C15101002DE9F04F04464FF6FE70ADF15C0DADF85400A44873
:200B800040784FF00008022812D1A148007878B92089002807BF30204146102001210EF0F9
:200BA000FDFE8DF8568052200DF1560121F002F96068217A08AA12F01DFA002800F0D98469
:200BC0009DF822000228B4BF012747469DF824000228A8BF4746BDF82A104FF6FE7BABF1EC
:200BE000060B8B450ED04FF6FE70401F884209D04FF6FE70001F884204D04FF6FE70C01E80
:200C0000884200D1474625F0D5FC9DF82310884240F0AF84002F00F0AC847D4840780228DB
:200C200004D19DF85100002840F0A384208D9DF82660678EADF84C00ADF82E70D6B1616839
:200C40009DF821209DF83C30012024F0FBFF002840F08F84C448001D007801280AD1208DD1
:200C600025F0F1FD30B1417901F0EF01417141F0080141719DF82570DFF8E492DFF8E4A283
:200C80004646002F49D19DF83D00474658BBBDF82A00034620F08EFE4546022808BF0125A7
:200CA000002D9DF8225018BF012749460988994208BF47F0020727B1002D14BF4021202185
:200CC0000F43184620F076FE012808BF47F00107002D3BD01298007825F0A6FA012818BFA2
:200CE00027F0010732E09DF8411041B1FF2906D09DF84000119A22F02BFA50B126E0524697
:200D0000BDF82A10508F884205D092F84A0004281CD101261AE0222718E0BDF82A10FF2009
:200D200023F0E6F9002804BF3D1C082708D09DF8250047F001052C2740F001008DF8250051
:200D400005F00305012D08BF47F0110730489DF82650407830F0010005D107F002010E43D5
:200D600008BF47F08007DFF8DCC295B961460E787EB107F0220122290BD007F042014229EA
:200D800040F0F78312990978062918BF072940F0F083F9094FEAA7155AD3BDF82A201299D6
:200DA00048B96046C01C0078800804D30878401E0A282FD909E00878C01E01282AD9001F2F
:200DC00028D0C01E26D0801E24D0B8F1000F21D148460088904240F0CC830D780520BDF845
:200DE0002C408DF8110004A824F036F9002800F0C0830269032313271370511C0F704C70B1
:200E000022128A70CD70448009F022FAB1E3C046E404012068081BD30878032802D148784F
:200E20000D2815D09DF8280038B1BDF82C000E990EF0AAFB012800F098839DF8270038B1EE
:200E4000BDF82A000D990EF09FFB012800F08A8309F10E00B4F844100088884209D1CDF856
:200E60000080208DB4F8421094F8462043460AF0C9FF9DF82600002843D0208DB4F8421069
:200E800020F092FC061C25D19DF8510088B99AF89000012835D112980078062801D1680892
:200EA0002FD2BDF82E100BF10700884240F0C5805FE3042024F04AF8011C00F05A836420D2
:200EC000087001274F70208D48809AF800001FF089FC4EE39DF821106068F3780A18527BFF
:200EE0009A4203D0F27040467060606840180421401C24F0EFFA7168814200F23A83401C46
:200F00007060B348DFF8C4B24078022800F08F8230F0010040F02D839AF832008008C0F0D9
:200F200028839DF8510030B3BDF82C0024F0E1FDE0B9A5495C46BDF82C000B686269990188
:200F4000A1EB83019047012840F01383A169BDF82C008847E168BDF82C00884709E3C04616
:200F60008A01012050010120500101206168487800F0DF0048709DF8320038B16168887957
:200F8000401E8871C0B28DF8320008B907F07F07380924D39DF82500F9084FF4805814D29F
:200FA00079091AD3811011F0070F01F0070604D0072E1CBF761EF6B20EB907F07F0700F0C8
:200FC000E30040EA8600C0B205E020F01C00C11021F0030108438DF82500616808729AF84B
:200FE0004A00042800F0E981092800F0E68117F0610F40F0EF809DF82200012811D1129817
:201000000078052800F0D88003280AD1BDF82A0024F06FFD28B1218D08A815AA002301F074
:20102000CFFB9DF8320078B99DF82200012804D112980078032800F09C8208A821461EF0B9
:20104000CBFC96E27F01012024F09EFA002840F090829DF83D0000286DD19DF82400BDF8F4
:201060002A10FD100028ADF854102ED13A0930D29DF82220012A28D0084600211BF0AEFC96
:20108000002620B14079012816D0022814D0BDF85400B4F8441020F087FB28B1807823F004
:2010A00088FF08B1082807DBBDF82C0024F021FD18B104208DF824000126BDF82A10002EF1
:2010C00008BF022272D09DF824006A0838BF002300D340230DF13D021BF0BAFC30B16168C0
:2010E000087848F0200800F03F0008709DF83D0040B1BDF82A1010A820F03CFC48F0400837
:20110000ADF854009DF82200012806D0BDF82A00BDF82C10002217F047FF68082CBF402224
:201120000022BDF82C10BDF82A0015F029F908B148F0200833E09DF840009DF84110119A04
:2011400022F006F800282ED09DF8410038B9BDF82A00ADF8540025F076FB00BB1DE01199D2
:201160009DF8286001EB400030F8020C002EADF854000CBF082110219DF8270008B10831F6
:20118000C9B29DF82500002200B1012266688918491CCAB2905D401E905548F0400823F011
:2011A000F1FC8146A8E0BDF82A100B22BDF82C0000231BF059F9DCE1218D08A815AA002379
:2011C00001F0FEFAD5E1C046BC800200E4020120E404012078084FF0000967D39DF8330052
:2011E000B4F828B0C04D494616901E20EA79169B934206D1BDF82C302A88934201D1AE789B
:201200002EB9401E05F1080501F10101EED11E2921D0AE79E6B1BAF84810584623F044F8E6
:2012200008B1761EAE71BE4833210279FF2A02D00288934504D0491E00F12400F5D102E018
:20124000A879401EA871A8794828A4BF4E46AE7127F060072AE023F095FC81469DF8320095
:2012600028B9BDF82C00218D814202D11EE0BDF82C00BAF83A10884202D19AF80600A8B1FF
:20128000218D08A84A4610F0DDFA58B1380932BFBDF82A004FF6FE70401C48F00408ADF877
:2012A000540003E027F020074FF00009B8094FEAA71510D394F8460094F8476094F94830CE
:2012C0008DF81000E26B8DF8116004A98DF8123008A804F037FF68080ED3218D08A815AA7A
:2012E0004B4601F06DFA5FEA000905D012980078012808BF48F01008BDF854104FF6FE70B0
:20130000884208BF4FF000099C49C97E012927D1628E411C914223D0228D914220D0BDF86C
:201320002A10401F88421BDDBDF82C00904217D025F089FAA0B10179012918BF02290FD149
:2013400001218DF810104088ADF81C0004A81EF06DFE28B105A81EF0B3F908B120F0EAFC29
:2013600037F07F0000F00581B9F1000F00F00181208918F025FE071C00F0FB806168228950
:2013800024F00CFC002605969DF822008DF81000CDF80090CDF8048004AD0296BDF8541024
:2013A0000395228D237A384614F09EFC002800F0E080384620F05EFBDBE04946BDF82A00A5
:2013C000098881420AD020F0F5FA022806D09DF8250000F00300012840F0CB809DF82200D8
:2013E00098B112980178042904D19DF83C10022900F090800078072804D19DF83C100429E9
:2014000000F0848003287CD0B3E094F846008DF8100094F847708DF8117094F948608DF864
:201420001260E26B08A804A904F08CFEA1E09AF84A00042818BF092840F09B80B80971D232
:2014400012986908C0F095800178042903D19DF83C1002295ED00178072903D19DF83C208A
:20146000042A53D003294CD00C2940F08280401C424A10F8017B0578164601215120D21CA6
:20148000F57025F051F93D4B3B49012658465C79067057B9002C14BF4EF660204FF47A706C
:2014A00051F8241000FB01F405E00846203000684EF6602444430320B4FBF0F441464FF405
:2014C00080400EF06BFA9AF8000002211DF02AFB68080BD2A8084CD39AF8000002212246C9
:2014E00025F0E7F945E0C046440200204FF48040214616F085FC4FF4804031460EF04EFAB5
:2015000037E008A8002112F017FA32E008A81AF0B1FA2EE0002008A90BF018FD29E0C0465B
:201520002C10002094F8460094F847709DF832508DF8100094F948608DF81170012D8DF8A0
:2015400012607FF46EAF208DBDF82C1088427FF468AFBDF82A0020F02DFA022808BF8DF80B
:2015600032805EE7BDF82A0001E0BDF82C001EF08DFF17B0BDE8F08F98800200E40401202B
:20158000B94A2DE9F04F0846ADF14C0D11780F90000C80F067849246B44D0F9A6878920B20
:2015A00080F03184022813D10F9A520810D39AF850000F2807D19AF84A0020B1012802D079
:2015C000002020F09DFF0F9880F0010000F06ABC0F9A920980F04C83DFF89892DFF898829C
:2015E00030F0010740F0BC820F9A520980F03D820F99C90980F0C4819D490F9F0A78390A9A
:2016000080F0AD813946490A43D23946090B2AD20F999AF80370490B1AD20F99C90BC0F09D
:201620009F824C46A06A70B1297D01290BD18047E06A00B180479AF800004FF480414FF4BE
:201640007A7225F036F90F9880F4804000F02ABC27B100208AF803001FF052FF0F9880F4B1
:20166000805000F01FBC1FF04BFF687C01280BD1A97C49B19AF800004FF47A7212FB01F2AD
:201680004FF4006125F015F9384680F4006000F009BC24F095FF4FF6FE7B834500F05B8182
:2016A0009AF832008008C0F0568100263446304623F00AF8071C19D03879012816D0022836
:2016C00014D0F879411CF9719AF88B1081420DDABC727C72388822F011F9388801A923F0A2
:2016E00096F901A81DF0ECFF20F024FB761C332EDDDBA8F11C0614275D46119436F81C0F49
:2017000085420CD0307B9AF88B40411C8442317305DA1198B0747074308822F0EFF87F1E79
:20172000ECD14C46032104F13C0010F8047F0FB17F1E0770491EF8D1B04C332605F1010921
:2017400034F8240F81451FD001208DF804006788ADF8107001A81EF069FCA8B1A8F11C0588
:20176000142735F81C0F2188814208D0BDF80610814204D002A8A91C24F000F910B1284685
:2017800024F08EF97F1EECD1761ED9D1119D2C46284622F099FF48B1077937F0040705D15D
:2017A000807A23F006FC08B1641CE4B26D1C332DEEDB23F02BFB119E5FEA00080ED0354607
:2017C000284622F087FD28B1807C23F0F2FB08B1761CF6B26D1CEDB2A845F1DCA019C7B229
:2017E000002F4BD0B80018F0EBFB1090002808BF119F45D0BA00FF211AF0F0FA119E3546AD
:20180000B44218DD284622F05FFF031C10D0187930F004000CD1987A23F0CBFB011C07D08F
:20182000009718885A7A109B19F07EFA761CF6B26D1C332DE4DBB8F1000F21D0119C2046D3
:2018400022F048FD061C0AD0B07C23F0B2FB011C05D00097109B3088727C19F065FA641C87
:20186000E4B2A045EBDC0BE050010120E4040120FE090120E40201209C0400201198109088
:201880009AF83000002808BF4FF0620805D024F0CDF9C0F154005FFA80F80320B8F1600F2E
:2018A00098FBF0FAA8BF4FF01F0ADDF84090ABF1020BB8F1000F0EBF119D2025DDF844807D
:2018C000BA45A6BF3C1C45F040055446032014FB00F0801C8DF8050001A823F0BDFB4E46E8
:2018E000031C26D01869082104F01F02017045EA02014170801CA4B12246C01E361F16F826
:20190000041F00F8031F318809124170B17801F0070CF178521E01F0070141EA0C118170CD
:20192000EDD1A3F802B001209876184608F090FC00E00120E90906D2641EE4B20CB109EBF7
:2019400084093F1BFFB205F040052843B1D0109808B120F08FF80F9880F48070A2E21043EF
:2019600008D1B3480179012902D10021C170017121F0F4F91EF09EFE384680F0800091E2CF
:20198000B44C1E2600214FF006084FF00409A778002F43D07F1EFBB26079A37023F0B6FFEA
:2019A000071C3AD06BB9787B022808BF87F80D8033D087F80D803868407BF0211FF0FEFB63
:2019C0002BE0A3791BB9787B032812D025E023791BB3E078401EC3B2E370F3B99AF82500BC
:2019E000E0702079401EC3B22371787B032814D133B92046394620F0BDF80EE008100020D8
:201A000087F80D9024F0C7FE00F00F00401C38819AF8000020211DF01BFB0121761E04F11C
:201A20000804B4D19AF80000012910D040211DF079F895F82A00012813D1002085F82A000F
:201A400095F82B0016F0B0FE20F074F909E040211FF0F0FF28B99AF800004021642224F0E7
:201A600028FF0F9880F040001CE2084610211FF0E1FF30B99AF8000010214FF47A7224F08D
:201A800018FFBB48DFF8EC82417808F2AC54491ECFB217BB012141700020052123F09CFCB6
:201AA000071C1BD006253846052123F095FC0646388978B1401E80B2388158B97889C0084C
:201AC00002D3387B21F002FF7D733868407BF0211FF074FB371CE6D100E0477064274FF621
:201AE000FE7600252079A0B1FF2812D0401E2071C0B270B96079032805D160882188022241
:201B00001CF060FD6079012803D0268066806571A5717F1E04F10804E4D108F15A04082736
:201B2000207A401E2072C0B230B9C048214622F01DF890B9668025707F1E04F10A04EFD106
:201B4000BB4AC82112F8080F08B1401E1070491EF8D10F9880F01000A4E11FF07DF8E4E7B4
:201B60004C460F992778890864D20F992289890A40D20F99090906D301200F9F8AF80600E3
:201B800087F008008EE10F99C90A26D20F98400C38BF0020C0F08681C44C332501262079FB
:201BA00080B105280EDA607900090BD28DF804606088ADF8100001A81EF038FA10B102A846
:201BC0001DF07EFD6D1E04F12404E8D100200F9F8AF8040087F4803064E1022801D11AF052
:201BE000DBFABAF84800012119F0F2FA0F9880F4806057E1BAF8485004F108015020AAF872
:201C0000482020F0D7F82689142744466089854205D0864204D0204623F042FF00E0668167
:201C20007F1E04F11C04F1D10F9880F4007039E1CCE8002087B9BAF83E10012021F0BCFA8F
:201C40006878022810D19AF8000001211CF06AFF0AE0C0464402002001A824F0F8FD24F054
:201C60009DFC01A91DF03CF90F9880F0020019E1084620211FF0DEFE28B9DAF81000002867
:201C800008BF012616D024F0D9FF044624F074FC4FF47A716043B0FBF1F1DAF8100000284E
:201CA00008BF002004D088428CBF4FF0FF30081A46086AD00020042123F08EFB071C64D004
:201CC000FF254FF0FF3B06244FF001093846042123F082FB10903889864204D8801B83B2EC
:201CE0003B8113B14EE000203881BB7B012B02D17889C00840D3002B36D08DF804508DF8BD
:201D000005508DF806B03968086AC97F02AA11F071F94FF00008012808BFC8465FEA08002B
:201D20001DD0788A40F08000ADF83600B87B8DF838007889000908D3BDF8360040F4807045
:201D4000ADF83600387B8DF83A007B6913B1187BADF8180001A9002202A804F0F3F97C73F9
:201D6000387B19F007FE0DE087F80D900AE0C046640F0120200100207C733868407BB721B2
:201D80001FF01CFA109F002FA0D10CF061F89AF800300020012123F01FFB18B118462021E1
:201DA0001DF056F90020042123F016FBB3B278B152460789147823F00FFBF8B9BB42AEBFE4
:201DC0000027FF1ABFB2204627B920211DF040F900200DE07A00202124F06EFD24F02EFFFD
:201DE000044624F0C9FB4FF47A716043B0FBF1F0CAF810000F9880F0200053E00289BA42A1
:201E0000D8BF171CD7E724F095FD294C0546201D00680746C0B157F80C1C9AF8000049B966
:201E20004FF400511CF06AFB08E0C04621130200E40900204FF400511DF00AF920463946E3
:201E40000022001D21F0BEFB284624F0F3FE2FB13846FEF78BFE384623F07EF90F9880F407
:201E600000501FE008461DF0C5F8071C17D0114920310A78FF2A0FD03C780B4600209442C1
:201E800007D0401CC0B2C200D1189A5CFF2AF6D102E0496838468847384623F05DF90F989E
:201EA00080F4004013B0BDE8F08FC0462C100020E40A0120987C02002DE9F04FC14DC24C8F
:201EC000DFF808A3C44E88465FEA1840ADF11C0D80F09E826F78DFF8F892DFF8F8B25FEA96
:201EE000580080F01B82384630F0010040F091805FEA980058D25FEA981044D25FEAD8303A
:201F0000C0F087800120022122F0CAFBC5B20DB3E80018F055F8071C1DD0C04C82464FF058
:201F2000010933262079012818BF02280DD18DF804906088ADF8100001A81EF077F820B1F0
:201F400002A9504624F0DCFC8246761E04F12404E8D100E0002797B175B10F204FF6FC76C7
:201F60008DF80C001F24ADF8046001A92A463B46C248009415F032FC38461FF07BFD88F497
:201F8000804000F00DBC207A38B92078062802D1072023F087FE23F06FF9E07910211DF0D3
:201FA00057F888F02000FBE3207AE8B92178E079082917D123F0F8FA092023F073FEBF485D
:201FC0000078052806D0072809D10720012105F0D3FA04E0012022F067FC1BF0C1FF23F01A
:201FE0004BF913E010210FE024F0DEFAEF2803DB002022F059FC09E024F0D6FA1030C0B2A3
:2020000024F0E4FAE07901211DF022F888F00200C6E3CE48CE4B0668B3F900005FEA58110E
:2020200080F04E815FEA181028BF88F0080080F0B7835FEA582080F0D1805FEAD80080F0CC
:20204000B78037F001001CD15FEAD81019D32069A0B116F071F92069076820691FF00AFD36
:2020600027615FB1FA8802E0F888801AF8803F68002FF9D1E079402124F01EFC88F0400092
:202080008EE35FEA182064D25FEA98205CD2C84C5FEA18302CD25FEAD82027D3142017F0D0
:2020A0008FFF071C1FD0002524342E46207A012812D10097042029463246142320F0A6FB5F
:2020C00050B9206838606068294614223B467860042021F0DDF926726D1C0C34C82DE5DBF0
:2020E00038461FF0C7FC88F4806059E3002057E3182017F065FF071C23D000252E46207AB2
:20210000012812D10097062029463246182320F07DFB50B9206838616068294618223B4630
:202120007861062021F0B4F926726D1C0C34032DE5DB38463146182219F050FE38461FF07E
:2021400099FC88F400602BE319F000F888F4007026E31BF005FF207805281DD1E0790421CA
:202160001CF0E0FCE07904211CF0C8F9062023F099FD687830F0010007D15046007800F086
:202180000700022801D024F0FFF81FF0D3FD18F0DDFF1EF08BF801E01FF0CCFD012021F0F3
:2021A00055FC0320012105F0E7F988F08000F7E2FF20032120F00AFE24F00EFAC249012040
:2021C0000860FEE7E4040120C4030120501A0120500101203C0501204C1A01204A4692F8C1
:2021E0004A00082818BF042845D124322120742124F09AFABF4E6878716832880024B146DD
:20220000A2423DDC30F001002DD1044CFF25002694F82100802822D102E0C0462C1000207C
:202220006788ADF8067023798DF80830A1798DF80A1062798DF809202088ADF80400E77948
:2022400084F82150237D8DF80B70A7698DF80C3031461022032001AB049721F019F9761C58
:202260002434332ED4DBBB48006800B180470020022120F0ABFD88F4807091E228040120EC
:20228000A30003EBC403CF5C37F07F0C13D017F07F07CF540B4405D101A8FF210C2219F051
:2022A0009DFD01AB012021460C2221F0F1F86878D9F804103288641CA4B2A1E76F060120B5
:2022C000B0F1FF3F37465C4602D1B8480078A0805FB17968087818B1486800781AF088FDA4
:2022E0003F68002FF5D1B4F90400B0F1FF3F02D0C0B21AF07DFD24F063F9AD49088023F0E9
:202300001DFC687C012806D14C4620784FF40061642224F0D1FA88F0100041E2012023F0AE
:20232000C1FC3046677801793546122201F0070A11F0070F16D1022F0CD0012F12D108201A
:2023400023F0B0FC24F020F80BE0C046C00A012040050120082023F0A5FC0020014612F00B
:2023600031F90246BAF1010F18BFBAF1020F45D107B3032F1ED0012F40D1BAF1010F3DD1A3
:202380000A2023F08FFC4C4620784FF480611CF0C9FB502005A922F073FABDF81400A4F855
:2023A0004800BDF81400002118F012FF2DE0C046E0E8002023F0A8FF002818BF032F16D105
:2023C000022023F06FFCB749E06809781CF04AFB0246A879000911D28AB959464878401CF0
:2023E000C0B20428487004BFBB48E06006E024F0D2F90146012012F0E5F802462AB1E079F9
:2024000001214FF47A7224F057FA88F00100C7E1DFF8CCB2BBE10646B04A337827781168EB
:2024200068781A46521E00F08D81521E00F09480183A00F0A681B93A00F09F812A3A00F0BA
:2024400083801B1F77D05B1E6ED05B1E54D05B1E3CD05B1E2CD05B1E40F0968120BB707F20
:20246000DBF8109000BBB9F1000F06F1050A1BD0BAF1000F18D04F46B81C5146082222F0A6
:202480005BFE18B9FF68002FF6D104E038461DF079FDDBF81090B9F1000F05D19BF800003B
:2024A0004FF400611CF03EFB304622F005FF6BE1012818BF022840F06781307916F074F9FD
:2024C0001FF038FC60E1C0467C052043002840F05B813079012800F05781022806D0042894
:2024E00040F05281304618F001FA4DE1304612F0B7FF49E1DC0A0120012840F045817088BC
:20250000002840F04181301D01A921F0D7F8012840F03A8124F054F8ADF80C00361D0296BA
:2025200001A816F0BBFB2FE1002840F02D81304611F0F2FC28E1012818BF022840F02481B3
:20254000304608F031FD1FE1002900F01D813046884719E13C090120012818BF022840F029
:2025600013815846C0795E46072818BF082805D1237A1BB9012104F0FFFF2778032F00F0FA
:2025800093800A2F16D0042F1AD00D2F18D00E2F16D00C2F14D0002F00F0F6801DF086FE60
:2025A000E07910211CF054FDEEE0C046671B0120E00301208048007800F00700012873D016
:2025C000277A6078002F35D10020E0720746F7701FF01EF8F8B120780D281CD00E281AD080
:2025E000062023F05FFB70480078000904D34FF4004001210DF0D2F9687830F0010007D1F2
:202600006E48007900F00700022801D023F0BCFE1DF04CFEB8E06878022803D108200121B5
:202620000DF0BCF9052023F03DFB42F2107022F013FEA9E0E17A01280BD003281ED16878BF
:2026400002281BD1594900260E7001270320677113E0491CC8B20428E07204DB54480078B8
:20266000012809D00AE0534800884FF6FF7181421CBF0426A672E8D10020607021F08EFA74
:2026800020F07CFC48480078000902D3287D01287AD16078032877D1082001210DF07EF9AA
:2026A00072E0C04699060120207A002848D1E07910211CF0CDFC1EF0ABFF98B968780228B5
:2026C00003D1082001210DF069F9052023F0EAFA01201FF0CFFB57E000F8FF0728070120E2
:2026E000680601206F78207837F001070AD10A2808D13149097801F00701022902D02B4A51
:202700000821117003280BD11DF0D0FDF079022806D1012021F09AF90220012104F02CFF9C
:20272000062023F0BFFA687830F001002CD12248007800F00700022826D023F025FE23E077
:202740000020C6E7022F1FD1012818BF02281BD123F0A8FF28B113F09BFBA8B168780228E6
:2027600008D023F0D5FF00280CBF002001201FF099FF09E019F010FD06E0304605F0A2F8D5
:2027800002E0304606F082FC069822F0E5FCE0791CF030FC002806907FF43DAE88F4004073
:2027A00007B0BDE8F08FC046521A01209A010120E006012098010120501A01204C1A01201C
:2027C0002DE9F04F064693460020ADF13C0DABF80000B06A099303460078884623F024FD5C
:2027E00048B1708904461FF0E5F8022804BFABF80040B36A01D0002009901878C84DDFF8BE
:202800002493401E0A2800F20B84DFE810F02F03B3020C04A0028D0151010904BE0088005D
:2028200066000B00BD4C207D012840F0F9835B1CB06913F8015B1F7824F032F8002800F0C8
:20284000F7830379002B00F0F383032B80F2F0830E2D1CDCDFB9D04907752DB901EB850126
:202860000A6BC261096B0AE001EB85010B6B9A01A2EB8302C2610A6B9101A1EB82018161B2
:20288000012180F820101FF055FA002500E001250320B689E4788DF8190006A822F0DCFBF2
:2028A000071C00F0C58338690C2100F8011B00F8015B04700124BC7723F040F9786204A9E8
:2028C000304622F0A4F810B17C7704A838627E80BC76384607F0BCFCAAE35C1C207820F0D0
:2028E0001F0700F01F00012840F09A83641C04A8214624F005F8284604A95D3023F03EF898
:20290000002800F08D83002F40F08A830834A2786178207801EB022120F0B0F988E3688F32
:202920007189884240F07C835C1C14F8016B04A8214623F0E5FF284604A95D3023F01EF8D9
:2029400006F01F0726F01F06002800F07183002E40F06E83780017F033FB011C00F0688320
:2029600067B184460834384663782278401E04F1020402EB03222CF8022BF5D100910EF035
:2029800058FC08461FF076F852E35C789A1C34F07F0704F01F0E40F04B83377F03201EFB9E
:2029A00000F0801CC1B2B94240F04283002714F01F0F04BF4FF6FE7C614618D0D9789B785A
:2029C00070464D4603EB012C5378117812F802EF01EB03213EF0770340F02A832B888B422F
:2029E00008BF0EF00707521C401EEDD1BFB960464FF6FE72824212D004F06002602A0ED043
:202A00004D462A88A30907D2E30902D2904203DD0EE3904203DD0BE39142C0F20983B0899F
:202A200023F011FF002836D1B0894FF6FF7121F03BFC041C14D120F011FD041C00F0F88261
:202A400000211C2219F0CAF9B0894D460E35208028886081AA23A374062222740121617472
:202A6000207C0C2805DB0620072F2074BCBF7F1CFFB2677400202073A01C22F01CFD002852
:202A800040F0D682307A002800F0D282B169A01C23F036FFCCE20021C171017A0C2905DBE9
:202AA0000621072F0172BCBF7F1CFFB24772BFE2484671890088884240F0B282307F02280E
:202AC00040F0AE82AA4CA01D00884FF6FE71814240F0AE82162022F039FA071C00F0A882CC
:202AE00001213970B07900280CBF081C02207870B06A4078B872000902D2B0891FF068FE3A
:202B0000B169B81C23F0FCFE0020F874287839461DF068FEB089E0808AE2C046E404012088
:202B2000500101208A01012070891EF043FF002840F076825F78B94987B10C2F03F1020399
:202B400080F276828C463D465A7818786D1E03F1020300EB02202CF8020BF5D14846758940
:202B60000488DFF8D892AC4200F0B280B37C002B00F05E823B1C0A974FF0000811D0A74A3D
:202B800038464146921E32F8023F9C4206D0401E01F10101F7D104E0688002000A914FF09F
:202BA00001082846002119F019FF00280B907ED0407901287BD10B98807910F0180F76D014
:202BC0000B984188384622F0AFFE10B9B8F1010F6DD109F55F794FF6FE704FF000080C9719
:202BE000B6F80CB0CDF820904FF0010A0D90C14611E0B8F1010F08BF4FF0010908D023F063
:202C0000CAFDC0B290FBF8F101FB08F1A0EB01094FF00008C246089D14271C3D35F81C4F5D
:202C20004FF6FE70A04213D0A34511D00C98214622F07AFE60B96B7C53B1072B08DA08F1AD
:202C40000100BAF1000F5FFA80F801D1C14521DD7F1EE3D1B34D332735F8244F0D98A04240
:202C60001AD0A34518D00C98214622F05DFE98B96B7A8BB1072B0FDA287901280CD00228C5
:202C80000AD008F10100BAF1000F5FFA80F803D1C14501DC0D9407E07F1EDDD1B8F1000F93
:202CA00002D0B9F1000FA4D00D980B994880B37C5A4C581EB074F77C00970A9D01950294B8
:202CC00001220392B189B269708915F02BFCAFE1B4890C2F80F2AC818846ADF81040BD4853
:202CE0008DF812700168CDF8148009B104A8884720461CF009FAC82803D14FF6FE701CF0DE
:202D000003FAC82880F2948109EBC00000F6CC05686808B11EF0AEFE2FB1780017F050F9D9
:202D2000686010B984E1002068606C80C2486F70007828706878002800F07A8168680028E5
:202D400000F076817A00414622F028FF70E1307F022840F06581099828B94D467189288853
:202D6000884240F06581099831460AF0EFF85EE1E4020120B5F8481040461EF015FDA8469B
:202D8000074608202FB17D781DB90621397007257D70B16A0A79CC788B794D7891F802A054
:202DA000CF7904EB02244A7902EB03296A0928BF1020AA0924BF0830C0B235F0700340F048
:202DC0003781327F904240F0338105F07005680938BF002006D306A8083123F091FD25F06C
:202DE00010050820A90907D3B16A091804A8083123F086FD25F020052046514621F0B2F861
:202E000008280DDA8D4B410001EBC001C9188879B84240F30D818F71002002E044010020D1
:202E20000420B8F83A10A14219D048B9B189484601222B460EF06CFC28B1F9E020010020F2
:202E4000042840F0F58006A804AE009049463A46534601962046029512F0CCF8E8E0B189AD
:202E6000484601222B460EF053FCE1E0B5F8481040461EF099FC4FF00609041C03D06078DB
:202E8000002800F0CD80B06A817847780891C378017900F1050A03EB0120099040461DF072
:202EA000EDFC9AF8001009185FFA81FAB80928BF4FF00E0937F0780040F0B28007F0180084
:202EC000182800F0AD80307F814540F0A9804FF00009CDF800900899B0895246434619F026
:202EE000F1FD032800F09C80002807F078074DD117F0180F18D195F8310028B1B089414683
:202F000001223B460EF004FC09984FF6FE714A463B460EF0FDFB002838D14FF6FF70ABF82B
:202F2000000039E00810002047F00107780928BF47F00207B089394619F050FD90B1817910
:202F400011F0180F0ED0417901290BD154B14088B5F848101EF028FC20B1437813B160787F
:202F600098425DDCB089414601223B460EF0D0FB60B94FF6FF70347AABF80000002C0CBFFC
:202F80004946B169B089524622F034FCBBF800104FF6FF70884243D1012000900899B08995
:202FA0005246434619F08EFD099839461DF0E6FF698F81422ED1099823F045FC60B1007911
:202FC000012818BF022807D1099804A921F01FFD08E0C0460404012022F0B0FD014604A8AB
:202FE00023F08EFC307A012803D1B16906A823F087FC06A8009004AF0197B06A407840F0A4
:20300000300002900999089BB0894A4611F0F2FF48460CE0B06A80F805A021F0B3FD06E096
:203020004FF00009F4E70999304610F085FC099009980FB0BDE8F08FFE0401207A010020F9
:203040002DE9F04FAD4C04F12C000768ADF1540D17B1002087F84500DFF89C82002517F1C5
:2030600048030BD0BF6DA34E73612FB940460068D0F84C05804773695868706023F05AFCAE
:203080001390082014F086F91AF0E6F8464610B181A023F0CBFD1CF0C3FB684623F03AF8F4
:2030A0000427284669468DF8007023F0ADF9206422F072FF09A823F0FFF8284609A98DF8B3
:2030C000247023F001F9A06322F070FF0DA823F003F928460DA98DF8347023F005F9A16B9D
:2030E000E06319B974A023F0A1FDE06B10B977A023F09CFD206C10B979A023F097FD306872
:20310000D0F8E00380473068D0F8180280473068D0F8F0028047404600682F460726A03083
:2031200001687B5823B11846804740460068A030761E07F10407F3D1D0F8B8028047EB20ED
:2031400023F044FAE06A2F4670B105A8FF21082218F044FEE06A05A9082221F0EDFF04F1E9
:203160002C06012818BF3768654A0CCA05A8391C80E80C0021D1082016F022FF5FEA0008F1
:2031800056D0A8F10206032723F005FB06F8020F7F1E4FEA20207070F6D13020F82706F8F2
:2031A000020F4146082204F1480088F8077022F0F5FC40461EF05EFC04E004F148000822DD
:2031C00022F0ECFC0120082105AA23F0A7FA04F14806002818BF092826D121F08AFC8008BF
:2031E0001DD205A8FF21082218F0F8FD07AFFF210822384618F0F2FD0120294608223B463C
:2032000022F0CEFF80B9384605A9082221F094FF28B930463946082222F0C0FC04E00120C9
:203220000821324623F080FAE22031461EF0C2FD21F05FFC400834BF2F1C0127314E55200C
:20324000012106F1320223F069FA18B917B1284620F0FCFB2C4EE22006F1400121F010FBCD
:2032600038461BF0AFFD05A82946102218F0B6FD707830F001004ED1DFF8908005A9102221
:20328000404621F059FF002842D105A84146102222F084FC3FE0C04652616E646F6D5F73B4
:2032A0006565644175746F6D617469632829206661696C656400C04641455343434D206F22
:2032C00070656E206661696C656400C0414553454342206F70656E206661696C656400C0AC
:2032E00054524E47206F70656E206661696C656400C046C0D405012014010020D4DB002078
:203300001083020068060120E40401207880020005A820F06BFB6220102105AA23F0FEF9F7
:2033200028B927B16220102105AA23F0FDF905A82946102218F052FD384612F03FFD38468A
:203340001FF056F9384613F083F87078A8B905A820F04CFB40F20110102105AA23F0DEF9B9
:2033600030B92FB140F20110102105AA23F0DCF905A82946102218F031FD1FB12846012195
:203380001FF024FD282016F01BFE0028606400F04081206B616B221D1AF07AFDCA49087057
:2033A00010211BF055FE616C201D0860206B616B04F108021AF06CFDC2490968D1F84C139F
:2033C0008847616C04F108004860206B616B04F10C021AF05DFD0DF071FB616C04F10C00B7
:2033E0008860206B616B04F110094A461AF050FDB64F7870B18EBD70381D0180303006F113
:203400005001119007F1340023F07AFADFF8C08296F8230006F148032946FB604FF4B472C8
:20342000387008F5057018F0D9FC04F1340B04F1300A626CDBF80010DAF800003C2308F553
:20344000057C0C324FF6FE7E5B1E2CF806EBF9D1C2F8009004F114021AF01AFD9F4B9D494E
:203460007B629D4A08709E4B606CBA6004F11802DBF80010BB6204F114030361DAF80000F0
:2034800012921AF005FDDFF85C9289F80700022289F824204FF6FE70A9F81C0022F04EFB7B
:2034A000914811990560AF4823F02AFA4046FF210E22801C18F092FC8C488E4B83608E4A86
:2034C000C2608B49416005708C4B03618C4A42618E4939618B4B83618B4AC2618C4B7B6156
:2034E0008C4ABA618E488C4B8C4AFB618E4910618C4FD16009F1300097601EF0CDF81EF0A6
:2035000065F8984809272C307F1E40F8045BFBD14F46F87948F201011CF0F0FEF8794FF4F2
:2035200000411CF0EBFEF87948F221011CF0E6FEF87948F222011CF0E1FEF87920211CF021
:20354000DDFEF87921211CF0D9FEF87922211CF0D5FE606C12994161DAF80000DBF8001099
:2035600004F11C021AF094FC704F48F2150138701CF0C4FE387838211CF0C0FE6D4B6E4AD6
:20358000FB606B483A61616C786102234FF6FE72DAF8000087F8283004F11C038B61DBF886
:2035A00000103A8404F120021AF072FC634904F12003634A0870634F606CDBF80010C36140
:2035C000DAF80000176004F124073A461AF060FC65497378087023B991F833300BB10221E4
:2035E000F17148F202011CF089FE606CDBF800100762DAF8000004F128021AF049FC2070B1
:203600005149087022F0C4FF4870616C04F1280048621BF073FF12F00FFD139823F00AFB29
:203620000FF03EFA21F086FB26480068D0F8D40090F8430021F090FB22480068D0F85824D2
:2036400029460120904722F079FD40481D4F05707868C068007830B938460068D0F858247F
:2036600028460146904717F051FA3A4F3D703848058145818581C581058245828582C58282
:2036800005832B464583344C858307210360344A43603248257021F0A3F816F0BFFB1EF0AC
:2036A000E3FF1DF041FA7078022807D13078012804D14FF4004001210CF070F915B0BDE8DC
:2036C000F08FC04614010020671B0120E006012020010020800A0120892001004D81010021
:2036E000F9620200C40301204805012020090120DDC700004941020099D901003B2E0200BF
:20370000F14602006913020019470200D5690100D54401003D4B02009DA40000FC09012046
:20372000F1420100E9B40100193401001C070120152A02001540020031480200C40A012023
:20374000D00A0120751C020028180020701B0120D8180120691B0120681B0120EC00002069
:20376000B9690200D8030120680601202DE9F04F0446B54DB5480021ADF14C0D001D2E6831
:203780000768A0780C910146102910DC102900F0AC80002900F0AE82491E012940F2FD81BA
:2037A000891E00F05581491E00F0248144E3113966D0491E1ED0491E03D0491E00F042834E
:2037C0003AE3207967798DF81000E0788DF8117022F02CF8002808BF022005D00C3004A95B
:2037E000022222F0DBF90C988DF82000132108AB01223BE3204634460421C61C304621F0E0
:2038000069FE0C9F0121002C35D0A268904203D02468002CF9D12EE06CB3361D304622F00A
:20382000FFFEB778804657B92868844218BF251C2068286020461EF01DF90C991BE0B81C0A
:2038400016F0BEFB051C04BF10210C9F13D00C9828706F7061683A46A81C414422F09EF9B0
:20386000BE1C642012212B46F2B21EF0D1FD28461EF000F9FDE23170334612217770F4E268
:2038800020460126C41C8DF82160204622F0C8FE6F68A3780FB3B3B938680090686818300F
:2038A0000190787E0290B87E03903969BA8AFB8A381D08F0A5F98DF8210068681EF0DAF87A
:2038C0000C9868600CE03968E41C1A4609180846214622F063F90C9800E010208DF82100F1
:2038E000112132460DF12103C0E22546BD4C89462D1DA07815F8011C002937D0491E10D014
:20390000491E02D0481E67D064E0287822F08CFD002869D041680978E170007820710C98C9
:2039200054E02D7800285FD1E1200DF1230120F0A7FF9DF8230085424AD00126A670304631
:2039400022F024FC0C9809A98DF8240052201EF031FA28461CF05AFC002839D0657020781D
:203960003146642222F0A8FFBA202FE000283BD1E1200DF1250120F083FF9B4E06F13C079A
:203980009DF825103878884222D0DDF8308001255220A5700DF126018DF826801EF00AFA5D
:2039A00096F83C000A2805DD1B2803DAE12039461EF000FA8DF8265052200DF126011EF0E1
:2039C000F9F9404622F0E2FB4046A07002460CE00C9A0AE00220F9E7284622F021FE0C9ADF
:2039E000A97822F0FBFE00B901228DF822200DF122031FE210218DF82710E1788046DFB138
:203A00007A681278384691420ED03F683FB17A681278914205D038463F68002FF7D1022022
:203A20000BE03968016002E0B1493868486038461EF020F80C9800E001208DF827000DF182
:203A40002703CDF83480A5E0FC0A0120BC0A012001218DF828100C990D900C2204A818F02D
:203A6000BDF925460224ED1C8DF81840284622F0D7FDAF1CADF8100017F8010B8DF819008C
:203A800017F8010B22F0D0FC8146384622F0C8FDBD1C0E9015F8010B15F801AB15F8018B2F
:203AA0002E788DF82900700016F08AFA0F9000286CD06D1C4EB183463746284622F0B0FDBA
:203AC000AD1C7F1E2BF8020BF7D1B9F1000F57D0CDF8409015F8013BDDF83C903746AB46BB
:203AE0000C2FBDF8105011934ADA28461BF00CFBC82815D14FF6FE701BF006FBC8280FD1C9
:203B0000C34890F8CC38012100F6D40C0C981CF8082B9342C4BF131C081C491CC829F6DB59
:203B2000C74C4FF6FE7604EBC0046068668018B11DF0A0FF0C9860606FB17E00304616F065
:203B40003FFA6060002808BF102419D060684946324622F023F8C9486580007867700DF121
:203B6000290620701099CDF800B00E9A0196119BCDF808A004A8CDF80C8008F041F8044698
:203B80000F988DF828401DF075FF02E010208DF828000AAB0D9881464CE194F801B00121A4
:203BA0000228814604F103048DF82B101ED114F8010B03288DF8180005D0204622F030FD0F
:203BC000ADF8100004E004A82146082221F0E6FF083414F8010B8DF81900204622F020FD92
:203BE000A41C11E0C40A01205001012002208DF81800204622F014FDA41CADF8100014F8EA
:203C0000010B8DF819000C98ADF81A0014F8010B22F00AFC8046204622F002FDA41C0D90CD
:203C2000B9F1020F14F8010B14F801AB14F8017B8DF82A001CBF14F8016B06F10A0006D197
:203C4000204622F0EDFCA41C064606F11400B8F1000F80B240D0FA2830DD6C68002C3BD1B7
:203C600006F11C0016F0ACF904466C6024B30C9804F11C0504A98DF82B000C222560201D92
:203C800021F08CFFC4F810800D98A082E6829DF82A50257684F819A0A7760F23E376784CC2
:203CA000207808214FF47A7222F006FEB8B1207808211BF0CDF912E010200EE000940DF161
:203CC0002A000D9A019041463346CDF808A004A8039707F095FF00E002208DF82B002BF077
:203CE0001F0BBBF1200F40F0C4800DF12B03A1E0BC0A01204FF0100A89468DF82CA05046A8
:203D000016F05EF9071C00F094805D48E41C7860207822F089FB00287CD120780C9E387015
:203D2000B04687F80C80142016F04AF90028B8606BD014F8011B017062782178A61C01EBD0
:203D40000221418031787278B41C01EB02218180817914F8022B01F0F00102F00F020A43A7
:203D60008271B96814F8010BC871BD68EB79464673B1580016F024F9A860B8688568002DE8
:203D800008BF564604D03046BA68D179814231DC2078B9680873BD682B7B73B1580016F0B9
:203DA0000FF92861BD682B69002B08BF564606D0641C4046297B814210DC102E2BD1A868B2
:203DC00010B11DF057FEBD68287B18B128691DF051FEBD6828461DF04DFE1CE062782178E8
:203DE0002B6901EB022123F81010BD68A41C421CD0B2DFE7637821789268451CA41C01EBDF
:203E0000032122F81010E8B2BEE7564603E0C04620010020B8268DF82C603EB938461DF0CE
:203E20003BFC8DF82C009DF82C0010B138461DF021FE0BAB4946DBE402200C9019E0C046AD
:203E4000EC0900200C988DF810008DF81100E07804A921F09DF89DF8117014219DF81000E3
:203E60008DF81D7007AB8DF81C00022264201EF0CFFA0C9813B0BDE8F08FC046FE040120AA
:203E8000671B01202DE9F04FADF13C0DC54C0B90C3480C91002147780E919FB137F00106F2
:203EA00008D0022F12D1207900F0F80141F00201204605E02046017901F0F80141F0010118
:203EC000017103E0207900F0F8002071261D3078402537F00102657100F00700307005D1BE
:203EE0008E20A0716FB940F0010009E0022F08D1AB4980200978A071012902D140F008005C
:203F0000A0710E99F170317150256572A020B071F171B072F172A089099140F43050A0813A
:203F20002174B2B1022F1CD1012019F00DFE28B9206820F00F0040F0020004E0206820F000
:203F40000F0040F001006FF30F1048F22021014306E0216894484CF21017084047EA0001B7
:203F60002160934B9149A0791F780A9381F8320067B90E981AF026FF8C4890F83200000984
:203F800011D30E9808A98DF8200009E0084690F83200000907D301200DF121018DF8210086
:203FA00052201DF007FF1BF0A9FA20F0A2FD800838BF0E9803D30E981FF048FD01200028E1
:203FC000DFF80CA30D9040F0D8800FF031FE5FEA000B40F0C380754ADDF83880212074211F
:203FE0002432174622F09AFB002859D12120414674223B4622F0D4F8002851D16B48408F8C
:204000004FF6FE7181424BD0684890F84A004FF00108082806D0042804D010F0A1FDDDF8CB
:2040200038803DE0C14642200DF122018DF822901DF0C0FE07F12F0143201DF0BBFE07F1D6
:204040002C0147201DF0B6FE07F11C014A201DF0B1FE07F11A014B201DF0ACFE07F124017E
:2040600028461DF0A7FE07F1160153201DF0A2FE07F12D0154201DF09DFE07F11801E1209D
:204080001DF098FE494890F83200000938BFDDF8389052200DF122018DF822901DF08AFE36
:2040A0000E9D17E0DAF804100E9AA80000EBC5000C23401881460090294601201EF0A6FB5B
:2040C00030B999F80000FF2804BF099889F800006D1CADB23248BAF800104078A942E1DCD6
:2040E00030F0010001D10FF0A7FC9548001D006800B180471EF000FCB8F1000F1BD022F092
:204100005FFA0A99888318B9307800F0F800307023484078022818BF012104D1234A09986E
:20412000032182F84A000A98393741703946143022F0E6FB01E04FF0090B804D0999184F14
:20414000A81C0180787818B91DF062FA38464078BBF1000FA94605D10E9904E01048DFF880
:20416000DC91407801210D9110490A9D91F83C20012707FA02F1E96087E00FF059FD10F054
:20418000EFFC0A4A21207421243222F0CDFA02A8FF210C2217F022FE0E9D574612E0C0467C
:2041A000E40401204C1A01200000FFFF50010120C4030120294601200C2202AB1FF068F93C
:2041C0006D1CADB23888A842F4DCB848407830F001000ED102A8FF21102217F0FFFD0E9D1B
:2041E00003202946102202AB1FF052F96D1C332DF6DB5348006800B180471FF08FFF099881
:2042000006220E99ADF8100002A817F0E7FD142015F0D6FE5FEA00081BD0A34810300768A2
:20422000A7B103270225A8B202A90622404421F0B5FCAD1D7F1EF6D104A94046022221F0CC
:20424000ADFC4C201421424622F06EFA40461DF011FC182015F0B4FE071C10D00E9D18229B
:20426000294617F0BBFD0620294618223B461FF00FF96D1C032DF6DB38461DF0FBFB17F097
:2042800013FF8A48DFF8B49040780D99864D012966D1B44F2437E8B1012807D002280BD190
:2042A000307800F0F80040F0020004E0307800F0F80040F001003070A34820F08BFE00284B
:2042C00008BF09980BD00A9A04210320917206E0DC0A01203178022001F0F8013170DDF894
:2042E000288088F8010022F056FA0B996F4E00F07F000818643080B20E90F06B0221C8F8A1
:204300000C00FF201EF062FD96494FF6FE70431C48870E46F0870998A1F848301EF048FE74
:2043200062484078012810D10C9801280AD0099902A8082217F052FD02A804E0100A0120D5
:204340003409012009981DF015FD212074213A4622F0EAF9099802211EF038FD534840789A
:20436000DDF834A018B9A08940F00100A0812F6987B9122015F024FE0646002E2E616ED0D0
:204380004FF6FE70B61F0327411C26F8060F7F1E7180FAD1BAF1000F61D1099906AB4C20D7
:2043A000022221F0FDFE002852D1BDF8180000284ED004284CDA182015F002FE03274FF077
:2043C00002084FF6FE7B0646099C2B691FFA88F14C2006221B1921F0E3FE78BB2869015B24
:2043E0008B452BD056B300962018099A4188182306201EF00BFA30692A6900F2E93333616D
:204400001019418805F11402880000EBC10029691350081973694188880000EBC1008018E3
:2044200029694360081941881822334606201FF02FF809993046182217F0D0FC7F1E04F197
:20444000060408F10608C0D116B130461DF012FB164B099971200822483321F0A1FE13481F
:204460004778381C06D121F069FB21F055FF0F48477817B121F048FF18B10120E870099E59
:204480002E713248324EC9F80C00C9F810607FB137F0010003D120F0B3F82F480BE020F02C
:2044A000AFF82E4807E0C046CCE80020E404012020F0A6F82A482749BAF1000F086019D07A
:2044C000284890F86500A8B92748407890B9DDF82480622102AA404618F068FB02A84146E4
:2044E0001FF078FC404614F05FF902A81022414617F074FC0A98006950B10A9C1034076818
:2045000020681DF0B7FA0A99384600280861F6D10A9A099F01200146107002F109045772DF
:204520008520093222F0FAF828B9852039460122234621F035FE0E9821F040F920F034FB93
:2045400050460FB0BDE8F08F1407012001F00000E9630200C808012091780100995402007D
:20456000F181010050010120E40401202DE9F04FBE48C84CADF1340D069025694068012111
:204580004FF0E047C06809934FF000080170C24808921F4080F800804FF0020000EA020011
:2045A00008BF002840F0E682DFF8F092DFF8F0A21E4611464FF4803018EA060700EA01000A
:2045C00008BF002833D141464FF4003011EA060700EA020008BF00280ED137464FF48000EC
:2045E000394000EA020008BF002800F0B78285F8048019F0B9FDB1E285F80480EB201EF0D1
:2046000091FE4A46514682F800800878862801D11EF00AFF22F08EF9E1690A6882F8048080
:204620000968E16122F006FB21F09AF996E285F804801EF0DFFE81262778A4F80C8099495C
:20464000A770994D0860994B2E70FF221A702169069E087A801E81B230684A46D0F8000156
:2046600082F80080C0890B918842C0F26B82E1690831096804F1180001600426A6810B989C
:20468000657EA17E04F11902C01E80B2069EE37E0B9005EB01205178C1F301193168608136
:2046A00001F1B80CDCF80010237109780792002908BFB9F1020F00F04582B9F1020F00F3A2
:2046C000418219B110F0070F00F03C82667800F00705AD1E022D08BF002E00F0338231B139
:2046E00051460978862902D1002D40F02B82001300F00200022864DA35435AD1DCF81C0016
:2047000090F88300022851D0E1690C31097805A801700527A78122F00DF95546064628782A
:20472000862840D106980068403001680F6837B9D0F80C05804706980068006C07689DF95D
:20474000140022F035F9787706980068016C096881F81E80006C9DF914100068C1773046DF
:2047600022F068FA2679678922F0E4F851460A7807F01007862A15D1BA4D05F11E031A88CB
:20478000521C1A8087220A7022F054FAE879B04206D11FB9404615F043FE07E01B20FAE7BD
:2047A000E920F8E70646304622F044FA21F0D8F8CAE151460878862803D11EF035FEA7787A
:2047C00066788FB186B9012F00F0BC816089022F03D110F0070F40F0B581032F05D100F0BD
:2047E0000701032901D0ADE16089010980F0AA81011301F00201022902DA810A80F0A2816B
:2048000007994978C1F3810BBBF1010F4FEAA1110A9100F09781012900F09481B9F1020FC3
:2048200014DA00F00701012918BF03290ED1BBF1000F0BD10A9F002F00F084810699096812
:20484000AC3109680F78002F00F07C81BC49B9F1020F0DD00A9E11F80B708A5DB918CFB265
:204860005EB3C10929D3BF1E12E0C046140100200A460A990BEB0207891809793A79521825
:20488000C109D7B214D20A995BEA010615D0BF1CFFB212E0B4180120B40A0120711B012014
:2048A000741B0120501B01206F1B01202D1A00200A995BEA010608BF02270B9AC0F3002152
:2048C000781A61718242C0F23D81069E1046C01B4018316880B2D1F850122081743080B2A6
:2048E000884700286678606100F02C814146742217F074FA84F8038062891EB9C14902F036
:2049000020000870BF4861790678C446002E30D000292ED102F00700032808D0012828D122
:2049200006980068D0F8D40090F882600EB306984068406906781EB121F060FBFE2815D0F7
:2049400006980068D0F84C02804750B906980068D0F84402804720B96289617994F803C0A3
:2049600007E00420E0706289617901E00420E07084466569268905F1740305F17400AB6594
:20498000079B686093F801A02E812089CAF301190029A5F85C001878AA8100F0780049EADA
:2049A00000004CEA000028744FF0FF06AE730CBF2079404685F83AB085F849000A9885F88A
:2049C0003000A089002FA0EB010086B2A68100F0B480E169E78068463A468919083114F082
:2049E00095FABF19B8B2A0812846017C4FEAAA0212F0030F02F003076D4601F0400B42D0E4
:204A0000B9F1020F434601D1C9090BD29DF801209DF8001001EB0221A0F844100DF1020576
:204A2000A0F84210814EB0F84410B6F846208A4203D04FF6FF728A4223D1032F14D06A78A0
:204A4000297801EB022189B24186B6F84420AD1C01208A4214D04FF6FF728A4218BF181C6B
:204A60000EE0C0460418002060692946323021F047FF60693B363146323020F07FFF083537
:204A80000346002B56D00798407886111ED06169B9F1020F03D0087CC00903D309E05BEAF7
:204AA000070306D16A782878AD1C00EB0220A1F84200032E05D068782A7802EB00220A85BC
:204AC00004E060692946283021F01AFF06990968AC310A686089167886B1B9F1020F0DDA89
:204AE00000F00702012A18BF032A0BD162692FB94F4BB2F842201B8893421BD100F00702FC
:204B0000032A05D0012A18D1886A90F88200A0B1D1F89C116069884778B90798817867698B
:204B2000407884F80380C1F3011100F078000843387402E019F018FB06E00BF087FC03E054
:204B4000D487020020F0FEFE21F0F4FEE1690A6882F804800968E16122F06CF80899099EBE
:204B6000202047460840374008BF002830D020F0B1FE2DE02F4991F90000002803DD91F95A
:204B80000000401E08702C4991F90000002803DD91F90000401E0870114640461E464FF058
:204BA00080770840374008BF00280DD0234991F90000002803DD91F90000401E08702048AD
:204BC0000121017021F0CEF885F8048019F0CCFADFF864C09CF90070B7B108994FF0E0472C
:204BE0000220374000EA010008BF002816D09CF90000002812DC06980068D0F84C058047CB
:204C00000CE0C046711B01200E48069F80F800803868D0F85824414608469047069840682C
:204C2000C06880F800800DB0BDE8F08FD40501201A060120B70A0120B60A0120B80A012092
:204C4000B50A0120B20A01202DE9F04F0446B54EA578F06A4FF0000BADF14C0D2946312974
:204C600011DC312900F0E280DFF8C882B24F142914D91C3900F06281491E00F01B811339E8
:204C800000F0E9807FE2323900F0BA80491E69D0491E012929D9891E17D074E2DFE811F0E6
:204CA0006402A502A102500299027302730224024E010A010D02F8018F0273028902DE0175
:204CC00073027302C901B801760240B1C06830B1E01C21F0A5FCF16AC968884700E00320E9
:204CE0008DF8380036210EAB61E201270028A8468DF839702ED0406A60B3204602A920F05C
:204D00009BF9342D044618BF584602D121F088FCA41C2578E0B902A821F07DFA641C0128A6
:204D20000DD1BDF80C00294622461FF06DFBBDF80C00012803D1E22021461DF03BF8F06AC5
:204D4000466A02AB93E803002A462346B04702E0042000E003208DF8390041460DF1390320
:204D60003D46A5E0002840D0C06900283DD0204602A920F061F9054602A821F04CFA0128A5
:204D800018BF584603D1BDF80C0021F041F90446284621F045FCAD788046F82DA8BFF72521
:204DA000A81C5FFA80F9484615F00AF9071C1AD0A4B9F06ABE1C02ABC469009693E803003B
:204DC00042462B46A047041C08D1584638704A4633213B467D7061201DF01AFB38461CF035
:204DE00049FE1CB90DE2102400E0032408A85946022216F0F3FF8DF82040332108ABFCE139
:204E000068B1806A58B104A9204620F015F9F06A826A04AF97E803009047014600E059463D
:204E200002A820F0AFFE32210422D8E160B1806950B1204602A920F0FFF8F06A826902AFD0
:204E400097E80300904700E003208DF83A0031210DF13A03ABE101258DF83B5010B30069BC
:204E600000B3204602A920F0E7F8042120F032FB5FEA000814D015F0A3F8F46A071C14D0E3
:204E80005946424616F0AAFF246902A803C842463B46A0478DF83B0038461CF0EBFD04E034
:204EA000052000E003208DF83B0030210DF13B032A46A3E1E41C8DF83CB0204621F0B0FBF6
:204EC000A846092D064609D0A01C21F0A9FB0746201D21F0A5FBA41D054602E0A778E57873
:204EE000241D242E03D12088352606AC069030461FF006FA7919884216DB27B93046294669
:204F000022461FF081FA30462946224621F00CFC30B9012E0BD1E22021461CF04BFF04E0A2
:204F20000A2002E0D4DB002002208DF83C0041460FAB3CE1671B01200C8802002646F61C9E
:204F4000304621F06DFBA9468046B8F1240F46D021F05EF80446082D08BFB67803D0B01C41
:204F600021F05EFB064640461FF0CAF986422BDA5CBB801B85B2F82DA8BFF725A81C5FFAA8
:204F800080FA504615F01CF8071C1BD0B81C59462A4616F023FFBB1C404631462A4621F07A
:204FA000FFF848B958463870524649463B467D7061201DF02DFA00E00A2438461CF05AFD7A
:204FC0001CB91EE1102400E002240AA85946022216F004FF8DF8284049460AAB0DE13520D1
:204FE0005946042207AB21F0DBF838B9BDF81C20584602210425ADF8262002E001205946FD
:2050000002258DF824008DF8251009AB08214FE7E01C21F005FB242802D01FF071F900E06F
:2050200058468DF82C00001213210BAB8DF82D00E3E0E01C21F0F4FA0546601D21F0F0FAF2
:205040000146242D03D0284621F0EBFB00E058468DF83F0012210DF13F03A8E0E078211DAD
:2050600070B1401E0AD10878012805D020B1522010A91FF005FC08E0522002E0022002E00C
:20508000E0201CF097FE8DF840000F2110AB8EE041460125087814F8031F8DF842500429B2
:2050A000A8BF022003DA37F8111019F03BFD8DF842000B210DF14203FAE6E41C207804281F
:2050C000A8BF02200ADA601C21F0AAFA267841460246087837F8161021F0EEFB8DF843002E
:2050E0000A210DF1430362E0E01C21F099FA0646601D21F095FAE779E51C0146242E19D013
:20510000B94205F1050510DD30465A4621F006FB8DF844009DF8440009280ED16FB1304637
:2051200039462A4621F000FB07E030462A4621F0F5FA00E058468DF84400072111AB36E066
:205140000127E41CE2208DF8457021461CF032FE30B938460821224621F0E6FA8DF8450095
:2051600003210DF14503FBE5E078284C30B1401E47D121F031FA01202060FEE721F02CFAC9
:2051800001202060FEE74FF0020B3AE094F903001F4F8DF83D003868D0F830240DF13D016B
:2051A000E020904714210DF13E038DF83E00012224E08DF841B00E210DF14103F7E721F0E4
:2051C000EAFA8DF830000C210CAB00128DF8310013E0E22002A91FF053FB0421082202AB91
:2051E0000CE00C4B02210A2208E05920062701218DF834000DAB8DF83570022261201DF020
:2052000007F9584613B0BDE8F08FC0467C05204314010020C0870200D249D14A03462DE90C
:20522000F04301F108009D78177800680024ADF1440D2A46402A2ADC402A00F0DE81202A3F
:2052400014DC202A00F010820A2A45D9103A00F03282521E00F02582D21E00F01982521E60
:2052600000F00F82501E00F0048263E1B2F1210000F0F481401E00F0EB81401E00F0DE81F5
:20528000401E00F0D481401E00F0C98152E14A2A11DC4A2A00F08E81413A00F0A381D21E4D
:2052A00000F09C81521E30D0D21E00F08B81521E00F084813EE1B2F14B0000F06881801E9C
:2052C00000F06181163800F04F81401E00F039817C3800F031812DE1121E00F0CE80521EA4
:2052E00070D0521E00F02A82521E00F01582521E00F00282521E00F0F281521E41D0D21E43
:2053000000F0DE81521E1DD014E1184606A9C01C20F05EFB2E468DF81E0048B99DF81800D5
:20532000BDF818708DF81F0038128DF8200005E00DF11F00FF21022216F050FD03220DF1E1
:205340001E031CE0DB1C5F782E460D4638B9684620F058FF012069460DF0B4FCA8603FB120
:20536000052F03D064211DF083FD03E0012129701DF012F88DF836400DF13603012235468F
:20538000EFE118468DF83740C71C384621F048F9BF782E46C0F304213FB9052903D04FF66F
:2053A000FF7181420BD1204607E0052903D04FF6FF71814203D14FF0FF30D64908600DF151
:2053C0003703DBE7202014F0FBFD061C00F0CD81FF21202216F002FD731C0120214608228D
:2053E00020F0DEFE751C071C18BF01272146042205AB842020F0D4FE083560B99DF8170049
:2054000028709DF8160068709DF81500A8709DF81400E87001E047F002078320214602225F
:2054200007AB20F0BDFE2D1D38B99DF81C002870BDF81C000012687001E047F00407ED1C84
:205440006120214601226B1E20F0AAFE08B147F008072146102262202B4620F0A1FE08B10D
:2054600047F01007012120223346672037701CF0CFFF30461CF0FEFA77E1264637F0010093
:205480008DF83C600AD10FA818F070FF9DF83C1080460E2000EB4100C7B201E0A0460E276C
:2054A000384614F08DFD5FEA00093DD0054621460822012005F8016B2B4620F071FE21F01A
:2054C0007FF80835072305F8010B001205F8010BA84A05F8013B1078A74905F8010B4B785B
:2054E00033F0010316D19DF83C0028709DF83C308BB141466D1C20469DF83C2082420ADDE6
:205500000A782A7031F8022B401CC0B212126A70AD1CF1E72E70672021463A464B461CF003
:2055200077FF48461CF0A6FAB8F1000F00F01D8146469EE7022418E122464720E02113461C
:2055400011E11846C11C4A7A087A00EB02208A7A8DF82E400EF0D8FD0DF12E0300E1C046EB
:20556000E5040120CCE8002018468DF82F400822C01C0146684620F011FB68461AF0A0F894
:205580000DF12F03ECE018460FF0C0FCEDE0D91C6846082220F002FB8DF80840CDF80CD0E1
:2055A00002208DF8090002A816F022F80CAB8DF83000D5E018461CF049FFD6E018461FF07B
:2055C00072FAD2E0DE1C307871781FF069F80222307000127070294630466FE0184612F068
:2055E000F3FFC2E0D81C21F01BF8ADF80200684616F02EFC01AE0822EDE7D91C01A8082205
:2056000020F0CCFA684618F073FBBDF802000DF122038DF8220000128DF8230016E0F5204A
:205620008DF827400DF126038DF826000EE0F52011460DF131038DF831003AE0F520FF2715
:205640008DF82A000DF12A038DF82B70022288E0F5200DF132038DF8320081E0F5200DF151
:2056600033038DF833007BE0F5200DAB8DF8340076E068462146092216F0B0FB16210922B2
:205680000DE068462146062216F0A8FB152105E068462146062216F0A1FB142106226E462C
:2056A0009AE7D8781CF02CFF11210DF135038DF83500012256E01A78D81C1021034651E036
:2056C00021F0BCFA054620F057FF2C496843B0FBF1F1684620F056FA09210422DFE7DE1C87
:2056E00062201EF00DFE01463246622021F01CF80EAB8DF8380033E0DE1C61201EF000FE99
:2057000001463246612021F00FF80DF139038DF8390025E0900A0120D81C04211FF0DAFE79
:20572000049084201EF0ECFD014604AA842020F0FBFF0DF13A038DF83A0011E0D81C20F0A8
:205740006FFFADF81A0083201EF0DAFD01460DF11A02832020F0E8FF0DF13B038DF83B009D
:205760000122294667201CF053FE204611B0BDE8F083C046C4030120E404012040420F00EC
:205780002DE9F04FCF48D04CDFF840830F46390CADF1240D80F06582790927D30023037015
:2057A000D7494370184620F065FFD649012020F061FFD549062020F05DFFD449072020F090
:2057C00059FFD849082020F055FF0522D6498DF80C300DF10D0020F0E1F94120802106229E
:2057E00003AB1CF015FE87F0100044E2B80828BF87F0020080F03F822068390931D217F406
:20580000706F08BF002000F03682380B04D3002020F008FC87F40067F80A04D3012020F0E0
:2058200001FC87F48067B80A04D3022020F0FAFB87F40077780A04D3032020F0F3FB87F462
:205840008077384617E22168884205D0016829601CF010F9286804E0016821601CF00AF93E
:20586000206808BB606858B1C27EC17E521E491ED6B2C17626B960681CF0FCF80020606070
:205880002668002E08BF00280BD04446207808214FF47A7221F010F818B12078082119F05C
:2058A000D7FB87F00800E6E1017B491E0173C9B20029C8D005460068D3E70546D9F8046050
:2058C00028781A280EDC1A2854D0401E00F06C81401E00F02B81801E00F0B581801E00F00F
:2058E0001781BBE1243800F0A881AD3800F09E81801E03D02A3800F08B81AFE1A87C09304F
:20590000C0B2804614F05CFB061C00F0A781A97800F8011B6988091200F8011B99F80C10B8
:2059200000F8011B99F80E1000F8011BB9F80E10091200F8011B99F8101000F8011B99F83C
:20594000111000F8011B99F8141000F8011BB9F81410091200F8011BAA7CA96920F01EF9E6
:205960004520FF21424633461CF052FD30461CF081F873E1B5F824A0E97B0AF114001FFAFA
:2059800080F820F02BFF002640B9A87B032805D0B8F1F00FD8BF4FF0810B16DD08F10A0013
:2059A0004FF0820B1FFA80F8B8F1FA0F0DDD0AF1100014F005FB061C00F0508106F11000F5
:2059C000A8EB0A0470601FFA84F8404614F0F8FA079020B9002E00F041813046A0E00446B5
:2059E000A87804F8010B6888001204F8010B287904F8010BA888BBF1820F4FEA202004F8EA
:205A0000010B1AD1A87B04F8010BA87B032805D0A8792070E8880012607004E0A91D20462E
:205A2000082220F0BBF8E87B083404F8010B287C04F8010B288A001207E0A87904F8010B52
:205A4000E888001204F8010BE87B04F8010B287D04F8010B687D04F8010BA87D04F8010B8A
:205A6000687E04F8010BE969204620F08BF8241DBBF1820F04D0002004F8010B504606E0F7
:205A8000002004F8010B04F801AB4FEA2A2004F8010B0E480078DEB10B4909680A4B3160A3
:205AA0004FF47A721E6008210F23337320F004FF20B106480078082119F0CAFAE869B06037
:205AC000706807E088040120FC0A0120671B012020465444A96A524620F060F895F82C00C6
:205AE00004F8010BA88D5FFA88F85946001204F8010B95F82E00079E2070442032E7C04664
:205B0000D1E3010093350200351902004D370200A878401DC0B214F053FA002800F09E80BA
:205B2000064623E785280200C087020029790B2000EB4100C0B21FF009FA002800F08E8074
:205B4000A9782E798DF80010EC788DF802608DF801400DF10301FEB1AA792C79EE880A706E
:205B6000022C4FEA26218DF804100DF1050113DB2A7A2C792E890A70032C4FEA26218DF83E
:205B800006100DF1070107D1AA7A6E890A7031128DF808100DF109012A7BAE890A703212FA
:205BA0004A701FF0D9FA59E0002E57D070788DF81500B0788DF816003078FA2819DC9DF822
:205BC000150000F01E00162811DA2C499DF815000D4600F01F00820050194068091D30B15E
:205BE0008958304688478DF8140028B9BEE6012000E004208DF814009DF8150020F01F00CA
:205C000020287FF4B3AE60200021032205ABABE66878AE78EC788DF8180006AB8DF81960AB
:205C200003228DF81A404420802103E06B1C4520C02101221CF0ECFB10E0F0783346401D67
:205C4000C2B26920F0E7F078401DC4B2A11E701CC9B220F0E7F8A41904F8010C48461FF01D
:205C60007BFA0748007819F0C5F95FEA00097FF424AE87F4004009B0BDE8F08F8804012045
:205C8000671B01202DE9FC47D44C0F460646F80B80F00C826078B90F80F0AC81B90880F0D8
:205CA0009F81DFF84C83F90A80F00281390B80F0CC80380907D2F80FC0F02E8227F08047C9
:205CC00017F05CFD28E220F035FE81461FF084FA002800F0B480082020F0C0FC002840F02B
:205CE000AE80802020F0BAFC002840F0A880684613F040FA012803D10098002800F09F80D9
:205D000094F84102002840F09A8000250126E8B220F0E2F948B1837A3BB1867290F9090005
:205D200006FA00F0C0B21DF0DFF96D1C032DEED3032084F8240004F5CE7020F0F5FD484618
:205D400020F078FFC34800252A460168056050F8081CD44940F8085C04F160001FF04BF981
:205D600040460068006B8047A168401A010BE06AC1F1FF3282422CBF08444FF0FF30E062BC
:205D800094F8300020B12069E16AB1EBC02F25D91FF032FA294600B13146081C1BD0C2482E
:205DA00040F6090101804580417B06F00F0221F00F010A434273017B05F00F0321F00F01D3
:205DC00043EA010202732946416020F0F5FA418811F4406FFBD084F83060E5621AF0D2FF99
:205DE000D1482946056002201EF038FF02201DF03DFD112011F036F8207818B960685030D5
:205E000020F0AEFDC948007810B90E2011F02AF894F8310020B184F8315005201DF026FD44
:205E2000C348A06284F82450B4F9B400B4F9B610884214BF0220072015F0C2F802E048467C
:205E400020F0F8FE27F008073AE720B104201DF00DFD0020607065681CF0C0FD38B128460C
:205E60002D6A6FF4807100224FF00073A847E06858B140460068006B8047E2686168801A56
:205E8000C860000BC8600026E660AA4904F1600000221FF0B0F80221D4F8A00084F82410DB
:205EA00018B104F1E00020F063FD27F4006707E720F040FD06461FF08FF9D4F89810002898
:205EC000894600F08480002900F081809A49042504F16000002284F824501FF08CF8304669
:205EE00020F0A8FE04F5CE7020F01EFD40460068006B8047E0604FF0010884F80180284677
:205F00001DF0CCFCD9F810006060D9F81000816AC90803D3436A294600229847404618F0ED
:205F200031FE606880F81980606811F0BBF86568D5F808A040F60A02D01F564600F1010CD0
:205F400000E01E46736833B119888A4203D0884218BF8C45F5D100217160727B08F00F03DD
:205F600022F00F0213437373D9F80C201288904224D06046904221D02B8F03B3E96305F14A
:205F80003802518095F8440001F00F0320F00F00034385F8443095F8450008F00F0320F0E0
:205FA0000F00034385F845307260707B01F00F0520F00F0045EA0001717300E0E1605046EE
:205FC00020F0FAF9514640461EF048FE02E0304620F030FE27F480679EE0C04668F20020B7
:205FE0000AF036F8D4F8A00008B927F0020793E08C010010514A116841F08001116020B114
:2060000004201DF033FC0020607020F093FC80464B480068016804208847216A81421BD13A
:20602000357ECDB1A568BDB1D4F8A8506DB1E968098840F60300884204D0E9680988401CDB
:20604000884202D106F1140001E006F110001BF071FD06E01410044040F6C411316171617A
:206060002062404620F0E6FD1CF0B8FC80B1356A30466FF4807100224FF00073A847D4F83C
:206080009800002808BF47F0020701D017F076FBF569002130464FF080630A46A84727F083
:2060A000005739E0ADF00100601A012020F042FCD4F8B06066B306F1280106C90A234FF099
:2060C000E0450B40154008BF002B21D106F1280191E8000306F1280595E8060006F12803B2
:2060E00022EA090221EA080183E8060020F0A2FDB16879B1B9F1000F08BFB8F1000F09D001
:206100003069B6F93010B5684B464246A84701E020F090FD27F4804727B104F1E000394646
:2061200020F026FCBDE8FC870000046086870200B546010035380100B9510200CC210840E7
:20614000E00100102DE9F04FADF17C0D1B91C0491C923CC9064610A83CC00EC980E80E001D
:2061600000248DF84240327F8DF84340B08D8DF84D40D6F828C0ADF844401746ADF85A00B1
:20618000F0898DF854706146ADF84A00087800F00303022B8DF8400000F3FD8123461D93B5
:2061A000491C1E9343083CD200F00C0EBEF10C0F0CD043093CBF11F8013B8DF84230BEF18E
:2061C000080F04BF01238DF84C3001D08DF84C40BEF10C0F0AD0737903F00303012B0CD14C
:2061E00040F00C0073898DF8400004E04D780B78891C03EB0523ADF84430430911D24D78AE
:206200000B78891C03EB0523ADF846300B784D78891C03EB0523ADF8483011F8013B8DF83B
:20622000433011F8013B30F07F058DF855301ED00B7833F003058DF8413040F0A88103F01A
:20624000030EBEF1030F00F0A28113F0030F01F101010ED011F8013B00F00305022D8DF881
:20626000573004BF11F8013B8DF8583001E08DF841401491A1EB0C017F1AFFB2BA42C0F265
:206280008681D21B8DF85470D1B28DF84D100F4300F08181C10907D370891BF08BFB0028C2
:2062A00040F079819DF8400000F00C012746091F08BF0127820932D301221E9279B3B28994
:2062C00020F07EF9904202D1F08D000A0DD220F077F9904221D0F18D080A38BF101C07D35C
:2062E0009DF8400000F003032DE07089ADF85A20804620F065F9BDF85A10884205D0404636
:2063000019F09BFC002800F04681A448026810A940469047002840F03E819DF84000F18D28
:2063200000F003030A0A0ED2C2090CD39DF8412012F0030F07D100F00C020C2A03D0082AAE
:206340001CBF01221D92DFF86082022B00F00081012B00F0CE8010F0030F40F01C81904818
:2063600090F82F00012803D1B579002D00F013819DF8540002221A900B0A9DF84240BDF8F2
:2063800046B0BDF848A09DF855E09DF857C0DDF850908DF86420B0899DF84350ADF85C00D4
:2063A00075D2454605F11C021468002F52D11D9F17B110A913F0ABFA7A484178022936D197
:2063C0000078012833D1B07C002830D070891BF0F1FA022801D0707948B37449B2893C20A2
:2063E0008B1F33F8064F944204D19C78F77CBC4200F0D180401EF4D16878891F3C234FF6B3
:20640000FE7731F8064FA74202D05B1EF9D1C2E00A80F27C8A700C228A8004211BF00AFB8A
:2064200028B9687804214FF4FA7220F045FAF07C1E9F00901C9D0197594C0295B07C1B9B50
:206440000390B4F8482017A910A811F02FFDA2E068850200307C002C8DF8560000F09B80C1
:2064600020F0AEF8BDF85C20904240F0948030791E9F00901C9D01971B9A02951D9B039140
:2064800096F8300010A9049017A8A04783E08DF820208DF822508DF82340ADF83010708966
:2064A000ADF818008DF835E0ADF826B0ADF828A0CDF82C901A9B8DF836C0327CADF82A303F
:2064C00035798DF83220B47C8DF8335096F832108DF83440324F8DF83810B7F84800ADF84C
:2064E000240096F830708DF8377006A805F08AFD51E01D9FB58937B1080A04D2284610A9D2
:2065000013F005FAB5899DF85400B6791030C0B21EF01CFD071C3ED07D81022038703E73A0
:206520007C709DF854203A7207F110057D609DF84000800928BF01247C72149978681FF0DC
:206540002DFB45466D1C287839461AF04BF922E09DF84100B189454624352B6810F0030FF7
:2065600010D110A807901248ADF8181006A91DF0FDFA80B1062141730068407B21461AF071
:206580001DFE08E03BB110A82246984703E08DF84D408DF854401FB0BDE8F08FC40801201F
:2065A00050010120E4040120E0060120340300201B0602002DE9F04F4FF0FF084146ADF11F
:2065C0004C0D0E910F914FF0000910914E46089609960A96AD4C0B9604F1300B0C96E06815
:2065E0000D96494611919EE0E068710306AA042320F0CCF8119903AA30461FF01BF802AA47
:20660000304601211FF016F83046022101AA1FF011F8069800F0FF0028709DF81900069FF1
:206620006870C7F30140E8709DF80E30AB702878FF2834D0BDF80C70FE2830D04FF6FF706B
:20664000B8422AD107A81BF03DFFE06871034FF088524FF4005320F099F8BA484FF40057A7
:2066600050F8041D3F1FBFB2B1F1FF3F07F1885201D1032FF4D810684FF0010A514600F017
:20668000FF03FF2B18BF8A46491C000A0529F6DB106007981FF06AFA5744EF8001E010201C
:2066A000E8809DF80A00BDF8087028719DF806302F81BDF804206B7129786A81E068FF29E1
:2066C0002AD0FE2922D07E291AD07C2912D078290BD0702904D00D99491CC9B20D9120E082
:2066E0000C99491CC9B20C911BE00B99491CC9B20B9116E00A990F96491CC9B20A9110E0B4
:2067000009990E96491CC9B209910AE00899B046491CC9B2089104E009F1010710965FFADA
:2067200087F9761CF6B2E578B54200F323810D9F002F38D10898022835DA0C98022832DA1D
:20674000099802282FDA4D452BD00C98C0B90898A0B90B980A99084325D01EF019F8854256
:2067600019DCB9F1000F14D094F83200FE211DF01DF8E5780120DDF8408015E0012013E06C
:20678000089860B9B9F1000F07D11EF001F8854201DC062008E0032006E00220EBE70220D7
:2067A00002E0119800E004200028A07000F0CC80401E49D0401E00F0AA80401E06D0401E55
:2067C00000F09880801E00F094800EE11DF0E0FF05460C2084F83C5015FB00B0817E84F87A
:2067E0003D10C07E84F83E000EF030FAE2782D1895FBF2F050432D1AE8B284F83200401C9D
:2068000090FBF2F15143401A84F831007C201CF0C9F8FF2810D17E201CF0C4F8FF280BD195
:20682000FF201CF0BFF8FF2806D178201CF0BAF8FF2808BF94F8310084F833000C2110FB90
:2068400001B0808BE0868FE00F9F08F1010090FBF5F184F832806943FF2FA0EB0100C1B287
:2068600084F8311014D10E98FF2804D10C200E9111FB00B004E00146880000EBC100584452
:2068800084F83310808BE086AFE0C046C01900203A46D0B2910084F8330001EBC2015944AC
:2068A000898B1729E18640F2A080C91F01AA89B212F058F99DF80F00C0083FD3119F0097E5
:2068C000BDF81220E18E94F833000323891AC91F01AA89B209F012FB002840F08680BDF8F3
:2068E0001010002900F081809DF8140019F054FF7BE0FEE7119EB54226DD304610F052FAAE
:206900006178E578761CF6B201436170F3E708F1010084F8328090FBF5F16943401A84F8FD
:2069200031005FFA88F010F03DFA6070FE215FFA88F01CF03BFF012084F83500119801F0AC
:2069400083FF52E00020001111986D1E84F831000C2184F8325010FB01B184F83300898BC6
:20696000E1867E211CF022FF94F83200FE211CF01DFF3AE00C2116FB01B506AA0423710386
:206980001FF004FF1199304603AA1EF053FE304602AA01211EF04EFE3046022101AA1EF0C9
:2069A00049FE0699163501F0FF0201F0FF00FF2A09D0FE2A07D07E2A05D07C2A03D0782A2B
:2069C00018BF702A0AD1119F47B9C1F38542032A04D19622B2EB116F3FF41EAE304610F0F4
:2069E000E1F9002860703FF4FFAD13B0BDE8F08F2DE9F04FC24CC44AE0790E46F108ADF14A
:206A00001C0D80F07281BF49330C07D3DFF8FCB24FF6FF7A9146AAF1010A42E00F78710BE4
:206A200027D2300A28BF86F0800080F0D581B0080BD2300B38BF0020C0F0CE81381C01D174
:206A40000EF04CFB86F40060C6E1012F18BF022F0CD168460021082215F0C0F9684610F0F6
:206A600009FE18B12078022118F0F2FA86F00200B2E1012F18BF022F10D1401E0AD0801E9D
:206A80000CD1607A022809D10120607200201BF0F1F903E0217A00201CF0DCFB86F4805068
:206AA0009AE1207818F0A6FA071C08BF86F4004000F092813D78D32D00F00B81E079A84200
:206AC00020D094F82F000A2D0BD08E480378002B40F00781092D40F004810021B81C884716
:206AE000FFE03871B9788DF812100322F9788DF814000DF112038DF813104F2080211BF031
:206B000087FCEEE099F801006D1E00F09080AD1E40F0E780012818BF022840F0E280BD78B4
:206B200075B36D1E40F0DD807D7820781DB31FF047FD4FF6FE720021824218BF0121081CAE
:206B400004D15846408F1146814209D010465D46ADF8100004A9A5F83AA053201BF02AF98D
:206B60001DF01CF81CF00AFA5946002081F84A0014F040FEB5E0022140F6B83261729DE0F8
:206B80007D78002D4FD11FF0C3FD002201460BF10800E1600D4602601046002D3FD10029C5
:206BA000E6D000280D46E3D080468D481EF012FA012809D0B9F830004FF6FF71814209D008
:206BC0002988884206D022E0854805F10C011EF0D5FEE0B1BBF83E002989884201D182451A
:206BE0000BD199F8010030F0010302D1EB7823B90DE0022801D12B794BB19BF836006979BD
:206C0000884207D199F80600A979884202D028461CF004FFAD69B8F10108C6D1A8E7AD69FC
:206C2000401CC0B2B9E700201BF03CFD59E0012818BF022855D17D7894F838003DB194F8C6
:206C40003710491CC9B2884284F837103EDB207A401E04D0401E36D0401E1AD041E01FF0BF
:206C600053FB78B994F8390000283AD1002102200D468DF808000246ADF8005068461EF081
:206C8000C7FD13E001201FF013FD014600F074FC27E0AB2000216A4619F0E6FCCDF808D02B
:206CA00004208DF80C0002A80DF0E4FE20784FF4805117F037FF207841F288324FF4805114
:206CC0001FF0FAFD0DE01BF015FF0AE001200021DCE7F88948F20201814202D138460AF0E7
:206CE000E5FE38461EF038FADBE65778217878B1401E6BD0C01E64D0801E58D06AE0C046E0
:206D000068060120E5040120E40401205001012094F82F00022F904601D181095AD2C1084C
:206D20002CD2800856D3042594F83000E571400850D394F832309BB9012F18BF022F17D19C
:206D40000127E01D00212A46A77015F047F80320E071384619F0FAFA38461EF07AFE05E04A
:206D60001EF072FD2846012100F006FC98F8017087BB2846002100F0FFFB2BE0E01D052526
:206D800094F8301005708908F3D394F832100029EFD10121A1700422002115F01FF8E571B8
:206DA000002019F0D3FA02201EF053FE12E0002084F82E00E0713222084604211FF07CFD00
:206DC00008E01EF041FD04200121D4E7012001461CF040FA86F0040007B0BDE8F08FC04675
:206DE000D80301202DE9F04FD14CDFF84893DFF84883080CADF1140D019180F0D38108465A
:206E0000400838BF0020C0F0D78167681FF016FF05461FF0B1FB4FF47A764FF6FF7268437E
:206E2000B0FBF6F081B267B13B887888CB1A9BB2984210DDC01A8242C8BF82B2FF68002FCB
:206E4000F2D14FF6FF70904200F09380207801211FF032FD8DE0B87902287DD01FF0EEFEDE
:206E600005461FF089FB97F838106843B0FBF6F0D34D38802878884266DD97F83600FF28B0
:206E800008D197F83800401C87F8380097F8370087F8360097F8356097F839200020012176
:206EA00001E0401CC0B282420FDD97F8365001FA00F385F0FF052B42F3D03618814097F829
:206EC0003600F6B2014387F8361097F83400B98F10FB06F2891A89B28842C7BFFF2087F8F1
:206EE0003600011C97F8360099F82220FF2818BF97F83A0006D140460078642510FB02F283
:206F000012FB05F0788046B9388D3E7A40F020003885386C87F82E600BE03A8D4FF6DF70F7
:206F2000104038853D6C87F82E6097F8342012FB06507862F879CEB287F82D0007F11000C9
:206F40007E8405F05FF810E0B87E97F82A10FA8BE9231BF097FD05E0387CFF2802D0B86911
:206F60001EF0FAF838461CF091FB2078012118F06FF8019880F001001EE12878012840F0D0
:206F80000E8195F8338095F813A06F6995F83100698802221CF036FF05F11C0405F1020BDD
:206FA00006460020002E02907BD1687F400876D3A87FCDF80CA01FF037FABA4605F11009FA
:206FC000071C60D01C2012F0FBFF061C59D000211C2214F003FFA87F69461DF0D9FF9DF826
:206FE00001000221307530461DF0E2FA6888317DB08095F83100FF22F07102FA01F070748A
:2070000078680078307495F83000B07495F8331011FB00F0303080B21DF098FF0746B7612C
:2070200027B930461CF032FB00262AE01A20387000237B701A467A80E0885946B880B81D33
:207040001EF05AF9E0783C4BF87303F1200000883882608BB88560897882A0783875207BC4
:20706000787599F80000B87599F80100F87599F902003876039A7A76C7F81CA007F13001F3
:20708000B962304600E000200028064600F08780274886F808800078012117F0D9FF002ED8
:2070A0007DD0307AA8EB0000B0F1FF3F04BF01200290307CFF285DD06078400828BF4FF0AB
:2070C0000008317DF07C4018404503DCF074FF2088407074B069B17C227D806A08FB0100D0
:2070E00021691EF05BFD029F317D727C012398FBF1F04843A8EB000003FA00F11143C9B2F0
:207100007174DFB1401CFF2202FA00F001437174B769B17C207D08FB0100B884707CFF282B
:207120000CD1307CB16919F05DFBFF20307421E0800A0120E4040120780101201FF07EFDAF
:2071400007461FF019FA204B204A4FF47A717843B0FBF1F0308093F8221010781F4610FB11
:2071600001F197F821006423401C10FB01F010FB03F07080F17C327DA8EB0100801AB0F1B5
:20718000FF3F04D0707CFF2801D0029F3FB1E175707C2076BBF80000214612F0B8FB284653
:2071A0001DF0DAFF0748007817F024FF051C7FF4E4AE019880F4004005B0BDE8F08FC046A6
:2071C00005050120800A0120E4040120780101202DE9F04FB64AB74CDFF8DCA20B46ADF19A
:2071E000340D90465178607805931A0C80F09C8031F0010709D11A46520806D3206A00B1BC
:207200008047059880F00100AEE11A46920805D301201F46E07087F00200A5E1022906D161
:2072200098F80010012902D11946C9085DD21846000938BF0020C0F0978150463230E76AC3
:2072400000780026B146000922D21FF0F7FC05461FF092F9236BB8F836204FF47A71684348
:20726000B0FBF1F098F825100690C01A824238D8B0FBF2F39BB29942ACBFDDB20D1C069BFD
:20728000B0FBF2F15143401A81B2581A206300E00125EFB1C846F878A8420ADD401BC0B288
:2072A000F87040B109F101061FFA86F93E467F680CE087F803807868002E82460CBFC4F826
:2072C0002CA0706038461AF0D5FB5746002FE2D16078B9F1000F04D100212163082117F000
:2072E00021FC059880F008003EE1A14B00263C244FF6FE71354633F8062F914208D09A886F
:20730000521E97B2002F9F8006BF19809D700126641EF0D126B104214FF4FA721FF0CCFA11
:20732000059880F004001FE117F064FE071C00F01881B87FC0B9788CE56A132815D1B7F854
:207340000290281C11D000260188894508D14568002E0CBFE56275601AF08CFB284601E07E
:20736000064640680028EFD1E56AB87A97F831102E46022853D1788856B13288904204D1B6
:20738000B27898F82530914247D07668002EF4D181460E46002D08BF002004D0012015B139
:2073A0006B68002B35D1B8F83810814237DD082012F006FE98F82510002830D0A0F80090B7
:2073C0008670C17000234360E66A86B9E0629AF83200000911D21FF031FC05461FF0CCF8E5
:2073E0004FF47A716843B0FBF1F0206300E06860504690F83200000911D3607808211AF0B5
:2074000019FB60B96078B8F8362008211FF051FA05E0401C1D4680B2C1E7F3709EE05548E2
:2074200005683878012806D0022840F09780384616F0CCF892E007F11004B81CBE89089442
:207440003B7E0690FA7C07967969099397F819B00A923C7F0B9107F11C0604F00C000C28B3
:207460000DD0B87F4FF0FE09FF2804D01EF0DCFF041C11D172E0002D70D06C6810E0B08811
:20748000FE211BF01BFB8146B9F1FE0F08BF01201EF0CAFF041C61D020781EF0C7F905466D
:2074A0004FF6FF7A11E020781EF0C0F905460CE0E4040120E006012050010120B078FF28B6
:2074C0004CD12D68002D49D06C68002C46D0AB68AAF1010823B9A3680BB1B3F8028007E030
:2074E00021780220984718B1B0F800801AF0C2FA3389227898450BD00AB913B908E09A45D7
:2075000006D0B3F5807F18DB4FF60240984214DD96F80280B27008980090099B01930A996C
:2075200002910B9A0392CDF810B0079B069A3046214610F053FF86F80280307800F00C00E4
:207540000C28BBD1B08849461BF0B8FA8146B9F1FE0F03D01EF068FF041CA4D138461DF001
:20756000FBFD059880F400400DB0BDE8F08FC0462E030020C00A01202DE97C43CD4C0E465D
:207580000146DFF83483DFF834936078491E00F04E81491E00F02281491E00F0E580C84AB2
:2075A000491E00F0B380491E6CD0891E2BD0491E40F07481052102288DF8011040F06E816B
:2075C000444694F82F00B6B1A07AE0710021A17242F2080008F0E2F994F82F00217900F00C
:2075E000DF0084F82F000D2084F82E0001B904201EF058FB52E140F0200084F82F00022695
:2076000084F82E604AE10025012E8DF801501AD0022813D11FF046F880B1052044468DF861
:20762000010004F12F01087840F0200008700820294608F0B3F90A201EF034FB444602208E
:2076400084F82E0019E018B909201EF02BFB6078022806D10820294608F0A0F904201EF026
:2076600021FB14F0E5FC44460D200421C82284F82E002078E5711FF01FF994F82F0000F0D9
:20768000EF00D1E00221012E8DF8011017D04446082130F0010084F82E102BD194F8320033
:2076A00040BB002552200DF105018DF805501AF081FB1EF0F8FD15F035F8284618E0002514
:2076C000484616460570308804F13002208683201FF02AF8032128461BF078FB60780128E1
:2076E00003D107201EF0DEFA6078444610B909201EF0D8FA0020E0712078042132221FF0E4
:20770000DBF894F82F0000F0FB008DE00121012E8DF8011004D0D0B902214846017016E027
:20772000002148461688017004F130022686022183201EF0F9FF6078012803D107201EF0E2
:20774000B1FA6078022802D106201EF0ABFA44460020E0712078042132221FF0ADF894F884
:207760002F0000F0FD005FE0012818BF022840F0958044462078042132221FF09DF894F874
:207780002F10E0685EB101210028E17100F090801CF044F9E0680028FAD1BDE87C8302206D
:2077A00084F82E0000258DF80450E57101268DF8016021F0020184F82F10522001A91AF0C9
:2077C000F9FA1EF070FD14F0ADFF28461EF06AFAE068002862D01CF021F9F9E700201EF0D5
:2077E000D5FC04250120207260788DF801507EB1002188F82E10012888F82F1003D107203D
:207800001EF050FA6078022802D106201EF04AFA44460020E0712078294632221FF04CF81A
:2078200094F82F0000F0FE0084F82F0036E0012818BF022832D1012E18D0012044460726C2
:207840008DF801004FF48051207884F82E6017F069F900201CF0FAF8002084F82F00207802
:20786000022141F288321FF027F817E0002003211BF0ACFA4446042132222078E1711FF0E2
:207880001BF80820002108F089F80020207220784FF4805117F046F9BDE87C8348460078C5
:2078A000002103226B468DF800000A201AF0C2FABDE87C83E4040120680601209606012063
:2078C000980101202DE9F0410646B948B94DF1890078ADF1380D0F46203F64D07F1E012FCA
:2078E00032D947F6DF72BF1A012F16D9213F012F00F28481002840F0818108352F68002F13
:2079000000F07C8142328A420CBF03200220B169727C097805F0C0FD70E1304615F09AFF8A
:20792000041C00F06B81207860B9608800218DF80810ADF80A00211D03A81EF0CBFD02A8DC
:207940000BF062FC204657E1307B002840F05681B16902A80C461EF0D3FF083414F8010B0C
:207960008DF8100061782078A41C00EB0120ADF8120014F8010B03288DF81C0006D06178EB
:20798000207800EB0120ADF8140007E005A821461EF0B6FF14F8080F8DF81E00304602A9E5
:2079A00007F0A0FE2AE1002840F02881707C77888DF80800337CADF80A70B4698DF8093005
:2079C00061782078A71C00EB0120ADF80C0039460DF10E001EF094FF07F1080414F8010B6E
:2079E00000268DF81600617820780796E41C099600EB0120ADF8180014F8010C8DF81A0098
:207A000070B19DF81A00400012F0DAFA0246079030B19DF81A0021461DF07AFD044601E0FB
:207A20008DF81A6014F8010B8DF8200068B19DF82000400012F0C4FA0246099028B19DF86D
:207A4000200021461DF064FD01E08DF82060A868C8B9502012F0B4FA0746AF608FB1314687
:207A6000502214F0BBF9384602A915F034FA40B1A9680120634F81F8400038881CF0D4FD55
:207A8000B0E0882065E090F84010012940F09480022780F8407002A9203015F01CFA28B9DB
:207AA00088204FF001088DF8340000E0B046AC68207EE16994F83220636B19F083FA84F89D
:207AC0004300B0B110FB07F000B212F079FA6064AC68606C28B988204FF001088DF83400AB
:207AE00007E094F84320606C05F1180152001EF055F894F83800E16BA27C636919F062FAC9
:207B000084F84800A8B110FB07F000B212F058FAE064AC68E06C002804BF88208DF8340050
:207B200016D094F84820E06C05F1180152001EF035F8B8F1000F0BD194F8431094F848003C
:207B4000084305D0304601460A4605F0A5FC49E086208DF83400BDF80A000DAF0224ADF894
:207B600028000AAE009748F2200201239DF809008DF830403146019002A819F06BFDA86848
:207B800098B190F8401002290FD18DF830400DAF41880097ADF8281040780190A86848F238
:207BA00020020123314619F055FD17F0DBFA19E0E50401203C050120BDF80A6088200DADEB
:207BC0008DF83400022700950AA948F220028DF830709DF80900ADF828600123019002A8D0
:207BE00019F038FD9DF81A0010B1079819F042FF9DF8200010B1099819F03CFF0EB0BDE830
:207C0000F081C046E40601202DE9F04F0E46074630687C68BD68ADF1140D00283AD01EF04C
:207C200089FED4F8E81081460120019008294FF0000088BF0198B168084202D171680842D7
:207C400005D0019880F00100C0B201281DD1D4F8C000B8B9C4F8C060C4F8C4600020C4F827
:207C6000D0000146C4F8D41094F8FC30C4F8D810002BC4F8DC100CBF01980520D4F8C410F5
:207C8000087410E094F8F80030B90320307448461EF0D0FF002050E1D4F8C4004661C4F895
:207CA000C46006233374D4F8C4000021416194F8FC00012808D1022194F8FB0084F8FC10C1
:207CC0004FF4E0211CF0CAF8706810F0704F06D128B104201BF0E2FD06201BF0DFFD02200E
:207CE0001BF0DCFD94F8F800DFF85482002840F0B480E86B3168884240F2AF8094F8FC0044
:207D0000002840F0AA8094F8F90028B1D4F8EC00B0F1FF3F40F0A18048461EF08BFFB76856
:207D2000AA463FB1D4F8E800B94609282CBF0220019802E004F1F40900207768039037B18B
:207D4000D4F8E80009282CBF0220019802E004F1F60700200290DAF80010D6F800B0486802
:207D60005FEA0B0540F0020048604ED04046A0F11008D4F8E800ABF1010B092820D301986A
:207D800003460DE0D8F800108A68398890470346002003B10198031C02D002986D1E3F1820
:207DA000DAF800000DB1012BECD0D8F80010C9680A4669469047BDF80000A9F800001FE00F
:207DC000019803460DE0D8F800108A68397890470346002003B10198031C02D002986D1EAE
:207DE0003F18DAF800000DB1012BECD0D8F80010C9680A46694690479DF8000089F80000B7
:207E00000398BBF1000F8144B3D17768DAF80010D4F8F030CA680020134218BF0198102BC4
:207E200018BF80F001000028F4D117F0704F06D12FB106201BF01AFD04201BF017FD0220E3
:207E40001BF014FDD4F8C010002008740746C4F8C4703E46C4F8C0606EE0D4F8D800002817
:207E600043D1D4F8DC00002842D128791EF064FD4646D4F8CC0032682969406852680068E1
:207E800091FAA1F1B1FA81F1134602229847D4F8CC003268696940685268006891FAA1F161
:207EA000B1FA81F113460222984728791EF03EFD28791EF043FD2046294609F091FE0021F2
:207EC000D4F8C000C4F8E0100068B0F5806F03D92046294609F084FE94F8FE0060B929680E
:207EE000486840F00200486006E0D4F8DC0018B92046294609F074FE2968486940F00100E6
:207F0000486148461EF096FE94F8F800A0B9D4F8EC1004F16C0528461EF0BCF960B1D4F86F
:207F2000C00003210174384606F02AFC284600211EF0B0F900200190019805B0BDE8F08FE5
:207F4000D40100102DE9F04FBF4CDFF80083207889465FEA1941ADF11C0D3FD25FEA5901FD
:207F600011D32079211D88F83C00E12019F022FF1DF032FC0020A8F89400012016F05CF954
:207F800089F001005CE1E7885FEA990116D25FEA191038BF0020C0F0538194F8310050B125
:207FA000E06A94F830101DF02DFD20B994F83100401E84F8310089F0080041E1002F04BF3E
:207FC0000020A07007D07F1EB9B24EF66022E18002211EF071FC89F0020031E117F00AF837
:207FE000071C00F02B81C346387894F83120A178313800F00B81401E00F0BC80A13840F09B
:208000001481FE89383E0FD047F6DD70361A40F00C81B8690678002E40F007814078C00952
:20802000C0F0038178885CE089490EC904A880E80E00D7F818A0042150461DF04BFA3D46EE
:2080400006460AF1040010F8011B049606298DF8141010DBFE2918BFFF290FD10278FF29AC
:208060008DF816200AD1401C4278007800EB0220ADF8180002E000788DF8150006295ADBBA
:20808000FE2931D0FF2912D0287B002840F0CD8068882084002600963346019332460292FD
:2080A00031460391687C802111F054FBBDE09DF816509BF89600A84205DB002D40F0B580C3
:2080C000FF2840F0B28028461AF072FF3EB1DBF84C00864203D0CBF84C601DF07DFBBDF8DC
:2080E00018001DF0EBFDA0E09DF8165098F89600A84205DB002D40F09880FF2840F0958027
:2081000028461AF055FF002001218140314202D1401C1B28F8DB98F83C10884200F085803D
:20812000207198F82B00642110FB01F2012120781EF0C2FB79E02B7B002B76D19DF815A030
:20814000BAF1000F71D0BAF1060F6EDA30461DF059FC002869D1AAF10106687C8DF8156062
:208160006B88607004A923840EC904F12C0585E80E005AE0FF2A12D0002016F05DF8024668
:20818000002000906078B8F894103B4613F071FA94F83100002848D008213222C7E798F85C
:2081A0003C007A6801213B46814011420EBF00213844017A5D68002001228240154203D011
:2081C000C218127A8A4204DB401C1B28F4DB002018D0B8F8920020841026009621896289D1
:2081E000002013F046FA0120E070A07840B93C20E080207802214EF660221EF05DFBA078DF
:20820000401CA070002084F831000EE004290CDA1048017810481DF0F5FB30B97888208174
:20822000FF2684F83160B888608138461CF094FF207816F0DFFE071C7FF4D6AE89F400407C
:2082400007B0BDE8F08FC0461C07012050010120BC860200A201012000F8FF072DE9F04F2C
:20826000ADF1440D0B908069007800210DF12A020F909C200EF01CF8B54D681C007830F03D
:20828000010009D1002004211CF00AFA5FFA80FA9DF82A00504402E001204FF0000A8DF8B7
:2082A0002A000F989DF82A10884280F2DE809DF82A000F99401AC0B20D900228C4BF0220E5
:2082C0000D901A2110FB01F000B211F079FE0E90002800F0CD800F980D9F0E9C0C90002FD5
:2082E00008BF002074D04FF00008B946012645460C9882450ADC0F9940468A4504DAA1EBA3
:208300000A01C9B20C9163E00C9561E0411CC9B20C911CF0D9F9071C54D08E480146B0F8B6
:2083200048005D312080A01C1EF0EAFA388860820223E375FF222276B87A60768DF81C5048
:208340003888ADF81E0007A813F082FDAB46012808BFB34604F10A00BBF1000F06D104F109
:208360000A00FF21082213F039FD02E008A91EF0C7FA3B797BB93F88002F04BF2575281C8F
:2083800004D07448267590F85C00401E207602206075A57515E06F4890F85C00401C207647
:2083A0003879032804DB26753879032805D106E0022020753879012801D0667500E06575D8
:2083C000A6751A34B9F1010908F1010890D140460D9981424CDD0D9DDFF878B104F102085C
:2083E00004F10A0702264FF0000A4FF001091A3C2D1A0C9987206A460DF05AFF5749BDF879
:208400000A0024F81A0F40461EF07AFA0DF1020138461EF075FABDF800004D4B608258780A
:2084200030F0010003D16675A675FF2006E084F8159084F816A09BF85C00401E2076E675BB
:20844000638A9DF81200002B60760CBF84F814A084F814900C9808F11A081A376D1E00F1E0
:208460000100C0B20C90C4D102E000200E900D900B98417C0D9F0E9D8DF82B10801C1621D1
:208480000B9017FB01F0001DC0B28346401C11F097FD5FEA000854D008F101040020A2467A
:2084A0008AF800009DF82A000F9F88F802000D9E88F8037088F8046096B30D9F2E46241D1F
:2084C00006F102090A36204649461EF019FA0834314620461EF014FA0446A87C04F8010B99
:2084E000688A001204F8010B287D2070697D40EA8100C0B22070A97D40EA011004F8010B3F
:20850000E87D04F8010B287E04F8010B687E09F11A091A367F1E05F11A0504F8010BD2D190
:208520000D4D0B990DF12B0048F231025B462C1DC4F800A015F0B0FD404619F09BFA09344E
:208540006C600E9808B119F095FA11B0BDE8F08FE40401205001012028040120AD010120DC
:20856000B8492DE9F04F0A68B449ADF11C0D002A06BF8B1C1D780225AB4BDF689E686D1F4E
:2085800000F04B816D1E00F04581DFF8A482002A65D09279012A62D0A44C276B022A04D098
:2085A000E169002900F03C8139E138460027002851D1780011F004FD5FEA000900F0238132
:2085C000206B40B10021028829F8112040684E1CF1B20028F7D14446B4F89200618F814202
:2085E00033D080460A2000EB47008DF80D0003A81CF032FD061C2CD035690920287004F16C
:208600005D016F70A81C1EF07BF95FB108354846017805F8021F30F8021B7F1E4FEA212108
:208620006970F5D10124B4771DF088FA706201A940461CF0ECF910B1747701A83062A6F844
:208640000280304601F004FE03E0CDF8009008F0F0FD4E46D4E040687F1CFFB2A7E7407890
:20866000DFF8D0B18DF810009BF8030070B90BF14801086838B900208DF8050001A9012033
:208680001BF09CF9CCE0096804A8C8E000208BF803001EF03DF805461EF03AF80027002806
:2086A00040F0B48064484078002630F0010037D11EF02EF858B10A8801888A4204D08469BE
:2086C00014B1201CF8D102E008B18A4228D01C2011F076FC061C23D04146B1F84800308085
:2086E00091F83C40B4701DF065FF7071524880795D31B07106F10C001EF002F941200DF152
:2087000011011CF0BDF89DF8110000280CBF4FF6FE70BBF81C007F1CB5613546FFB23081DD
:208720009BF804A0574510DBA7EB0A005FFA80F8B8F1060FA8BF4FF00508BAF1000F06D00D
:208740005046AD69401EFCD101E04FF000089BF802000C248DF8120018FB04F0001DC0B228
:208760000690401C11F02CFC5FEA000942D009F10104002120460170059089F8027089F87A
:2087800003A0B8F1000F89F8048021D04746241D4FF0FF0A4FF6FE7805F10C0120461EF040
:2087A000AFF8A878083404F8010BA8792070697940EA011004F8010B04F801AB28898045BA
:2087C0000CBF0020012004F8010BAD697F1EE3D11B4D05982C1D0BF1260148F23002069BA0
:2087E00020600DF1120015F057FC484619F042F909346C601048407830F0010003D116B1EA
:20880000304619F037F91AF0B9FB09E080697F1CFFB244E727B1394601E00EB13146884765
:2088200007B0BDE8F08FC046FC090120E402012050010120C4030120E4040120980101200D
:2088400028040120000A01202DE9F04FB04E4FF0000A8146ADF1140D57467069CDF808A09B
:20886000CDF80CA010B1804700B90B27F078002F40F09B8096F8314096F832700146B9F112
:20888000000FA1F101011FFA81F818BF012155464FF0F80B86F83F1022E0AF421ED0F068C7
:2088A00069036A4604231DF071FF009911F4403F1CBF0AF101005FFA80FA01F0FF017C299B
:2088C00018BF782909D1284606215A461CF0C0FE0C2015FB006080F848B0F0786D1CEDB2AB
:2088E000A842DADC401E504503D196F8350000285BD0B8F1000F06F1300500F0CF8003983D
:208900004FF4005B019096F83F30F06813B9012186F83F106A46610304231DF037FFB9F1F0
:20892000000F05D00099F07811F4403F40F09B80009800F0FF00702803D0204670211AF090
:2089400035FFF06879036A4604231DF01FFF009800F0FF00FE2803D03846FE211AF026FFC1
:2089600038460621FE221CF073FEB800FE2300EBC700FF2186F83C70A200A6F840B0401957
:2089800086F83D4000F1180A8AF80030019B86F83E1002EBC4004019A6F84430808BA6F8EA
:2089A000420001F0C5F8102801D10020ADE0B9F1000F0CBF10214946B9F1000F07D0B6F88E
:2089C0004000C0F50050814207DC01200390B6F84000C0F50050814201DD782100E07C214E
:2089E00038461AF0E3FE0CF031F996F83F300446A8EB04000621FC221FFA80F8181B86F883
:208A00003F0038461CF024FEFC208AF80000029A96F83210F078091996F83E400C278918F7
:208A200091FBF0F24243891AC9B286F83210491C91FBF0F24243891A86F8311014FB075144
:208A4000898B102905D1611C91FBF0F24243891ACCB20198B9F1000F96F83270029019D065
:208A60000398B8B11AE096F83F30641C94FBF0F1A8F101024143A6F840B01FFA82F8581E54
:208A8000641A029986F83F00E4B286F83D40481C80B20290B8F1000F7FF435AF7C2019F093
:208AA00081FF00240746FF2F1CD17E2019F07AFF0746FF2F16D196F831700C2017FB00506B
:208AC000807DFF280AD0F27896F832008018401E90FBF2F15143401AC7B203E038467E21A3
:208AE0001AF064FE0C2086F8337017FB0050808BF08696F83200FE211AF058FEB6F84000AD
:208B000086F83540C0F5005000B205B0BDE8F08FC01900202DE9F04F81460D462C20ADF180
:208B2000240D11F04DFA071C00F049811DF048FD698B884214BF012002203870697B28699C
:208B40000026401A7860687B87F82660B8707C68B87887F827602418207800F007007870E0
:208B60002078C0F3C100387420780421C0F3401A601C1CF0AFFC4FF00508B861BAF1010F20
:208B800087F81C8006D007F108003146082213F025F908E0397F07F1080009191DF0B0FEA5
:208BA000387F08303877387C012805D1387F205CB875387F401C38772878DFF80CA200F02D
:208BC0000300012803D0504630300078804687F8018078781DF02AF87877397F28692C7D62
:208BE00040182861397F7B7F601AC01AC0B22875F8704FF6FF74BC82B869B0F1FF3F32D01F
:208C0000387C01281CD038B9062078823946484614F012FD40B30CE0387C022802D00328A0
:208C200007D01EE0062078823946484614F004FDD0B1042078823946484608F0BFF913E0DE
:208C40009AF82F507E82B32075B99AF8651001290AD1B87D17F0B2FAB882844218BF301CEB
:208C600002D1A12000E0A32004463878022806D11CF064FF014607F108001DF041FE002C94
:208C800040F09980514D6878B046012818BF02281CD197F82600012803D097F82700012870
:208CA00014D1B978F8784018397F4018001D11F087F95FEA000809D0B878FA783C7F7968C0
:208CC000121840461219121D1CF068FF38460AF081F804466878012818BF022865D1002C70
:208CE00063D0B8F1000F66D040F203154FF0680A4FF0010900E05C4697F82600012803D0DC
:208D000097F82700012850D1B978FA783B7F786852184146D218121D1CF040FF97F826000C
:208D2000A34630B997F8270040B1BD8287F8276003E0A7F814A087F826607E8238460AF0C2
:208D400049F8041CD8D168463146142213F046F87B8A8DF81190D3B9B88A682803D085424A
:208D600015D1FF2011E07868C17B0529C3D12A30FF211CF054FE0028BDD005A8082213F0B8
:208D80002DF805A81DF0C8FAFC208DF8100002A807A9324612F0A4FF01469DF81C0020B141
:208DA000042014226B461AF073FBB8F1000F02D0404618F05FFE384618F05CFE00E01024C7
:208DC000204609B0BDE8F08F50010120E40401202DE9F84F1DF0DCFBA94CE06011F0AAF8BC
:208DE000A94800681DF01EFFA64D4FF000084FF0010A4FF0020B38E085F80080A3691CF0F3
:208E00003BF920B9E06920F00200E06103E018461DF008FFE069010917D360691DF0FEFE45
:208E2000071C05D0B86817F0D1FF384618F022FE60691DF0EFFE20B9A0691DF0F3FEE069B1
:208E400003E0E06920F00800E061C1080DD320F00400E06120691DF0DDFE30B9E06940F0BC
:208E60001000E061A0691DF0DDFEA0694FF0FF311DF0CCFE1BF0CEFEE7882689A4F806804A
:208E8000A288A4F80880E169A4F80480114347EA010246EA0201E1611DF047F8E069010A7D
:208EA00024BF20F08000E061207816F0A3F868B316F044F8071C29D00C2011F081F8061C84
:208EC0001ED01BF0A7FEB7603B7881465BB9206931461DF097FEE06940F01000E061A069DA
:208EE0001DF0A0FE08E0304618F0C4FD78681CF033F9384618F0BEFD48461DF016F805E0B9
:208F000078681CF029F9384618F0B4FDE06941092DD320691DF07EFEE0B91DF069FBC8B9DC
:208F20001BF078FE064620691DF078FE071C0ED0B9684868498811F07DFFB86840681CF064
:208F40000BF9B86818F096FD384618F093FD30461CF0EBFF20691DF05DFE20B9A0691DF0F0
:208F600061FEE06903E0E06920F01000E0618108FFF451AF66E09DF800006B78AE686F6895
:208F8000A870D81C5FFA80F9494630461CF04AFF9DF80010814205D13FB1484631464246DE
:208FA000B84702E030461CF0D7F885F8008049E0AF68E8789DF80010C019C170E878401C77
:208FC000C3B2EB701CF058F86978C6B2C91AB1420CDBD8193146C01C1AF038F8E878697890
:208FE0008019C0B2E870814222D02BE0DB1989B2DB1C18461AF02AF86878E87018E09DF8D9
:20900000000085F803809DF800706870F81C1BF09DFF0028A8603FF4EFAE6978017085F8E9
:2090200000A00FE09DF80000A9688870687808B9052006E0042004E09DF80000FE2801D1C2
:20904000032028701CF018F800283FF4D7AE6846514619F0FBFF28780028EDD0401E08D056
:20906000401EDFD0401ECAD0401EA1D0401E82D0E8E79DF80000A968487085F800B0E1E74A
:2090800070F70020680A0120EC0101202DE9F04F064606F1060BBBF80000ADF1440DADF8B8
:2090A0000A00707D8DF81400B088ADF81600707E8DF81800B08C4FF00208401E8DF81A0020
:2090C000B06A8DF81280411C089100788DF81900708AADF81C00B08DADF824009648076845
:2090E0000024002F30D04FF0D30A4FF6FF79BDF81600F988884206D0894522D1C10BCD03FB
:2091000001D113281DD19DF81A00203080B21BF01DFF051C15D002A920221CF03FFD9DF82C
:209120001A203AB105F12000A861089905F120001CF034FD85F800A03879294617F052FB66
:2091400001243F68002FD2D17C4800780D940024002800F0BB80BDF81600B6F804901338C5
:209160005ED047F6ED71401A01280BD9001F40F08580B08C062880F28180A6F824804020EC
:20918000B0807BE002A814F065FB071C74D0387800286ED1397BBDF816A00D20884600EBB3
:2091A000480200EB4105D2B20E92E8B210F008FF00280F905DD005463878391D05F8010B21
:2091C00028461DF09DFBB878083505F8010B7888001205F8010B787B4AF0800A5FFA8AFA57
:2091E00005F8010B07F10E0005F8018B06E00178297030F8021B09126970AD1C41464A1EEE
:2092000000295FFA82F8F2D1DDF83C800E9A45205146434619F0FCF8404618F02BFC28E017
:2092200002A80AA91BF0A3FEBDF80A500D2010F0C7FE071C20D0804608F8015B281208F8B5
:20924000010B9DF8280008F8010BBDF828000DF12A01001208F8010B40461DF051FB9DF8A1
:209260003200C1210D223B4608F8080F452019F0CFF8384618F0FEFB012027D14FEAD93004
:20928000C00323D0B08C401CC0B2814610F098FE071C1BD0B0889BF8005040F080003D702B
:2092A0005FFA80F8BBF8000000127870B16AB28CB81C491C521E1CF071FC45204A463B463F
:2092C000414619F0A5F8384618F0D4FB1C48083002884FF6FF7191420DD0BDF81630E500A1
:2092E0002A18455BAB4221D0641CE4B2E5002A18455BA942F6D10D98D8B9BDF81610C80B3B
:20930000C00316D19DF8140098B9132911D041F4004100919DF8180001909DF819008422F3
:2093200000230DF10A011AF08BFE02E0516802A8884711B0BDE8F08F3004012011050120E9
:20934000E07B02002DE9F04305468078ADF14C0D1CF0DCFAA14C071C00F02B816878F87354
:20936000DFF88092DFF880826878F12809D0CD2807D01A2805D0E92803D0E12818BF1D286D
:2093800011D1607830F0010006D17889000B24BF0520787380F0EA803846002103F0EAFCCA
:2093A000002840F0A38010976B788DF84430A87B8DF84500387C002866D1894802685AB169
:2093C000384619469047012804D179894FF6FE70084078819DF84430787B02282AD17989C2
:2093E000890825D3CD2B23D0F02B21D0788A000A07D3B87E28B1B8733868008818F0DAFAC9
:2094000003E094F82100401CB873B87B401EC0B2B876B87304267E73608E43463881A3F1FA
:2094200032000078202115F013FE9DF84430787B022801D0062818D17889400815D37E6905
:2094400046B1707810F0030F04D1B078317BB28819F018FB79894FF6FE7008407881386886
:20946000008818F0A7FA9DF84430607830F001000FD173B948463E680368308818F09AFABA
:2094800028B923B1984702E010A807F0B9FB9DF84430E92B18BF002B07D1396801200090AA
:2094A000EA7B0888498902F0ADFC607830F0010077D140460078800873D3787B022802D14D
:2094C0007889C00806D26878E9286AD1384618F049F966E03B68188818F06CFA20B94FF6E2
:2094E000FF701880052060E003205EE0607830F001002AD140460078800826D33968086A19
:2095000018B3C97F02AA09F075FD6B78E92B07D1396801200090EA7B0888498902F072FCD9
:20952000BDF81200396808809DF80D0000280CBF00224022BDF81200BDF814100CF020FF67
:2095400018B1788940F0200078816E783889E13E18BFB6F1100608D1798911F0300F04D0AF
:209560001DF019F900F00700801C3881607830F0010016D16878E92813D04846006800B125
:2095800080471A4E706A60B140460078800808D339680888498918F007F910B1726A6978C7
:2095A0009047787B022801D106207873A87812F0E1F904F04DFC607802280CD1207850B91B
:2095C00000208DF8480012A9522018F0F3FB2020012106F0E3F913B0BDE8F083E404012063
:2095E000F80601200403012082010120E40201202DE9FC47A24D009004782F5D002FADF8C5
:20960000047000F03B81DFF87C820D2C4FF000094ED0052C15D0072C08D00C2C1AD14068CA
:20962000C08A400A28BF4FF0010913E08678002E08BF07F11B000BD0807D242110FB0170D4
:2096400006E08178012900F01981007CC0192430ADF80400BDF804001BF078FC071C1FD1DA
:209660000C2C40F00B8100984068002800F006811DF060F9064640460068009FD0F85413A9
:20968000381D8847BDF804001BF060FC071C04D130461DF0CFFABDE8FC8730461DF0CAFAD3
:2096A000072C20D02A5D009938461CF077FA18E045462868D0F8282401A953209047BDF89C
:2096C00004104FF6FE70884200F0D380BDF80410401C884200F0CD80009F3889002800F012
:2096E000C880052C46D0072C55D1009908783870487878708878B870C878F8700A7ACE797E
:209700008D79487900EB026000EB064000EB05207860BE78E6B18E7D3E7266B1896951B189
:20972000B20007F1100002EB46121CF037FA07F11000F86002E00020F86038720098806908
:2097400048B318F097F9009800218161817522E01B223A72896907F110001CF01FFA07F1E3
:209760001000009EF860B06918F084F900980021816110E0796807F11805242228461CF004
:209780000DFA7D6079693A7C05F124001CF006FA7868243078613C48016819B13846884716
:2097A00000285BD1DFF8E8A00D2C0DD00C2C2CD1009840781A2828D07E6836B3F08A400890
:2097C00023D30EF000FF20E000984268117801F00203022B3FDA2D4B1B78C1F383018B427F
:2097E00039D1567836F03F0635D190F83000022831D10EF0E8FE0098418E4FF6FF728A426F
:2098000003D140688079022808DAB9F1010F25D050460078394616F0E5FF1FE0381C1AD064
:2098200057F80C6CAEB910F8021CFF2911D15446217800F8021C17480A22394618F0F4FC7F
:20984000012808D120784FF4005115F001FCBDE8FC871BF081FC454628680BE00C2C0DD10C
:209860000098416851B145462968D1F85413001D03E02868D0F8541368468847BDE8FC87F5
:209880008086020014010020D00A01208601012050010120E80A01202DE9F04FDFF84C9259
:2098A00004460D460020ADF1440D01461F460D9016460E9183460F91D9F808A0CDF840B021
:2098C00011F018FF262803D011F014FF252825D1308843F6070181420ED040F60201814262
:2098E00006D0B0F5C15F19D1F07B022816DD43E0F07B022812DD3FE096F8240002280DDDCF
:20990000307C0F2838D13169C1F31421B1F5803F04D00F2830D1B1F5A02F2DD1002D2BD0CC
:2099200056B328784FF0010808FA00F01AEA000F22D0304659461DF00BF865606C4DA66096
:20994000A86980B110A800900DA90EAA0FAB30460AF066FA0E980B214FF6FF7250231AF080
:2099600003FFFF2808D01CF0E5FF82462878022804DB50461DF05EF95C46B3E000286DD1F0
:2099800005F06CF85B495C4E086840F00200086009A8C9F800601CF02FFD584E58497078DD
:2099A00009AA0B9005F1E00016F0C2FA554905F58E7009AA16F0BCFA09A81CF0DDFC1921EC
:2099C00009AB3078504A0A9005F1600018F0B0FB4E4A05F17C001A2109AB18F0A9FB4C49B4
:2099E0005A4605F5AC70134617F064FF49495A4605F5CE70134617F05DFF47480068C0F31E
:209A0000814030B1454A05F1340004215B461AF0E7FEB078012802D10E200DF0BBFC05F13A
:209A2000A0001CF0E1FA05F198001CF0DDFA594685F8241085F83010072085F84002A96032
:209A4000E962374B1970E960052685F83110354A2E610420AA621BF001F9287805EB80012A
:209A6000401CC1F8B840C0B2287050461DF0E2F81FB901A81CF0FEFA01AF38684FF4FA76CA
:209A8000E6602060B8694146A062388A61766083F8692063786800280CBF40F6C41059467A
:209AA00020616061204E266266622176E661F86800B12062786900B16062B86800B1E061CF
:209AC000C82204F13800594612F088F904F1500059461AF05DFA15495A4604F1B800134604
:209AE00017F0E8FE204611B0BDE8F08FCC21084068F2002000200940110000E08487020018
:209B0000155C0200E9650100ADF00100F9DE01009951020031570200B44F00503108020009
:209B2000661B0120B5460100734A0100BF6802002DE9F04F994E96F83D0096F83F10F37851
:209B400096F83C800027ADF12C0D0918491E91FBF3F296F83D4077705A43891AC9B208917E
:209B6000810001EBC0018919B1F84C0096F83C10ADF81C00880000EBC1008019B0F84C5074
:209B8000CDF8248006A818F09DFC70780A97A04500F0A180B946CB46BBF1010F00F09080C2
:209BA000BDF81C10162966DD002840F09580BDF81C0001AAC01F81B2ADF81C1020460EF012
:209BC000D1FFBDF81210BDF81C30884608F1070008F1100287B29A4246D89DF80E00962870
:209BE00042D19DF80F00420839D2800837D3BDF81C0000230093A0EB08001FFA80FA9DF885
:209C00000D20BDF81C002346401A80B219F038FAF8B9E819B0F5005F15DCF068C5F1885287
:209C20000AEB443A3B46D21B514602F500521CF0ADFDED1909F10109ADB2B5F5005F08BF74
:209C40004FF0010B0BE0BDF81C004FF0010BC01D2EE0BDF81C00401EADF81C0004E0BDF83E
:209C60001C00A0EB080023E0204607A914F014FC01281FD030E0F278B9F1000F07D0484B53
:209C8000BDF81C70A10001EBC401C9188F830899A14220D04249641C94FBF2F05043241A7D
:209CA000E4B2A00000EBC4004018808B4FF00009ADF81C0009997078A1427FF46DAF0AE06D
:209CC000B9F1000F07D0364ABDF81C70A10001EBC40189188F8320B106981BF047FF10203E
:209CE00059E0DDF824804FF6F0704FF40051C5EA0040C5EA0141E1FA40F01FFAA0F283B2AE
:209D0000102102F18852404617F084F871780843707006981BF02AFFA0450FD1F278204FB8
:209D20001019401E90FBF2F15143401AC4B2A00000EBC400C019808BADF81C00184FBDF8BA
:209D40001C00A6F840504FEA8801A6F8440001EBC80186F83E40C9198D83B6F9422096F8D3
:209D60003D10012340461AF027FD96F83E10B6F94420022340461AF01FFDBDF81C001628EF
:209D8000DCBF01200A90B5F5005F03DB0A9840F002000A900A980BB0BDE8F08FC01900209E
:209DA000F01900202DE9F04F0546ADF1140D02911CF0C0FD8A4C012D039000F0D280A346FD
:209DC000DBF80000D0F838038047002800F0C58015F0D6FD002800F0C080DBF80410864CA0
:209DE000896960680F783C30002F40F0B6807D4E0068357880477168F268AB00401AB0FB97
:209E0000F3F7B0684FF00008C2469146534611464F4573EB0A0301DA884206D84146524689
:209E200087428A4143DA024600E041461046EB172A46C01B71EB08011CF000F807466F48B2
:209E400000688846418B00694018643081464FF00001B7EB090778EB0A08784271EB08015E
:209E600025DA1CF089FB024653464146384613F0D1FA884607464FF00001784271EB080125
:209E800015DA1AF0C7FE054630691CF055FA10B130691CF049FD28461CF047F83069394648
:209EA0001CF03EFD30691CF03DFD002000E001204D490870884698F8000000284DD1DBF8D6
:209EC0000000D0F8940000780027394614F048FB00B101274FF0000A381C3CD1DBF8040067
:209EE00080690078002836D16068404D436C286902216A4698479DF8000060B302984FF00A
:209F0000010901281ED03A4F6268286997F9001011F1020F05D0926B97F900109047626876
:209F20002869344E96F9001011F1020F05D0926B96F900109047626828696FF001013170B7
:209F4000397001E062682869DBF80410896981F80090D169884788F800A003981CF06AFE02
:209F60003AE02068D0F894000078012114F0F8FA03981CF05FFE606880690078012811D11B
:209F80001BF0FAF960B1606880690178012909D10021029F0170012F04D01BF007FF01E05B
:209FA0000EF0F2FC1BF0E8F9B0B960680C30C1680978022909D101680F7837B12068D0F885
:209FC0004C058047241D20680C3001680F781FB9C16808780228FCD005B0BDE8F08FC0461E
:209FE00014010020D8000020721B0120A4060120B00A0120B10A0120D4050120B40601202F
:20A00000F0B58E4D05F1320184788E4A0E782746ADF11C0D7F1E0B2F03D9FE3F00F0D680D3
:20A0200008E1DFE817F0C000AC00A0008900F9007B004D003D00300021000C00E100002177
:20A040008DF80A1010F8031F31F0030706D1521C1170512001211CF067FB02E002208DF8BC
:20A060000A000DF10A03E0E03EB100200146F9F709FF002808BF002000D001208DF80B002D
:20A080000DF10B03D1E0002210F8031F8DF80C2000290CBF101C01201CF010FB03ABC4E05C
:20A0A000C01C002110F8017B8DF80D1004211BF011FA002F0CBF6862A8620DF10D03B4E0D2
:20A0C000C01C10F8016B002108220746684611F085FEEFB15A4900204870301C15D0401EBC
:20A0E0000ED0401E0AD0401E03D0401E10D101204870384669460CF073F80AE001204870AA
:20A10000384669460CF002FC03E016F05FFA00E002208DF80E000DF10E0386E0002210F8A2
:20A12000031F8DF80F2000290CBF101C01201BF0A7FB0DF10F0378E0C01C002110F8012BC2
:20A140008DF811100146521E00F1080004D0521E06D10CF045F801E00CF0D8FB8DF811000F
:20A160000DF1110361E0844600201CF8037F8DF8120007B101200DF11203107055E00021B3
:20A180008DF8131010F8031F0E2906DCD21C1170532001211CF0C8FA02E002208DF8130066
:20A1A0000DF1130341E000218DF8141010F8031F0E2906DC921C1170522001211CF0B4FAE0
:20A1C00002E002208DF8140005AB2EE00025C01C04218DF808501BF07DF91B4948604D80C7
:20A1E00010F0B4FF02AB20E00021C51C8DF8091028461CF015FA06460421A81C1BF06AF933
:20A20000014630460DF0FCFD104A352028211CF08BFA0DF1090308E0014600208DF8100014
:20A2200011F8030F03F0A2FF04AB21466F20012218F0EEF807B00020F0BDC04668060120A0
:20A24000CCE80020E6040120100A0120300301202DE9F04F8F4E054696F84A00ADF11C0D74
:20A2600008280CD004280AD0287800F00300012840F0088128690078062840F0038168887C
:20A280004FF6FE74844200F0FD80718F814206D1287F20B9284612F00BFA0446F3E01BF01D
:20A2A00073F9002840F0EC80287FDFF8ECA14FF000082746C34608B30AF12400007804212F
:20A2C00040EAC00010FB01F05FFA80F9698885F81C90FF2019F00CFF48B1E88A49F00103D1
:20A2E0004FF00108671C2B7740F00400E8825046407830F0010008BF4FF0400B688817F09C
:20A3000059FB08B100206876A87E08B90F20A876287830F07F0008D1E87E50B996F82400C5
:20A32000411C86F82410E87603E0287800F003002870287E012806D196F82F0018B92878CE
:20A3400008B9002028769AF8010030F0010020D196F8320080081CD3B8F1000F0AD168881F
:20A3600017F028FBA8B1287820B1286900781BF05BFF70B1E88AC00902D3A87E012804D027
:20A3800028461AF081F820B97AE0E98AE01E0840E8822878012807D128690078022803D1CE
:20A3A000E88A40F04000E882E88AC0093CD2B8F1000F39D19AF8010030F0010034D196F8FF
:20A3C0003200800830D3687E6988AA1D5B4612F03FFB28B10020EB8A687643F02000E8823C
:20A3E000A87978B1698805F1080017F0C3FA07466888B84204BF0021A971E98A41F0400146
:20A40000E98200E068882978012904D0A9885A460EF0CAFD6888A9885A460BF0B1FF18B197
:20A42000E88A40F02000E882284606A904F04CFF8046BC4208BF6F88B8F1000F1DD00595D3
:20A4400028788DF810006C8DADF812406B7D0093E88A019095F82C00029004AA0392728FCA
:20A460009DF81830394640460BF03EFC0446102C04D1404617F0FEFA00E0102420460CE778
:20A48000112400E0C224284617F0F4FA204607B0BDE8F08F50010120E40401202DE9F04F4D
:20A4A00009AF00268B46ADF14C0D099034469BF80380BBF806100B93B8680A92854D0D903B
:20A4C00038790F964FF00E090C900CE014FB09F02A5C904505D140191AF0F6FB08B1761C70
:20A4E000B6B2641CE4B2002CF0D0002E0E9600F0D7809BF81450F1B2182000EBC10084B225
:20A50000281900B20FF05CFD051C06D00F99224611F064FC2E742819E860002D00F0BB8005
:20A520009BF80340DDF83C80BBF806102046424616F090FD06466C71BBF80600E8809BF88D
:20A540001600688185F808809BF81420E868DBF81010CDF820801BF021FB4446109411948E
:20A56000B8896882387CDFF87091287555E008994FEAC80005EB000A4019817570780AF184
:20A580001604012810D0B0788AF81D007088ADF81C0004218DF8101004A815F047FDBDF8A4
:20A5A0001200AAF8180005E00120207001230F9370886080307920719BF80000C00903D32F
:20A5C000A07940F00200A0710F9ED6B9B9F83A006188884215D120798BF80200109E0096FD
:20A5E0000C9B01930D9A0292314603910A9B0999B9F8482058460DF059FCA07940F005003C
:20A60000A07108F101005FFA80F8BBF806109BF80300424616F01EFD064616B10E98404518
:20A62000A5DC2E4C201D06681198314604E00E4620E00968401CC0B20029FAD1052813DBCE
:20A6400096B1334600E01B6813B99E4202D00BE09E42F8D1306801216060304614F0DEF8FB
:20A66000304617F007FA6668607828716078401C6070284616B131680029D8D11199002EA1
:20A6800001600CBF606030600C9B00950B993A78584600F077FB0E98002818BF002D15D1F4
:20A6A0009BF803009BF816708DF81300BBF806608DF814700E9DADF81660002D0CBFB9209A
:20A6C00010208DF8180004A81BF0FDFE13B0BDE8F08FC0462201002050010120EC0A012042
:20A6E0002DE9F04F0746861CADF11C0D30461CF0D7F886490446182268460EF007FC7D7807
:20A700000DF10B0031461CF0FBF84FF6FE794FF0000B02208DF816004FF00108ADF8149066
:20A72000B87A8DF808B0810805D3B87A000934BF0326042603E000092CBF02264646744881
:20A740000378002B08BF002D00F09680714890F84A10082940F093801BF0D6FD10B1012D7D
:20A7600000F08A80002C27D02079864218BF022D74D1042818BF032803D1042E10D0032ECB
:20A780000ED0022818BF012812D1022E08D0012E06D0022818BF01280AD11CF0DDF807E0F4
:20A7A000208882461AF0BCF808B9ADF814A003E0B81C14F085FF5C46BDF81430994514D1B4
:20A7C00019F05AFF70B95448008882462DB11AF0A7F8002808BF504601D01BF0FDFDADF87B
:20A7E000140003464846984235D0BA7A1846B91C2B4611F0F9F907F1020A002841D14648F8
:20A80000801D016811B1BDF814008847BDF814005146324609F078FC04463E4800784FF408
:20A82000803141F288321CF047F83A494046087174B1022D05D0012D07D1607940F0100065
:20A8400002E0607940F0080060718DF816B011E0ADF8149015E04FF0C70812E020888DF88D
:20A8600016B0ADF814002279BDF81400B91C2B4611F0BAF9D84604E04FF0C30801E04FF0CF
:20A88000C208C5B1254803789BB9012D11D144B902208DF816003146012268460FF004FB2C
:20A8A00030E08DF816B00122684631460FF0FCFA04E02A46F8E7684616F0EAF806469CB19E
:20A8C00045B16079022D40F04000607104BF40F020006071B87AC00903D3607940F08000FB
:20A8E0006071A079401CA07156EA08000AD014B1B81C14F0E5FEBDF814104846884201D05D
:20A900001CF02AF807B0BDE8F08FC046A07C0200FC09012050010120EA020120E50401205B
:20A920002DE9FE4F824C00906068C06801910121017080484FF0000A80F800A07E4880F8DA
:20A9400000A02068403001680D681E46174615B9D0F80C0580477949DFF8E481DFF8E49108
:20A96000886E4FF0E2450AEA0702354008BF002A40F089800D46B5F89E10082253463A40F4
:20A9800013EA060708BF002A0BD118B14246508B401C50834A4692F90000401E10701D204F
:20A9A000ABE04A4692F90030DFF89CB142F201468E42A3F10103137002D0321D8A4216D163
:20A9C00018B14246508B401C5083584600680199826C0098904750B1424602F11601008804
:20A9E000B5F89E30098842F60147874233D15748411C0A78B5F86610B1F5105F12D0AF6E49
:20AA000042F60600884206D0002FC8D04246508B401C5083C3E7002F71D04246508B401C26
:20AA200050836CE0A96F5B460C3319604189062A0CD1427A022902F10102427206DB491ED6
:20AA400089B24181062002F0FBFD58E016F068FE0EF00EFA53E0491C361D88B29E42D082E8
:20AA600014BFE1201C200FF0DBFC99F9000020B199F90000002854DC48E02068D0F85824AF
:20AA8000514650464CE04A4692F900102768491E117007F1400118B14346588B401C588316
:20AAA0000868006840680078800925D2284A1078832824D125484378032B1BD1042347795B
:20AAC000D1F8945013707B1CDBB2437195F8241099420DDB817895F831304D1CAB42C4BF2A
:20AAE000491CCBB28370832010701BF0EFF906E0E12002E0852051E7E9200FF091FC99F99E
:20AB0000000040B199F9000000280ADC2068D0F84C05804705E02068D0F8582450460146AE
:20AB200090476068C06880F800A0BDE8FE8FC04614010020B40A0120B30A01205800012093
:20AB4000D8180120B60A0120D805012004180020741B01202DE9F04F7F4E7068416EADF1D2
:20AB6000340D02A88847DFF8F4B19BF9000038B17B4890F90000002818BF002040F0E9801E
:20AB80001BF0D8FEDFF8DC910A9099F80000800806D27D2000210CF09FFB0025079001E014
:20ABA0000025079502958DF80C50059503228DF818206D4CA4F8BE50C4F8C45094F8C80059
:20ABC000012705F00F013B4620F00F00014384F8C810DFF898A10B9394F8C81063F3C711D0
:20ABE00094F8D73084F8C81023F0010007F0010343EA000184F8D71094F8D70067F34100D0
:20AC000084F8D70094F8D70065F3820084F8D70094F8D70065F3C30084F8D70094F8D7001D
:20AC200065F3041084F8D70094F8D70062F3461084F8D700DAF80000D0F8282404F1D80140
:20AC4000F4209047DFF8288198F80030A3B94946706809788446890910D3C06B8047C4F898
:20AC6000C40094F8C81021F00F0141F0020184F8C8108DF80C700290D6F804C03E4A3D48D1
:20AC80004FF080738DE80C00DCF850703B4B006804F1BC01894602AAB8470028708006D560
:20ACA000022041F2883113F0F1FC0B954DE02C49334F91F90000401C087097F90000401C88
:20ACC00038709BF90000C6F808902946401C8BF80000022013F0DAFCDAF8001001F1AC0217
:20ACE0001068077888F8005007B18025308F17684FF67F7303401D432843308794F8D42076
:20AD0000387860F3C71284F8D420D1F8D400C28CA6F84620428D00F14403A6F844201A686D
:20AD200006F13B052A6058686860D1F8D400C18CA4F8EE10418D00F14407A4F8EC10396803
:20AD400004F1E4063160786870600A981BF072FF0B980DB0BDE8F08FD4050120B80A012054
:20AD6000B70A0120701B01205800012014010020B50A0120B4060120200043006D450000C7
:20AD8000B60A01202DE9F04F0646ADF13C0D032700200A91189D0C93297C0B920CE005EBF3
:20ADA000C002127F530805D3D30803D212093CBF7F1EFFB2401CC0B2814201DD002FEED19C
:20ADC000B9460124002010E005EBC002177FFB1109D07A0807D307F0040207F00807174359
:20ADE00004BF641EE4B2401CC0B2814201DD002CEAD1A346B9F1000F08BF002000F0CC805D
:20AE00004FF00008BEE04FEAC8002A184019007F02F11604400880F0B180002760480D97C9
:20AE2000077837F0010714D1277897B9108B1BF00AFD70B10079012818BF032809D1A0792B
:20AE4000BBF1000F40F08000A07100F0968001200D900C98002814BF2027002700210C2256
:20AE6000684610F0BBFF237813BB0A9800280EBF4FF0080A47F040074FF00A0A60884FF61B
:20AE8000FE71814228D104208DF81800E379ADF8243006A815F0CAF84FF6FE7000210346DF
:20AEA000B0800A46ADF8003007A813F0CBFE15E03C480078012808D0608847F00C074FF05F
:20AEC0000C0AB0804FF6FF7006E06088FF2147F00807217141F2080AADF800008DF80270D1
:20AEE000307D8DF8040001238DF80530684607F061FE9DF8141061BB0398417D6171A0F8A2
:20AF000016A00B9F4776277817B126490978017769890185698A4185297D80F82C106979D8
:20AF200080F83A10217980F83B10F188C1873189A0F84010717D80F84910B1888187406CE3
:20AF4000327D31691AF02AFE684616F093FC9DF81410A07940F00100A07151B90D9818B1A7
:20AF6000ABF101075FFA87FBA9F101075FFA87F903E0A07940F00800A071297C08F10100F3
:20AF80005FFA80F8414503DDB9F1000F7FF43BAF2846002113F042FC0FB0BDE8F08FC046AB
:20AFA000E5040120DC0101202DE9F041064606F11600ADF1380D16F0DDFE7A48007806F1F4
:20AFC0001607012818BF02282FD100200DF1320501A905AC8DF8320001220095601A83B25C
:20AFE00001A907A815F084FE98B16F4800680DF1330101AA10F074FEADF81C00BDF81C40E8
:20B00000C82C12DA03A8394608221AF0C7FD214606E003A8394608221AF0C0FDBDF81C10E5
:20B020000420142201AB18F033FA3846FF211AF0F6FC10B15D4901200870002402A83946EE
:20B040008DF804401BF05CFC1BF05EF948B901A812F04EFE012804D02046394608AA19F0CD
:20B0600005F83079534D012861D006285FD0691C0B7804282AD0032840F0918038460DF1BD
:20B080001E0119F055FA58B14FF6FE7039460DF11E0218F0EBFF214638460A4613F0D2FDE7
:20B0A000BDF81E0006A918F0F7FF069838B906A818F0B6F818B9BDF81E0006990880B11D84
:20B0C00038460EF06DFC12F0FFF868E0002B66D038460DA901AA10F003FE01469DF83400F9
:20B0E00000285CD08DF8154020460290019001278DF81640142201AB8DF81470042018F07F
:20B10000C7F9B21D4FF4817010211BF007FB06F1060828B94FF48170102142461BF004FB51
:20B120002D1F384603216C7118F094F837E0721D1021204612F8017F1FB9491E00F10100B8
:20B14000F8D11B4F10280CD07179B01D18F042FE387808B12878D0B170790DF025FB2C707D
:20B1600015E0387898B9204662210DF1220211F01DFD0DF12200214618F02CFE20460DF097
:20B1800013FB0DF122002146102210F027FE0A480178052903D1C079802113F059FF0EB003
:20B1A000BDE8F081E5040120EC060120CFE80020B50101206C060120C40301202DE9FE4FD0
:20B1C0009B461546894682461BF0B4FB7B49019008680CAF504508BF48687B4C6FF0010827
:20B1E00028B1B8301BF0A8F8002840F0D68019F023FD061C00F0DB8004F5CE701BF094FBCE
:20B200000023B4F9B400C6F80C90401C86F832306FF31F30A4F8B400C6F808B0B4F8B4003D
:20B2200030866748C6F810A097E80C0020210027B8461940104006F1180383E80300424699
:20B2400086F8332006F1200383E88001E8683064287C86F8440028687063287986F8380013
:20B26000A868F0636869B064A869F064287F86F85000687F86F851002F7C27B9EF6817B14C
:20B28000012086F844002F795FB999F80C0000F00F00022805D1012086F83800D9F80800BF
:20B2A0007063484608274568002D18BF002F70D100886FF30900B0F5305F18BF022506D1E1
:20B2C00096F83300082540F0100086F8330006F1180090E80C00414606F1180745EA02002E
:20B2E000194387E80300D4F8D800824507D194F8DC00410824BF00F0FE0084F8DC003148EA
:20B300000768002F39D004F1A0000090D4F8A810D4F8AC2004F198052B463046B84710F1CC
:20B32000030F10D0B6F93010B4F9B420914207D0B4F9B41001F6FF716FF31F31A4F8B41017
:20B3400010F1020F1BD010F1030F18D096F83300B6F9308040F0800086F8330000278AF8CB
:20B36000FC702868864205D0F068007B00F00F0002281CD112F002FA19E06FF00200B4F946
:20B38000B410804601F6FF716FF31F31A4F8B41005E07F1E2846FFB285E76FF0020894F8A8
:20B3A000DC0040F0040084F8DC00C4F8D8A001981BF040FC4046BDE8FE8FC04620F3002020
:20B3C000FFEFFF9F040B012068F200202DE9F04F8246DAF8185069782878EA7800EB0120F1
:20B3E000A978ADF1240D034601EB0221069116F0E1FA012800F0D6804FF00008CDF8108082
:20B400001846CDF8148016F0D5FA2D1D48B96F480088984205D06E480078022800F0C280DD
:20B42000D0E015F8014B5CB160000EF0C9FD049030B1049A204629461AF06AF8054600E053
:20B44000444615F8017B5FEA07090AD078000EF0B7FD059028B1059A384629461AF058F828
:20B4600000E0C1465B480568002D76D04646079608966868017800296CD0AA7B520869D332
:20B48000AA68002A04BF8668DDF820B004D0012090474FF0010B0646002E5BD070880699C7
:20B4A000814204D006984FF6FF7181424CD1F279B3680499204618F09EF838B9327B336961
:20B4C0000599484618F097F800283DD009EB0400022110FB01F01430C0B219F037FD071C47
:20B4E0002AD0D2203870BAF80200788087F80C90002C3C7104BF0798B86008D007F11400BA
:20B500000499B860620007F114001AF047FBB9F1000F04BF0898386108D0059907EB44005B
:20B520004FEA4902143038611AF038FB686840680078394615F056F93078274908F1010791
:20B5400001F808005FFA87F8BBF1000F02D0304616F090FA2D68002D8BD1B8F1000F05D1D3
:20B560009AF80C00A8B90023984600E00023174800880090CDF80480174F02979AF8100067
:20B5800003909AF811100AF1020248F2060012F01BFD049808B116F06DFA059890B116F066
:20B5A00069FA0FE000930020019002909AF8100003909AF811100AF10202802348F2060099
:20B5C00012F002FD09B0BDE8F08FC046E0030120E5040120C00A012054050120FEB50E460D
:20B5E0001BF0A8F900257F4A7F4C517855708A080ED2C9081AD31BF01DFBA4F1080000F177
:20B6000008048068D0F858242846014690470FE01BF010FB6068C068007828B92068D0F8C8
:20B6200058242946012090471BF084F91BF002FBB00941D337E02168D1F898205060009861
:20B64000D1F8401388472168D1F89800D1F85413001D884732E01BF06DF92168CA6B117B2C
:20B66000491E11731BF0E6FA216800983C31CB6D0278586000988DF8042047782FB1162ADC
:20B680000AD1D1F81813684601E0D1F80413884721689DF804203C31162A06D0C86DD1F8DA
:20B6A0001813001D884721683C310868001D18F04CFB00280090CED1300C08D32068D0F8E3
:20B6C0009400007813F096FC00280090B3D1700907D327682E20D7F840138DF8040001A809
:20B6E0008847700807D327682520D7F840138DF8040001A88847B00807D327682620D7F8FC
:20B7000040138DF8040001A88847F00807D327682720D7F840138DF8040001A888473009D1
:20B7200007D327682920D7F840138DF8040001A88847F00909D32D2027688DF80400D7F82B
:20B7400040138DF8055001A88847300A09D3302027688DF80400D7F840138DF8055001A821
:20B760008847700A09D3352027688DF80400D7F840138DF8055001A88847300B07D38DF829
:20B78000055037208DF8040001A81BF037FA700B07D38DF8055038208DF8040001A81BF0CB
:20B7A0002DFA2068D0F898000068C8B11BF0C2F82168D1F898100A6800920D601BF03AFA2A
:20B7C00021680098D1F8982050600098D1F8401388472168D1F89800D1F85413001D88478E
:20B7E0002846FEBDD8000020140100207D492DE9F04F0A680646ADF11C0D0DF10E000260E5
:20B8000049684160F08900280CBF08210221B569764A15F80180D0B973490F781046294621
:20B820001AF0ACF880B937F001004FF6FE7434D128461BF035F800282FD00179012918BFF5
:20B8400002292AD1048821E06948048825E069782878674F00EB01243888A0421CD0624973
:20B860000878002530F0010017D120461AF0EBFF98B10179012910D18DF800504088ADF8B0
:20B880000C00684614F0D2FB00B101ADB8F1000F18BF4FF0FF0800E015464FF6FE70A04219
:20B8A00018BF002D03D1377B002F40F0988051494F68A0424FF00B0910D07DB138F00100CA
:20B8C00008D0307B012800F08A804FF0000B4FF0800A0DE04FF0000BDA4609E0F3894FF0B4
:20B8E000000B4FF0810A002B0CBF441C0DF10E0507F801AB002D14BF291C0DF10E01384691
:20B900001AF0FEFF0746384D07F8014B20123870287830F0010053D1B8F1010F50D13448EE
:20B920000088A0424CD1BAF1000F49D18DF816B00DF1160012F01AFD7F1C051C3CD0F489EF
:20B94000002C0CBF08210221B0699DF816404018427805EB4201A242A4BF58468DF81600DB
:20B960000ADA9DF81600801A8DF816009DF8160009EB40095FFA89F99DF8160007F8010B8A
:20B980003A709DF816407CB17F1E087807F8020F9DF8164031F8020B00127870601EC4B2A9
:20B9A000002C8DF81640F0D1284616F063F809F102005FFA80F903E087F800B04FF00C09BC
:20B9C0000C49F28910204B46C87042F4004206F11100B11C12F060FB064880F803B007B0C4
:20B9E000BDE8F08FE07B0200E50401201C030120E0030120280401202DE9F0470646F08919
:20BA000017468946ADF1280DC01D80B205460DF00DFE7A4CFF280BD12846FCF715FF8542C0
:20BA200004DD641C207800B90520E3E0012000E000206178D9B917B1022F18D1B8B1307AEB
:20BA40008DF80C00F788ADF80A70B588ADF8085000230093E18E94F8330001AA032304F0D4
:20BA60004DFA9DF814003074BDF81070B78194F83310E58EE06806AA0423884649031AF040
:20BA800085FE069800F0FF0100F0FF007E2806D140467C2117F08AFE069901F0FF017C2942
:20BAA00040F0A580F08942F20102C11D8FB2E9198A4240F39A80F188327AC1F301238DF8C5
:20BAC0001D10B18843EA82038DF81C308A1006468DF81E200423C0F3851201F0030142EA42
:20BAE00081128DF81F2010FB03F1F21D01F0FC01731990B28DF820101FFA83FA0D282BDB9F
:20BB00004846314600221AF079FD0246052107A81AF074FD9DF82010334600F03F064A46E3
:20BB200041EAA011B0008DF8201040F0020096268DF8210029468DF82260404615F06AF9CC
:20BB40000646514607AA07234046667015F062F9304360704DD135E004F1240049463246D5
:20BB60000DF0D4F907A90A68301900F12409484609790260731D0171002204F1240099B278
:20BB80001AF03CFD9DF82010962300F03F068DF8223041EAA011B0008DF820103B4640F0E6
:20BBA000020007AE49468DF821003268B0790A60B288887140468A8004F12402294615F01A
:20BBC00029F96070E18EED194FEA8806AAB2C919E18606EBC8010919A1F84C2048B1404632
:20BBE000514614F0D9FD607803E0052000E001206070C0B20AB0BDE8F087C046C0190020DC
:20BC00002DE9F04F09AF3D7AD7F804800E1C9A4693460446ADF12C0D26D0207A29098DF8C2
:20BC2000260010D302281FD121881AF0C9FC884209D008460322012111F0F1FF002818BF41
:20BC4000CD2040F0D580237A022B07D00F2B05D0032B0DD0012B0BD033B909E0208815F02E
:20BC6000A9FE18B90F2B03D10220C1E00F2323728DF80830032B1CBF2088ADF8000003D1CD
:20BC8000684621461AF03CFEA8081DD25A484FF000090368ADF8109043B15868864203D0C3
:20BCA0001B68002BF9D101E09A681AB9B3688BB158880DE031780220904758B10188ADF859
:20BCC000101015F0D7FE05E04FF6FF704FF00009ADF810006809ADF818900BD39DF808009B
:20BCE0000F2807D0012805D0BDF8180040F00400ADF8180035F07F0005D0BDF8180040F004
:20BD00001000ADF81800E80938BF484606D3BDF8180040F00100ADF8180001208DF8250081
:20BD2000E80805D3BDF8180040F04000ADF818008DF82490A80934BF012004208DF81B007F
:20BD400039680591ADF80EB0ADF812A03D7B8DF81C50637A8DF80B3098F800008DF81A007D
:20BD60006189ADF80C1030788DF80A0019F05EFD20B1016911B168468847637A19461AF0BD
:20BD80002DFD78B909A815F041F9504506DA1B480168A1B168468847074611E0684600F06C
:20BDA00031F9F9E716480068D0F80001C0892238C0B2504503DB684605F010FCECE70227B7
:20BDC0009DF8080002280CD11AF0FAFBBDF80010884206D1307898F800105A463B4616F0EB
:20BDE00051FE27B998F80000401C88F8000038460BB0BDE8F08FC046C00A0120E80601204B
:20BE0000140100202DE9F84F0AAF97F80090984692460D46044615F0C7FC0746754800266D
:20BE2000B346002F38D1B9F1000F20D117F016FB071C00F0DC8031461C220FF0CFFF3C8062
:20BE4000BAF1000F7D8106BF0120B87487F812A069485E300078012818BF072002D15046A0
:20BE600019F0A7F8787406203874BDE8F88FB9F1010F0FD105466878B8F1000F52D030F071
:20BE800001074FD15C49097889084BD3204617F035FD41E005463FE005466878B9F1000F97
:20BEA00012D1B8F1000F0BD1B97851444910CBB2BB700BB90121B9707B780BB90321797071
:20BEC000B97806292EDD2BE030F0010306D14B4920310B6813B1184680476878B8F1000F18
:20BEE0001CD030F001031DD143490978890819D342482430026812B1414638469047387823
:20BF00000D2809DA401CC0B20C28387004D1204617F0F4FC7E700126687803E03146397035
:20BF20004FF0010B022825D1B9F1010F22D1B8F1000F1BD0B8F1EB0F18D0B8F1E10F19D039
:20BF4000B8F1F10F16D0B8F11A0F13D0B8F1190F10D02A49AB7D0A79521CD2B29342C8BF80
:20BF60000A7107DC002201260A7106E023490022091D0A7056EA0B0739D030F0010714D123
:20BF80001D490978890810D320461AF05CFC58B1BBF1000F03D0417901F0FE01417136B3A2
:20BFA000417941F001014171687806B3144E30F001000DD196F83200800809D3204619F055
:20BFC0008CFD28B12146002017F0F6F8BDE8F88FF08FA0420BD12146012017F0EDF86878C6
:20BFE000022804D14FF40050012103F0D7FCBDE8F88FC046E404012082010120E4020120E1
:20C00000500101202DE9F04705467B4895F80B900078ADF1180D002808BFBA2000F0E980CE
:20C02000684600210C220FF0D9FE01264FF0000A298B8DF80560C8080AD39DF80220C810E3
:20C040000B0942F040028DF8022038BF032602E09DF80220C8104B0928BF46F04006400821
:20C060000FD342F0C00288098DF8022039BF9DF8030040F002009DF8030040F001008DF8A2
:20C08000030001EA6100000A28BF46F00806287A5A4F002830D00F2828D0022822D0032833
:20C0A00018D0012832D1387848B94FF6FD70ADF80000288842F00C0246F0040608E028889C
:20C0C00042F0080246F480564FF0FF09ADF80000824619E02846694617F0F0FA9DF80220A2
:20C0E000298B13E02888ADF800000FE0288842F0080246F0040605E01AF062FA9DF8022027
:20C1000042F00402ADF800008DF8022048081AD312F00C0F0DD1288813F08FFD002808BF35
:20C12000BB2066D09DF80220298B42F020028DF80220480807D302F00C00042804BF42F03F
:20C1400020028DF80220A87C8DF80400684606F031FD9DF8140000284BD1039CE682E87E3D
:20C160006076287FA076287A012804BF38782077A87E2085288B6085E87F84F82C00288B32
:20C1800000EA6000000A15D395F82000667D804617F0B2F9071C0DD03A7C002008E007EBAB
:20C1A000C001CB7E984504BFCE763A7C401CC0B28242F4DCA87A84F83A0084F83B90A4F8BE
:20C1C0003CA0E889E087288AA4F84000A87E84F84A00A87F84F84B00687F84F84900606CCB
:20C1E00069696A8A19F0DAFC684615F043FB9DF8140006B0BDE8F087E3060120DC01012026
:20C200002DE9FE4F07462C200DF0DAFE0028386100F0E48000212C220FF0E0FD38694FF607
:20C22000FF7585823C6938880DF1020111F03AFADFF8B4B158B30DF10200694619F0C8FB26
:20C24000BDF80000854222D000200626BDF800102074BDF80020634B66828E00A28206EBBD
:20C26000C100C2181168A1611168491C11601E584FF47A74B6FBF4F06043361A07D1012031
:20C280005E46107230784FF4006112F0E1FE39693888083111F006FA5448846880461AF057
:20C2A00033F868B138690021418238696826868238690223037438698461621CC8F8082055
:20C2C0004B48D0F800903869DFF828A10446A18A2E468E4254D104F10800494619F04EFB76
:20C2E00048B919F02BFC0146484619F047FB10B91AF00AF860B13888396902F065FC00242E
:20C3000000B1012400200CB139698D823969087438690446A18A8E4232D15146303991F829
:20C320002F303BBB91F86510012923D101200DF10A013A221AF0E3F8C8B901209DF80A5090
:20C34000207400233A22A5755D466382D8F80410A2822878A161D8F80410491C0129C8F84B
:20C36000041005D14FF4007112F072FE00E0A5823C692046828A3146914204BFA121397512
:20C38000818A8E4224D0017C01290ED0BE6856B919F0BAFF20B9B878400838BF052100D311
:20C3A0000D21204602E00D2100E00E210177B87800F0030001281ABF51460878052039694F
:20C3C00048703C69607819F031FC6077BDE8FE8F15F050FB00203861BDE8FE8F10203875D1
:20C3E000BDE8FE8FE0E80020CB030120100A0120EC060120800101202DE9F04785682A6878
:20C40000D16944681162490832D3D4F8C01049BB2968486820F0020048602968486A20F07F
:20C4200003004862D4F8CC002A6941686F69096847EA0200C862D4F8CC006E6941682A692A
:20C44000096846EA0200C1F804052968486920F001004861286801210162284618F038FABE
:20C46000BDE8F08703220A7402F08AF9BDE8F087D4F8CC0041682A696F6909684FF0000907
:20C480000226CA4647EA0200C1F80405D4F8C070002F00F0A880D4F8CC00D5F814E040682B
:20C4A000D4F8E0C0D0F80080BCF1000F04D1EA69A86904F1D80103E004F1DC016A6A286AEA
:20C4C000D8F8043513EA0E0F11D0806810F0070F0DD13868D4F8D030984208D17F6937B985
:20C4E0002B68586A20F002005862C8F804E5906810F0070F74D10F68002F71D0D4F8D40098
:20C50000BCF1000F3844C4F8D40014BF48462020C4F8E000C1F80090D4F8C010D4F8D02075
:20C52000086890424BD8D4F8D420904247D881F81090D4F8C80004F1300730B9D4F8C01087
:20C54000C4F8C810D4F8C80008E04369002B34D1D4F8C0104161D4F8C01040694969C4F8FE
:20C56000C010C0F814A0D4F8E00000280CBFD4F8D800D4F8DC00C4F8D000D4F8C000C4F8C0
:20C58000D49088B12046294605F02AFB94F8FE0078B1D4F8CC00406801686869D1F80425F0
:20C5A000024218BF886204E02968486A20F00300486238461AF0DEF912E01846C5E72046D1
:20C5C000294605F00DFB94F8FE0048B1D4F8CC00406801686869D1F80425024218BF8862FB
:20C5E000761E7FF453AFBDE8F08770472DE9F84F0746714D714C28684030D0F89410267830
:20C6000091F883B026B1D0F80C0580472868403001680E6816B9D0F80C058047A046694901
:20C62000674C0120012F88F80000D1F8009067702AD9DFF894A1654EBF1E59D07F1E52D0BF
:20C640007F1E3DD07F1E73D07F1E34D12968096C096891F86D20628191F86E70002F06BFE3
:20C66000E070071CE770686840683178007811FB00F0784381005046C16690F8701021F049
:20C680000F0141F0030151E000202E686071306C0068D6F8D410C08AC00934BF91F8250033
:20C6A00091F84E00A070B7B9CF78A7B10228C4BF0220A0700FE02868D0F84C05804737E02F
:20C6C0002868006C006890F86910617190F86A00A0700027A77109F0C7F92868006C0068C5
:20C6E00030BBBDE8F88F0020607116F053F81FE030788700D9F83C00804771683C22401A4E
:20C70000B0FBF7F0B0FBF2F15143401AC0F1780086B2D9F83C00804707FB06015046C16610
:20C7200090F8701021F00F0141F0020180F870102748007898B92868403001680F682FB9A4
:20C74000D0F80C0580472868006C07687A686178107800F0200020719078E07100E06178D8
:20C76000032903D0022918BF062923D11AF0E2F805466078022815D01648077817B9164973
:20C780000F787FB10221BBF1010F88F8001004D10078832801D112F027FE28461AF04AFAC6
:20C7A000BDE8F88F832088F8000028461AF042FA18F098FBBDE8F88F14010020741B0120CA
:20C7C00004180020D805012058000120D8000020641B01206F1B0120711B01202DE9F04F61
:20C7E0000746ADF11C0D10980D460590287A99461646012818BF032805D127B1FF2F02D0DF
:20C80000032802D10EB90020CFE0694C237833BB0420684B8DF800001888ADF8020019F09A
:20C820008DF90DF104080146404619F053FE684606F0EAFC19F0B2FEBDF8021081420BD099
:20C840004FF6FE71814207D0ADF80200404619F0FEFF684606F0D8FC01202070287A4FF04D
:20C86000040B02284FF000048DF800B015D003280AD001281CBF4FF6FE71ADF80C1017D1BC
:20C880002888ADF80C0012E001A8294619F022FE684611F02DFA38B109E02888ADF8020005
:20C8A00068460FF0D5FA10B9684606F0ADFC287ABDF80C10012818BF049402D1012026467B
:20C8C00004904FF6FE7088426ED0DFF8EC8025460E2015E015FB00F318F80320BA420DD128
:20C8E0004344DDF810C05A78624507D15A888A4204D11A79B24208BF1C1C04D06D1CEDB2B6
:20C90000002DE7D02CB3B9F1000F4DD0DDF814A04F468146AAF1020A3AF8026F2046314672
:20C9200018F0D2F990B984B1607904280DDA04EB4000C6806079294615FB09834A46401C75
:20C940006071022016F0A4FD00E000247F1EE3D12AE02546824625E015FB0AF018F800206C
:20C96000FF2A1DD100EB080408F80070049860706180B9F1040F2671C8BFD94605994FEA1B
:20C980004902A01D84F8059019F008F92B01022029465246A3EB4503434416F079FD03E063
:20C9A0006D1CEDB2002DD7D0204607B0BDE8F08F200901208A010120220100202DE9F04FAC
:20C9C000724C002704F19800ADF1140DB946B846056802978246CDF80C903DB3D4F8AC0092
:20C9E000B84203D1D4F8A800B8421DD0D4F8A8600EB3D4F8A8102869096988421BD195F8AF
:20CA00003300400917D3D4F8AC60A6B90127D4F8A800C06840880028F9D0D4F8A800C06860
:20CA200040880128F3D006E0012704E004F1E000022119F09DFF002D43D087F0010B03A845
:20CA400002AA59460BF010FE5FEA000809D0012F07D0039929B104F5AC7019F071FA4D46BF
:20CA60002FE0002D2DD04A48066856B3B8F1000F27D0039828BBCDF800B002980190D4F8DB
:20CA8000A800D4F8AC100AF108035246B047401E02D0401E08D014E0029800B92846012194
:20CAA0004B460091014605E001230093D4F8A800D4F8A8100069B1F930104A4604F056FC50
:20CAC00060E0002F5ED0002D5CD060682969884252D1B8F1000F0BD0039848B1D4F8A8007E
:20CAE00030B9D4F8AC0018B9082016F0FDFA49E0082018F047FE95F8330004F1E006C0F3F3
:20CB0000001028B9504618F010FAC4F8A80004E0504618F00AFAC4F8AC00A8691D49C043B0
:20CB20000860A8694A6810434860E869C04341F8080CE86951F8042C104341F8040CEC6874
:20CB40000820294618F08AF8204618F051F82088A0F6020040B141F21E01401A04D041F615
:20CB6000E671401A012803D80120214618F076F84FF08041304603E004F1E0004FF48061B0
:20CB800019F0F6FE05B0BDE8F08FC04668F20020080B0120101004402DE9F047ADF1200D8F
:20CBA000109C1D4682460E469046E811002110221FFA80F920460FF011F9C5F3C307D6B11E
:20CBC00004A82146102218F0E9FF20465146102218F0E4FF04A8214616F088F810262246CF
:20CBE00013781AF8011B761E81EA030102F8011BF6D18035ADB24846411E00281FFA81F9E0
:20CC000040F09980002F72D00E2F28DA04A82146102218F0C3FF204600210E220FF0DEF880
:20CC20003A462046414618F0B9FF2E128020E05521461022E5736846A67318F0AFFF04A898
:20CC4000214616F053F810206B46227813F8011B401E81EA020104F8011BF6D187E004A8BC
:20CC60002146102218F09AFF2046002110220FF0B5F83A462046414618F090FF802021460A
:20CC80001022E055684618F089FF04A8214616F02DF8102721466B460A7813F8010B7F1E2C
:20CCA00080EA020001F8010BF6D104A82146102218F074FF204600210E220FF08FF8281205
:20CCC000E57321461022A073684618F067FF04A8214616F00BF810206B46227813F8011B76
:20CCE000401E81EA020104F8011BF6D13FE004A82146102218F052FF204600210E220FF016
:20CD00006DF82F128020E573214620701022A773684618F043FF04A8214615F0E7FF10200C
:20CD20006B46227813F8011B401E81EA020104F8011BF6D11BE004A82146102218F02EFF61
:20CD400020464146102218F029FF04A8214615F0CDFF22460021137818F8010B491C1029D2
:20CD600080EA030002F8010BBFF645AFF3E708B0BDE8F0872DE9F8430646307B8946034689
:20CD800018F0C4FD0125041C5ED1D6F8008077891C461C200DF014F950B100214173047312
:20CDA000478101818173C173C0F8008041614160041C00F0C18000270781307C2074708A4C
:20CDC0006082337C23BB716911B30F460E200DF0F7F8E0B1394691F83820027091F8392092
:20CDE000427091F83A20827091F83B20C270CA8F8280B1F84020C28091F84220027291F808
:20CE00004A2002734A88428191F849104173074638466061308B20836189B07E4FF67F47FB
:20CE20002E46A07607EA0100C108608108D2454914310A78802707EBC2110843608104E021
:20CE4000608940F08000F9E700266089DFF8F080B9F1000FC0F3C21224D10AB3810911D2A4
:20CE6000410909D2C00838BF281C10D319F093FC00F02000801C0AE019F08DFC00F00F00E8
:20CE80000A3004E019F087FC00F07F005F3020810420474660733878202112F0D9F817E00A
:20CEA000002515E0022060732068C089C00803D3404634300088208152B160894FF67F41F0
:20CEC0004FF680770140618107EBC21001436181012E32D1667B27893CB3012E0AD0042E1C
:20CEE00002D0022E0BD020E0042017F07DFF142805DD1AE0012017F077FF202815DC6673E6
:20CF000000202781104960600868002808BF0C6003D00146486830B94C60404600782021C7
:20CF200012F096F809E00146F4E7606908B114F0A1FD204614F09EFD00252846BDE8F8837A
:20CF400050010120E5040120E40A01202DE9F0430E4680460E220021ADF11C0D03A80EF022
:20CF60003DFFB06A417811F01F0F18BF002040F0CC80880924BF01208DF8180031F07F002E
:20CF80001CBF01208DF81700C80924BF01208DF816009DF816200024012A03D0307A00B141
:20CFA000B46902E0F07900B1746934B10DF10E00214619F0A5FC9DF81620554DB189012AA7
:20CFC0006F78ADF80C1020D1287F27F00102104300F09A80002F00F09780022F04D119F055
:20CFE000DDFA884240F09080708914F0E3FC002840F08A804CB118F0A1FD01460DF10E001C
:20D0000018F0BCFC00287FD06F78DFF8089137F0010019D148460078800815D39DF816004F
:20D02000012811D0BDF80C1019F0B8FA88420BD09DF81700012807D0084618F05AFD18B193
:20D04000BDF80C0015F0C4FB9DF81600012821D0BDF80C1019F0A2FA884211D19DF81700B8
:20D06000012808D02C48007800F00700022807D101208DF818009DF818000AF055FB3EE0F7
:20D080009DF817209DF8183008460DF10E0107F089FB34E000249DF818008DF81A4028BB6A
:20D0A0006978074631F0010003D0022908BF251C01E09DF8175019F0F6F8484618300078F8
:20D0C000082818BF042811D14FF6FD70ADF8000018F034FD01908DF809408DF808708DF8CA
:20D0E0000A508DF80B4068460CF0EAFC9DF818000AF01AFB52200DF11A0114F05BFE074883
:20D10000016809B103A88847404607B0BDE8F083E404012082010120501A01201C040120A4
:20D120002DE9F043002507460C22ADF1340D294668468DF814500EF051FE6A4CDFF8A8811E
:20D14000B87804282DD001280BD0062809D0022805D003281CBFB3208DF8140024D11B20CA
:20D1600020E06078D8B919F097FA40B9B9684646082206F11C0018F011FD38883080E079EA
:20D1800002280CD1B8680BA906AA0EF0A9FD9DF8280010B99DF82C0008B9B1209FE02320C5
:20D1A00000E022208DF804009DF81400002840F087803888BE7BADF800003B698DF8056090
:20D1C0007A7B0293012A14BF012021208DF80200684605F0EFFC9DF81400002870D10398A3
:20D1E000466C05233370B8787070796829B9B01C294610220EF0F2FD03E0B01C102218F09C
:20D20000CDFCB8781236012812BF0628F87806F8010BB968304619F05DF9B878083604289B
:20D2200006D0012804D006281CBF387B307004D1AB202946324613F017FA388814F0BAFBAB
:20D2400010B103980421C1829DF81400002837D1B878042809D0386918B9684614F00AFBD3
:20D260002EE068460CF04EF92AE0B8680DF12D0106AA0EF035FD06469DF82D0018B94FF655
:20D28000FF70B0421CD038694FF0010918B9684614F0F0FA02E068460CF034F9B96808A860
:20D2A000082218F07BFC8DF8289028468DF8295031461422079006AB0690042016F0E8F887
:20D2C000607850B919F0E8F938B946462946082206F11C000EF082FD35809DF814000DB0C2
:20D2E000BDE8F083E4040120B4080120F8B5694C2168054614310868407F002800F0C88026
:20D30000D1F8C000B5F84220C08C904240F0C080D1F8581305F128008847002800F0B88076
:20D32000206840690026467721687031486E90F8290028B16068816A0220884721687031A1
:20D34000086890F82B0018B16068816A01208847287C400908D36068816A1020884720683C
:20D36000D0F82813802088476068C16B202088472168C868D1F8FC1410308847686822683D
:20D3800041785269007800EB0120C0F30321517622685269C0F3003797762268526900F086
:20D3A0000F03C0F3031793772068D0F8D40080F82C7022680C32D2F8C81091F84F000F28D3
:20D3C00006D093689B7F984202DD6B68DF780FB19068807F4873106880F83060D2F8C800FB
:20D3E000417B0F290BD19068C07E022850D1D2F8580180472068D0F86C018047F8BDD2F8EF
:20D4000000252846904723680C339868C07E022815D1D3F8F014186888472268D2F8D40044
:20D420001169467BD06831F81630D2F8F0244FF4707707FA06F1C91A904723680C33D3F8BB
:20D44000C8002A89D3F8A83190F82C1002209847206800F11401D1F8C020D0F8D400527B48
:20D4600090F82C0082420FD00868D1F8E81488472268D2F87C015169886050694169D2F8B1
:20D48000F024904721681431D1F8141310208847F8BDC046140100202DE9F047674CA368E9
:20D4A000002589468046ADF1280D002B8DF8245000F0BC802F46FF264FF6FF7AB8F1030F7C
:20D4C00018BFB8F1020F04D193F84200904240F0AD80384617F0A8F8B8F1010F04BF8520A4
:20D4E0008DF82400B8F1000F10D0B8F1030F0DD0B8F1020F08D1A068B9F1000F0CBF012112
:20D50000022180F841100DE0A0680BE0A0680121B8F1030F80F8411004D1B9F1000F18BF2C
:20D520008DF82490B8F1000F4FF0020112D090F84120012A0ED190F8433033B990F84830FC
:20D5400013B15B1E80F8483004E090F84320521E80F8432090F843304BB990F8483083B151
:20D56000A568C26C867B00F12007AD1D05E00746A568426C97F82E60263502EB430232F8CC
:20D5800002AC9DF824308DF8181043BB3FB390F84110012914BF212422247988254BADF8E0
:20D5A00010101978032280F842100DF11A0029468DF8222019F0A4F9CDF800A00DF11A005A
:20D5C0000190029678780390BB7BBA1D04A920460DF040FE1848008817F026F826E0418868
:20D5E000ADF8101009AF009740780190A06848F22002012304A914F02DF804F108052868DE
:20D6000090F8401002290FD1418CADF8101009AF009790F821000190286848F220020123FC
:20D6200004A9203014F016F811F09CFD0AB0BDE8F087C04628040120E40601203C050120AB
:20D640002DE9F047634F8046381D0068416EADF1280D02A888475B4D2A68403210680068C1
:20D6600020B9D2F80C0580472A68403256484FF001096E6880F80090F068007830B9D2F8E3
:20D6800018244846002190472A684032106801684C68088921788246C1F3401109F01CFE25
:20D6A000079010F095FD494E746786F873A00024A6F8664019F03EF9059482463146B8F115
:20D6C000010FA6F8664004BF4148C1F8B80038F001083E4654D1A1F89E4001F16400C1F8D9
:20D6E000A00091F8A90002231A4602F00F0220F00F00024381F8A92091F8A80004F00F07EF
:20D7000020F00F0047EA000291F8B3708C6627F00F0081F8A82040F0040009F00F0291F8EB
:20D72000717081F8B30027F00F00024381F8712028684030006800684268127801F1640706
:20D7400092090FD301F120028A66406891F87150807803F00F0381F82E0025F00F00034348
:20D7600081F8713001F1100001F19C0242604A7F04F00F0322F00F0213434B77014601E029
:20D7800064310F467068174A056D08238DE81800114B106802AAA84710490028088006D4EA
:20D7A0000F4991F90000B760401C087004E0484641F2883110F06AFF504619F03BFA0AB047
:20D7C000BDE8F08714010020B30A012058000120801A0600D405012021A90000D40A01203E
:20D7E000B60A0120B40601202DE9F04FDFF898910646A9F1080000F108078068D0F8000179
:20D80000807AADF12C0DC0000CF0DAFB0028089008BF1A2500F0B48019F08CF800244FF0CC
:20D82000FF0B25460A9027E0ADF800608DF80240D2F88823D02069469047D8B99DF80C00E9
:20D84000012802D19DF80B1019B998B99DF8071081B1002814BF082304230DF103005B1E54
:20D8600000F801BBFBD105703868D0F894246946D0209047641CE4B23A6802F58072106804
:20D88000C07AA042D0DC4C462068D0F80001C0884FF6FF78AA461DE0089901EBC0018A888C
:20D8A00096421CBF401CC0B261D1C1F800A0A1F804803A68D42004A9904702E07F1CBFB237
:20D8C00025E020682268D0F800016D1CEDB202F58072C088A842D8BF55464BDDADF80060C6
:20D8E000ADF80250D2F88823D120694690470028E7D1BDF804008045E3D0ADF810002068F7
:20D90000D0F8882404A9D420904790BB5746226802F580721068C088B84210DDADF8006014
:20D92000ADF80270D2F88823D120694690470028C4D1BDF81000BDF804108842BED12068B8
:20D94000D0F80001C088B842BBD1ADF81480ADF8168006A8594608220EF040FA2068D9F8B4
:20D96000003000F29447D3F80001837A5046834292DC19250A9819F05DF9089814F07AF8C3
:20D9800028460BB0BDE8F08F140100202DE9F04160485F4E614C604D70601030B06004F1FA
:20D9A0004400B0E88C1005F17C01A1E88C108DC881E88D00182204F1140705F13400394619
:20D9C0000BF0A4FA1822394605F14C000BF09EFA05F164071822384604F12C010BF096FA5A
:20D9E00095F870003C2204F1840140F0800085F8700005F1BC000BF089FA95F8CB100120FC
:20DA0000024602F0010221F001010A4385F8CB2095F8CB1060F3820185F8CB1095F8CB1003
:20DA200021F0200185F8CB1095F8CB1060F3C71185F8CB1004F16401B1E8085105F19C0291
:20DA4000A2E8085191E80A5082E80A50C5F8A07095F8A81060F3C71185F8A81095F8A91094
:20DA600021F00F0141F0020185F8A910042385F8AD30052185F8AC1095F8AE1000F01F02DF
:20DA800021F01F010A4385F8AE20032185F8B01095F8B31000F00F0221F00F010A4385F820
:20DAA000B320B4E8841005F12001A1E8841014CC81E8140095F82C1060F3C71185F82C1025
:20DAC00095F82F1003F00F0321F00F010B4385F82F3095F82F1060F3C71185F82F1095F8EA
:20DAE0002D1000F00F0021F00F01084385F82D004FF4586028630A48F0600A480068406949
:20DB0000007808B10CF08AF90AF0BAFCBDE8F081A40601205817002058000120207B02001F
:20DB2000140B01201801002001282DE9F84F40F0B080DFF88491D9F83401012840F0A68015
:20DB40000220C9F8340117F0C9FD012015F05EF85FEA000805D00120C9F8340117F0CCFD57
:20DB600099E0112018F074FD00280CBF00250125102018F06DFD08B145F002050F2018F076
:20DB800067FD08B145F00405444CA06A0068014601208847012805D099F83801012818BF29
:20DBA000002703D1002004F045FD012718F04AFDDFF8ECA040080AD20026206A8068014637
:20DBC000504688478346BBF1040FF6D000E00126304600214FF0FF3201F08EFF012E0ED0F9
:20DBE000BBF1010F05D1206A4068012102465046904732496C39086840F0030008602068D7
:20DC000040690146284688470B2018F021FD254E30B12068C06A3146091D02460888904734
:20DC20000A2018F015FD28B12068C06A31460246088890471C4903200124C9F834011B4EE3
:20DC40000C6000233360284612F05AFD0128FAD1174D2868042014F0D9FF064615480460E6
:20DC60002868012F02D1204604F0E4FC18F0BAFC082014F0CBFF0746C9F8344117F03CFD60
:20DC800057EA060018BF4FF0FF3804E06FF0040801E06FF001084046BDE8F88FB8010010DD
:20DCA000004003406A810200282008600C2008402C2009400C400940501800209022084024
:20DCC000F8B5074661485F4C001DC26A0168B7F5C067C2F30722C4F81071C1F38441C4F821
:20DCE0001421C069C4F81811C0F38120C4F8280100F0A38094F830616EB9C4F82C71D4F82C
:20DD00001801C4F82001D4F81461C4F81C61D4F82851C4F82451D4F82C01D4F814510028CB
:20DD200054BF02236FF0010304F59072116800EB4000C018431000EB937001EBA001116092
:20DD4000D4F82011C4F81C5100291CDD1E293DDDD4F8240130B93429B4BF15391E21C4F827
:20DD6000201125E02A29BABFD4F820010B381E20C4F82001D4F81C013E28D4BF401C3F20B9
:20DD8000C4F81C011FE0D4F82401032812D011F10A0FA6BFD4F820010B300120C4F8200107
:20DDA000D4F81C010028CCBF401E0020C4F81C01032009E011F1140FA6BFD4F820011530A8
:20DDC0000120C4F820010020C4F824014FF08057D7F8A401B4F81C111B4D40684FF47F42CD
:20DDE00008230646009128463021B047D7F8A40101214FF40032112340680091064604217C
:20DE00002846B047D7F8A401B4F8201140684FF4F80212230646009104212846B047D7F8FC
:20DE2000A401B4F8241140684FF440620A230446009120212846A047F8BD002084F83001AF
:20DE4000F8BDC0465018002000A00C4000A00C402DE9F84F604B5879002840F0B88000201E
:20DE6000012117F0B9FA002800F0B1800668002E00F0AD800746594A408951789246C2099F
:20DE800070D231F001054FF6FE7465D1994699F83220920860D3326A51791579400B05EB6E
:20DEA00001252CBF402600263868B7F818800088834613F07FFD002840D15846032113F010
:20DEC00095FC002838D15846002113F057F831460EF084FD061C2AD07079012804D003284C
:20DEE0001AD0042818D12AE0B179708811F0180F0DD0FF21A842317103D0404518BF844251
:20DF000008D128464146224606F016FF02E099F838103171844208D17079022807D058463C
:20DF2000072113F063FC10B106E0834604E0584617F082F9044602E05846FBE7641CA542D0
:20DF400002D0388BA04213D1386801880222002328460EF089FA0FE0022909D118F01EFBF2
:20DF6000044605E038680088044613F023FD28B94FF6FE70A04203D1CD211EE04FF6FF74EF
:20DF800038680480204613F015FD00280CBF012000203968C8810F4938680AF055FC011C64
:20DFA0000BD19AF8010002280CD19AF8000048B92020012101F0F2FC04E03868407B13F0D5
:20DFC000FDF820B91FB138460121FEF7D3FEBDE8F88FC046452C020050010120E40401201D
:20DFE0002DE9FE4F5D4C5E4994F83C80B4F848500A68834601A8026049684160DFF868A16A
:20E0000001A80AF11409494617F0B8FC00280CBF01260026A76887B11EB93888854206D03A
:20E0200008E007F10C00494617F0A8FC10B1B878804502D0BF69002FEED1002F08BFCA203C
:20E0400000F0898039894FF6FE70884208BFC32000F0818018F0B4FA884208BFC2207AD07A
:20E060003888A84218BFA4F8480016F06DFCF87A4946401C84F85C0004F15D0018F040FC01
:20E0800002208DF80100684616F0E6FF04F12405061C5BD03069062100F8011B94F8321032
:20E0A00001704FF0010986F81E9017F047FD706286F81A904020F0823889708086F818B06C
:20E0C0003046FCF7C5F8061C41D1092084F84A003B89E38794F83C00804518BF84F83C802D
:20E0E00005F11A014B2013F065FE05F12401502013F060FE05F11801E12013F05BFE05F1F0
:20E100001601532013F056FE0820494601F046FC4FF40050002101F041FC20784FF4806196
:20E1200010F000FD0F484178022905D10078012808BF4FF4DC6203D008200FF005FD82006A
:20E1400020784FF4806118F0B7FB00E0102600208AF805003046BDE8FE8FC046500101206C
:20E16000987C0200E4040120C40301202DE9F04120F039055C4E5D4C96F82F00ADF1180D30
:20E18000002840F08E803078042113F053FC002840F0878096F82F10777805F03F0541EA7B
:20E1A0000500012F41EA050186F82F1001466FD04FF0010806F132035520002186F80180AD
:20E1C0001F46424617F0ECFF387801285ED12078012818BF022842D1454804680021204603
:20E1E00017F01DFC00283AD118F08EF8002836D1204605A96A460DF073FD04469DF81000EF
:20E20000FD282CD002282AD0C82C16DA6846002114220DF0E3FDFF20214614226B468DF801
:20E220001000042015F034F93249A000002200EBC4000A5009184A604A720024552041468B
:20E240003A4686F8324018F06FFAFF20032114F0BDFDF4713078042110F0FAFE40E096F804
:20E260002F00072440F01000F471284386F82F0000200146F5F706FE002831D0002015F0E2
:20E28000E5FB20460021F9F777F929E096F82F103078002904BF0724F471F2D00021F17178
:20E2A000D9E7307AE0B9217896F82F00022901D1810915D296F832706FB1A9080BD341096E
:20E2C00009D217F0C1FA04200121F9F755F996F82F0085F0020505F03F05054386F82F5066
:20E2E00006B0BDE8F081C04668060120E5040120EC06012004E900202DE9F8435F4CDFF8C0
:20E3000068815B4DD4F83C0100286ED0574E401E0AD0401E60D0401E1CD0401E53D0401E69
:20E320001AD0401E33D02FE04E4801250221006884F83A51702204234068009100210746D5
:20E340004046B847356004F1500018F0EBFA2846BDE8F883022100E003214FF08059D9F8D3
:20E36000A40184F83A1140680025702204232946074600954046B847D9F8A401C0687022A5
:20E38000294613460125DAE70320BDE8F88300262E606E6028688008FCD268688008FCD2FD
:20E3A000374834490127001D06600E200F6008F059FD022015F05AFAC4F83C6184F83B61DF
:20E3C0000220BDE8F8830520C4F83C010027376030688008FCD242E00320C4F83C010027CC
:20E3E000376030688008FCD239E0234F01260F202E6042F62A21C7F80B004FF08059C7F805
:20E400000F10D9F8A40140684FF4C072072302218446404600910021E047D9F8A401C06836
:20E4200000214FF4C072072384464046E0472E6028688008FCD394F83901C7F81B6018B95F
:20E44000032100200E4602E0002028630321C4F83C6147F8011C686068688008FCD20020B0
:20E46000BDE8F883A401001000A00C4058600C4054600C4004800C4001400C4050180020F2
:20E4800038500C402DE9F8430446DFF87C81A078471E53D07F1E40F0B480814600252C2060
:20E4A0008DF8005016F052FD071C04BF01208DF80000E41CA078002818BF02283AD19DF8C5
:20E4C0000000A8BB14F8010BB87014F8010BF87014F8010B387130B92046042116F0FAFFE5
:20E4E0000C34B86007E0241D07F108000822214617F054FB083414F8010B387414F8010B9D
:20E50000387514F8010B10222146787507F11C0017F044FB042104F1100016F0DBFFB86133
:20E520000820387046467D703078394612F05AF96B4661E002208DF80000F9E78146E41CD6
:20E540000026607C8DF801600546183080B216F0FDFC071C04BF01208DF80100A078002842
:20E5600018BF022843D19DF80100002842D114F8013B304603B10120B87014F8010BF8707A
:20E5800014F8010B387130B92046042116F0A2FF0C34B86007E0241D07F10800082221468E
:20E5A00017F0FCFA083414F8010B387414F8010B787414F8010B2A462146B87507F117002F
:20E5C00017F0ECFA641914F8010BB87414F8010B787514F8010B0525387520783D70F874E8
:20E5E00043467E701878394612F0FCF802E002208DF801000DF1010375204946012213F0C9
:20E6000007FF0020BDE8F883E80901202DE9F84F534D2968D1F8D40090F883A040310868EB
:20E62000006820B9D1F80C05804729684031886F4C4EDFF83491DFF834810078E8B918F01C
:20E6400079F9377883464FB949460F7837B9832041460870584618F0EDFA60E002214046AA
:20E66000BAF1010F017004D13078832801D110F0BBFE584618F0DEFA65E014F08BF83C48ED
:20E6800000683C4F016C38688847044618F052F9824630460778002F44D149460F78002FC8
:20E6A00040D12868D0F8B800C16C002088472868D0F828246946F42090479DF90000A04267
:20E6C0001EDC2D4CA079D8B9504618F0B3FA6078042803D02868D0F84C05804704204146E0
:20E6E000A7792E680870781CA071D6F8B800C16C09B103208847032060810FF001FD22E0E5
:20E70000832041460870002014F05AFE504618F091FA1A486968C01D09690078087016F03A
:20E72000E1FB10E0022241460A700078832801D110F05AFE504618F07DFA2868D0F8B80076
:20E74000C16C042088476868C068007828B92868D0F85824002001469047BDE8F88FC04604
:20E76000140100206F1B0120711B0120741B0120D8050120B406012004180020051800200A
:20E780002DE9F04106467468B56818F0D3F8D4F8C0108046002900F0A18094F8F80028B919
:20E7A000087C032818BF042840F09D80287918F0C3F8D4F8CC0041686F690968CF6294F8AF
:20E7C000F90018B92968C8684009FCD22968486820F002004860D4F8CC0041682F69096852
:20E7E000CF622968486A20F003004862D4F8CC002A6941686B69096843EA0200C1F80405DE
:20E800002968486920F001004861286801270762D4F8D400D4F8C0100860D4F8D87067B10B
:20E82000E8698068C0F30910401C874205D3D4F8C0201168C919091A1160D4F8DC7067B10B
:20E84000686A8068C0F30910401C874205D3D4F8C0201168C919091A1160304610F03AFDED
:20E86000287918F063F8287918F068F8D4F8C070386857B100230222397C03291CBF0429B7
:20E880003A743B607F69002FF6D1D4F8C0100860D4F8C8100022002904BFD4F8C000C4F853
:20E8A000C80004D04869B8B9D4F8C0004861C4F8D020C4F8D420C4F8D820C4F8DC20C4F8E1
:20E8C000C020C4F8C420404618F0B4F904F1300018F050F8BDE8F0810146E3E729684868A0
:20E8E00020F002004860404618F0A4F9BDE8F081F0B504466568267A00213422ADF1740D2B
:20E9000004A80DF06BFA8DF810606978287800EB012004A913F069FC02208DF811009DF805
:20E920001000AD1C801E8DF82C00608E0E9504F12801ADF81E0019A817F03CFC9DF8120096
:20E94000032840F0868017F035FE9DF8131088427FD19DF814109DF815009DF816709DF837
:20E960002D609DF817509DF81830084347EA000146EA010045EA000153EA010069D111A822
:20E9800000211C220DF02AFA0E9DBDF81E202846ADF84E209DF82C1010F8017B07F0030287
:20E9A0008DF84470D21E1ED107F00C06082E14BF002301238DF850300C2E06D14678037897
:20E9C000801C03EB0623ADF8483046780378801C03EB0623ADF84A300378467803EB06230C
:20E9E000ADF84C30801C1590401B081AC0B28DF85800091A8DF851105ABB07F00C0004289C
:20EA000027D007F0200127F07F00084321D1FE2794F94830104894F8466094F847508DF8B8
:20EA200047709DF823208DF86230007800928DF860608DF8615000270197E16B0291039773
:20EA4000B4F842208DF8460018AB11A819A909F02DFA1DB0F0BDC046C80A01202DE9F043C3
:20EA6000584C94F84201ADF1140D002840F091804A484B4E4FF00108027B3368416884F84B
:20EA80004281814684F84121C3F38147C4F86C11BFB9D9F81000A0B156F8085C17F06CFD8B
:20EAA00064210246C5F306604143B1FBF2F23D49002304F1940012F0FDFE3B494FF0004025
:20EAC000086001A817F053FE00252F4604F10C00029501AB8DF80470344903953A4612F05F
:20EAE000E9FE01A817F043FE04F150000822029501AB8DF804702E49039512F0DBFE2D4A32
:20EB000004F1D80032213B4613F012FB2B4A2A4F04F1F4002C212B463D6013F009FB306873
:20EB200099F80D30C0F381501BB1032803D184F8398103281FD002281DD001281BD14FF0FD
:20EB40008059D9F8A4011E4C406803214FF040521C230746009129462046B847D9F8A401F8
:20EB6000406829464FF4007209230746CDF800802046B84706E0386840F0400038600220F6
:20EB800014F08CFE56F8040CC00802D2284614F085FE05B00020BDE8F083C046308602004D
:20EBA000B44F0050555E020000A10C4003950100ED0E0200994902009022084081C80100A2
:20EBC00000A00C40501800202DE9F0430E460024ADF1240DADF8160006F108078DF8144097
:20EBE000384616F068FC50B905A80DF031F9A124012840F0938005A814F078FD8EE038460D
:20EC00000DF122016A460DF06BF805464FF6FF70A8427FD09DF82200DFF80C81002834D044
:20EC2000404801789DF8100040B3401E1AD0401E04D0FB381DD0801E1BD051E0012915D0D8
:20EC4000022913D039B9748240F20110B0829DF8127086F8287006F11E0002A9082216F02C
:20EC60009DFF3DE0012918BF022902D14FF4817001E040F20310B082748231E005219DF88E
:20EC80001300718200F07F0029E002A83946082216F084FF4FF001098DF81190FF208DF807
:20ECA000100017F078FD274600F00F0000942946142201976B468DF81200042014F0E8FB38
:20ECC000AF0007EBC507404621460C223F1838460DF084F8748287F8099040F20310B082D9
:20ECE000A8003474414600EBC5000A58B2610F580A237F1CB7FBF3F20F505A43BF1A0DD19F
:20ED000040180121094F017238784FF4806110F09FF903E0748240F20310B082204609B0D3
:20ED2000BDE8F083E504012004E90020CB0301202DE9F04F044608469A46ADF1240D2146B2
:20ED400005908E680692129B04914C68756807935044854238BF6FF00304C0F093804B4D10
:20ED600028684FF0FF3117F095FA4948328C079F48496368026083460B60780819D238462E
:20ED8000800813D3F768002F3AD03569002D37D000970195012002900599069A0498534648
:20EDA0000DF036FA5FEA000813D114E04FF0000811E0A0683AEA00070AEA00021CBFB168A8
:20EDC0000A4405990140049808F09CFB5FEA000801D0044652E034680598DDF818905746EA
:20EDE000241805E0BBF80010049817F02FFAA944AFB90798C00840D3F16809B1306910B91F
:20EE00006FF007043AE00091019000270297069A0599049853460DF0FBF980462DE00498B9
:20EE200010F082FD38BB049814F048FA18BB04F0FF05C5F58075BD4288BF3D1C210C8DF8B3
:20EE40000D1002208DF80F40230A8DF80C00BBF8001004988DF80E3017F0EFF903A8042100
:20EE600011F09CFA7F1B641928B94846294611F095FA0028B6D04FF0FF3844460348006815
:20EE800017F06EFD204609B0BDE8F08F141B0120101B01200C1B0120F0B50446207CADF1B0
:20EEA0003C0D0F28C0F2A680656860690DF1260210F0F6FA9DF82600002840F09B80207C84
:20EEC0000B28C0F29780287A022840F09380A88900F00F010F2940F08D80C0F303100F2884
:20EEE00040F088809DF82860002E18BF022E40F08180414C414894F84A20022A3BD00068AC
:20EF0000062A39D010B18179012935D0082A18BF042A6FD16D8910B18079022827D0B4F8DA
:20EF20004800854266D1012E07D004F15D000DF12D0116F023FD00285CD120784FF4007140
:20EF400012F078FD002855D1E06C029001268DF80D6002238DF80E3094F852708DF80C70BE
:20EF600002A80FF0AFFD10B114F008F842E0284615F06EF93EE0006840B900230093288896
:20EF800069896A7CFCF73EFF9DF828602888ADF810006889ADF81200A87B8DF81400AF894B
:20EFA00000206FF30E0707B101208DF818608DF815009DF827408DF819409DF82C708DF8BA
:20EFC00017709DF82A009DF82B308DF81600687C0DF12D018DF81A009DF838608DF81B30B4
:20EFE00008228DF81C600DF11D0016F0D7FD04A803F03EFC0FB0F0BD50010120000A01200F
:20F000002DE9F04380460E20ADF1340D15464FF001098DF80100B8F1000F8DF802305048A3
:20F020008DF8005000F1010000788DF804900F468DF8030047D1112004A93A2217F05FFAE9
:20F0400000283CD1444E0DF111007B199DF80320716803901C4642F02802481C7060581CBC
:20F06000227016F08FFD054616F068FD0146284617F046FC48460DF131013A2217F03FFA5E
:20F08000083500280CBF9DF831000020287016F055FD01460DF1210017F032FC7088401C7B
:20F0A00080B27080B0F57A7F02D8706801282FD12A4800784FF400710FF0CAFF28E0002027
:20F0C0007C19039024E07C19ED19687B11F076F83A2808D03B280FD1112004A93B2217F058
:20F0E0000EFA30B108E0112004A93A2217F007FA10B90DF1110000E0002003909DF80300FA
:20F10000217808432070611D0DF1210017F0F8FB0DF12900611C042216F040FD039E20789E
:20F12000002E8DF82D0008BFA12012D0404669460DF121023B4604F0EBF8054620780021D3
:20F14000102200F0F80020700DF111000CF046FE28460DB0BDE8F083100A0120CB03012049
:20F160007F0101202DE9F047564CA4F1080000F108058068D0F80001807AADF1280DC00026
:20F180000AF01EFF0028089008BF1A2400F0958017F0D0FB8246286800F59162D0F80001B3
:20F1A00000894FF6FF780026C14608E020682268D0F80001761CB6B202F591620089B042BB
:20F1C000D8BF002473DD2068D0F80001C07A0127002548E0ADF81480ADF8168006A8FF21E2
:20F1E00008220CF0FBFD2068D0F8942404A9D42090472068ADF80480D0F894246946D120A0
:20F2000090472068D0F800012268C0886D1CEDB202F5916230E0ADF800608DF8025012687C
:20F22000D02069469047A8B99DF80C00012810D19DF80B0068B90DF102020820002112F836
:20F24000013FFF2B03D1401E01F10101F7D10829ACD0002720682268D0F800016D1CEDB27F
:20F2600002F59162C07AA842D5DC002F9ED12068D0F80001C0880025A84297DDADF8006010
:20F28000ADF802501268D120694690470028B8D1BDF804008145B4D0ADF810002068D0F8CD
:20F2A000882404A9D4209047002893D01924504617F0C0FC089812F0DDFB20460AB0BDE8CA
:20F2C000F087C04614010020F8B50546687F0C4600280CBF08201020AF7F0FB10830C0B268
:20F2E0002F7F0FB1401CC0B2AF7927B1297A00EB4100801CC0B22F7E6870002F0CBF002650
:20F300000E2647494A78022A0AD10A7D012A07D12A78012A04D0CF78002F18BF012100D1F5
:20F32000002185F834102F7E297D09188919217037B13C48007816F079FC2178081820709C
:20F340002078742869DC0AF03BFE071C66D017F031F90346A97F6A7F95F834002C7F41EA86
:20F360004001A87942EA410240EA42012A7E002042EA410204B10120297840EA42006A7E4D
:20F3800041EA830102F0030241EA821141EA002188B2397000127870A878B8706888001296
:20F3A000F87028793871A88800127871A87EB871E87EF871687F002808BF082405D0296AE8
:20F3C00007F1080017F09CFA1024A87F28B1696A381917F095FA0834E4B2A87988B1287AD4
:20F3E0003855697A631CD8B239542A7AE968431CDCB2E019520016F0D1FB287A04EB400433
:20F40000E4B2287F00B13855687829692A7D8019C0B2C01916F0C2FB00E000273846F8BD77
:20F42000E4040120800101202DE9F0470546A87A022840F09B804E4CAF7B5248DFF840A1DC
:20F44000A66A002F7CD12169F9B16769EFB1A769DFB1E768CFB114300078012815D1688852
:20F460008847AE1C88B943490A6830889101A1EB820162699047012878D1A16930888847B6
:20F48000E16830888847BDE8F0873B486D88006878B101680A88954208D1096A4A78097816
:20F4A00001EB0221490A01D220B136E040680028EFD10020314933230027012401F60C72EF
:20F4C0001679FF2E02D01688B54206D05B1E02F124024FEA4404F3D100E0274601F1AC0869
:20F4E00001F13C09002319F803208AB19E0058F8064027420CD0104616F008FA38B1417BC7
:20F50000052904D1BC431E2348F8064000E000205B1CDBB21E2BE6DB68B1417B05290AD136
:20F52000016801270D8056464773307820210FF08FFDBDE8F087284611F0D0FABDE8F08772
:20F54000A6B1017D012911D1C07840080ED3042015F0FCFC011C09D06420087001274F706F
:20F56000688856464880307811F03CF9BDE8F087E4020120BC800200E40A012020010020A8
:20F5800050010120E40401202DE9F0478A46071CADF1200D08BF002000F099804D480088D8
:20F5A000B8420AD116F0CAFA0146504616F0E6F900280CBF0125002500E012254FF000094D
:20F5C000ADF8027068468DF800900CF041FC68B101AC204615F06FFF012807D1504621467B
:20F5E00016F0CCF900280CBF01254D46DFF8F0804146087830F0010044D1122D42D1504628
:20F6000017F04EF928B101888F4202D00679052E03DBB9F1000F34D134E00780EEB1414688
:20F62000491E0D79032E18DA2B493DB901EB8502126B01EB8501C261096B0AE001EB8501FB
:20F640000B6B9A01A2EB8302C2610A6B9101A1EB8201816180F8209003E06FF00101C161DE
:20F6600081614E46C6600125ADF8107051468DF80E500DF1120016F02DFF0DF10E0003F0E8
:20F68000C3FD4D463846514610F028FF0A2818D0A02813D1114C142604F102084046514662
:20F6A00016F06CF930B9761E04F11C0408F11C08F4D100E02780384612F07CFC012D01D0ED
:20F6C00004E001253846494614F0DEFB284608B0BDE8F0878A010120688002009C0400209E
:20F6E000E50401202DE9F041054603200C46ADF1300D8DF81E000DF1160017F001F916F060
:20F700001DFA01460DF1160016F038F9002878D0217D032918BF012973D1207A00286ED0C1
:20F72000FE286CDC032904D1A07D002867D0FE2865DC3E490A6809A80260496841603C4F8E
:20F74000082209A9384615F0F7FCC8B9AE1C394831880088884213D0608988B900208DF8CE
:20F7600008003946082203A816F018FA02A80EF0BFFA3088BDF80A10884218BF8D2042D1CC
:20F780002D48EB890768AE1C212B11D02B48076867B1207A6189A37D04F10C02B84728B999
:20F7A00000208DF82C0012F0C5FA2EE088202AE08C2063898DF82C00ADF822302FB30DF1D7
:20F7C00022000090A27D207A04F10C010123B847D8B100278DF82C7012F0ACFA207D032858
:20F7E00013D104F10C0008A913F068FF04F10C0858B9394640460A460FF024FA05E08220F6
:20F8000000E08420AE1C8DF82C000BA80090287C0190EA893146012305F1110042F40042E4
:20F8200011F018FF0CB0BDE8F081C046E48702004C0501208A01012024090120F0060120E8
:20F840002DE9F041524D2968F4310A68064692F84400ADF1180D82281ABF92F84400401C10
:20F86000002082F84400086890F8441000EBE10090F82C104A1080F82C2048080AD22968F3
:20F88000F4310A6892F84400401C82F84400C0B28128E8DB2A68F4321168DFF8F88091F802
:20F8A0004400812824DB8878E8B944462168D1B10868C0B10F4615F0ADF98046386817F0D8
:20F8C0008BF810B1386817F095F9384617F08EF9384612F0CFF8083C0020A060404616F06C
:20F8E00024FB2A68F4322A203070D2F84C1249E0D2F83C234431E12090472C684FF6FF7335
:20F900000220ADF80830F43422688DF810009778BFB916F031FE4FF47A71B1FBF0F01E49C4
:20F92000434600220AF092FB00282DD02868D0F8F4001A2141702A2737702868D0F8401395
:20F9400020E0022F1CD0012F19BF07208321082080210027009749320192D4F8844202AAE4
:20F96000A047DB2807D0E52805D0F32803D0DF2818BFE82808D12968D1F8F4104870DAE758
:20F98000D4F874133046884706B0BDE8F081C046140100207C0A012091590100FEB5524DE4
:20F9A0006A78022A04D12A78012A04BF4F4A10404F4CB4F8707000290CBF87430743F80BB9
:20F9C000A4F87070C60308D001208DF8040001A9522012F0EFF9B4F87070B80B62D2F80BD4
:20F9E0000026C30358D1002F5AD06B784FF0FF306E460090022B4AD12D78002D47D1780852
:20FA000006D304F14C000168B1F1FF3F38BF061C380906D304F1500032680168914238BF3E
:20FA2000061C780906D304F1540032680168914238BF061CB80906D304F158003268016828
:20FA4000914238BF061CF80B06D304F15C0032680168914238BF061C780B06D304F16000ED
:20FA600032680168914238BF061CB80806D304F1640032680168914238BF061CF80806D3DD
:20FA800004F1680032680168914238BF061C6846B04208BF002603E0F80B28BF04F15C0669
:20FAA000374600E00027134D2878BFB1E66E1EB131683A68914215D03968E766012909D04B
:20FAC00001210FF02FF8E16E28780A68012116F0F0FEFEBD01210FF0BBFAFEBDE7660121AC
:20FAE0000FF020F8FEBDC046E4040120C0CFFFFFE4020120500101202DE9F0478246484E74
:20FB00004E4C56F80C0C9046894680082AD245480068810D28D2051704F13400006800682A
:20FB200080476D1CC0F13E0110F1020F4FEAE101D8BF07218D42B8BF0D1C3B480068C0F38C
:20FB40000320401B102803DA0028D8BF012000E00F20364900F00F0040F0F00081F84D00BF
:20FB6000087801E03248306000203249324F256808603868A96927208847324D304805F154
:20FB8000300211682B460840106003F17800006820F48070A8672068016B4FF480608847C4
:20FBA0002068016B4FF4816088472068016B4FF4C0608847244901200860C5F880912860EC
:20FBC00056F80C0C800806D2B8F1FF3F14BF40464FF0404030603868E8698008FCD3072061
:20FBE00010F0AAF80228FAD1BAF1010F13D0206A164E8168304688470428F8D0012804D1C2
:20FC0000206A4268032130469047D5F8180220F00300C5F818022068806B8047BDE8F08718
:20FC20001C000940B44F00500C1300500D620840FD0000400C4009402C200940B8010010B6
:20FC4000FFFFFEFE0C2008402820086000400340F0B5524C06466078ADF1240D022803D1CF
:20FC60002078002800F097804D4D95F84A00082818BF042840F08F8030460DF10E0115F052
:20FC800076F9607802280BD115F058FF04A915F075FE28B116F094FCBDF80E1088427AD040
:20FCA0004FF6FF7012F086F9BDF80E0004AF3946FFF76AFC01286ED00DF11A0016F0C7FD75
:20FCC0000DF11A00394615F059FE58B1BDF80E2016F064FC904205D005F13E014B200A800E
:20FCE00012F068F8607830F0010019D116F068FCB18A884214D004A816F0D2FD38B1007989
:20FD0000012818BF022802D104A80FF0D9FC2548016829B1207D012802D1BDF80E0088478B
:20FD2000BDF80E00002114F0ABFFBDF80E0014F01FFE00248DF80040BDF80E00ADF80200FA
:20FD400068460CF085F898B10DF11A00214608220CF044F801AC0DF11A00214615F00EFE15
:20FD600030B104A9204616F0B5FB684603F04CFA01A804A916F0AEFB68460DF0B9FF50B189
:20FD8000BDF80E00BDF80210884204D0ADF80200684603F039FA09B0F0BDC046E40401204B
:20FDA00050010120F00201202DE9F04F00210225C41CADF1540D8DF84A1081788DF848504D
:20FDC0002046139116F02CFCA41CADF84000204616F026FCA41C8146204616F021FCA41CE8
:20FDE00014F8018B8246B8F1110F0DDAB8F1000F0DD047466E46204616F012FCA41C7F1E46
:20FE000026F8020BF7D102E080208DF84A002678112E63DA5EB1641C37460DF1200B2046E9
:20FE200016F0FEFBA41C7F1E2BF8020BF7D19DF84A00002855D1304A53684746BC1948461C
:20FE4000514614FB05F4A41D5FFA84FCBCF1500F42DC9DF848400F2C18BF022C08D1BDF854
:20FE600040504FF6FF74AC4204BFA41EADF840404FF6FF74844208BFA01E03F8010B001286
:20FE800003F8010B03F8011B0D1203F8015B03F8017B67B168469B1E017803F8021F30F81B
:20FEA000021B7F1E4FEA21215970F5D19B1C1E705EB15B1E08A8017803F8021F30F8021B27
:20FEC000761E4FEA21215970F5D1104610A9634606220EF0E1F802E0102000E080208DF8B6
:20FEE0004A001399652001220DF14A0312F090FA15B0BDE8F08FC046280401202DE9F04FFC
:20FF000015460646287A0C4600F03F01E8886FF39F2040EA0130A988ADF1140D6FF39F2118
:20FF200041EA003B49490E9FC8789A464FF0000988462EE09DF80B10C8080CD3BDF80E00B6
:20FF4000844204DD241AA4B2162C13D931E02146304610F021FC0020F8F776FC98F83300E9
:20FF600098F803204FF00009401C90FBF2F15143401AC6B298F803008119491E91FBF0F254
:20FF80004243891ACEB2B10001EBC6014144B1F84C40484503DC0020A8810A2052E098F8FA
:20FFA000323009F10101B3421FFA81F9E4D0172CE2D3E41F30466A46A4B2214608F0D2FD02
:20FFC0009DF80B108808B7D34808B5D22A7AEB881AF00F0018D0401E12D0401E07D0401E95
:20FFE00018BF04202ED100985845A5D10CE09DF808009042A0D1BDF8060098429CD103E0AB
:020000040001F9
:200000009DF80800904297D1AFB10AF0F000102811D1BA89BB68684600210EF0BDFF00288E
:2000200088D1F988B868BA884018396814F0CAFE00287FF47FAF68460EC80EC503C885E867
:200040000300002005B0BDE8F08FC046C01900202DE9F84F504CD4F8A000D4F8A06000284C
:2000600000F095800546E86840F6030108274A1C02E040687F1EFFB260B15FB103889942B2
:2000800018BF9A42F5D129692CC838312CC189C881E8890006F1280090E800034FF0000AE5
:2000A00006F12807D34687E8000CB16821B357464FF0E24A07EA08001AEA090508BF002897
:2000C00013D036A090E80C0002EA080213EA090308BF002A04D0B5683069B6F93010A8478B
:2000E000504607EA080800EA0909B5683069B6F930104B464246A84716F01CFC0546B4F9AA
:20010000B600401C6FF31F30A4F8B600214886F833B06FF00207378614F007FF284616F05D
:2001200089FDB4F9B400B4F9B61088422FD16068D4F8B860D4F8BC7090F8FC1000290CBF6F
:20014000052007200AF03CFF58462EB196F8FC5005B9306886F8FCB05E462FB197F8FC50E8
:2001600005B93E6887F8FCB0864238BF061C66B1B6F1FF3F0BD016F0FFF9B6FBF0F104F5AF
:20018000CE7015F0DDFEBDE8F88F15F0D1FABDE8F88FC04608F3002068F20020F0FFFFFF91
:2001A000FFFFFF8E2DE9F0478046D8F808603068076CD8F8045047646A6CA96B286C17F406
:2001C000F06FA0EB020937D1F8091FD2780979D3B9B196F82100464A145C601E814294BFB6
:2001E0000C1C641E4046214612F064FDA86B001BA863A86B002865D105F18800012116F0B5
:20020000B7FB4046494613F05DF95BE00029F8D0404612F04FFD014695F82D00A96318B9E0
:20022000A86B00284ED101E00020A86305F18800012116F09DFB45E0F80A21D24FF0000AB7
:20024000544603E0A86B401EA863A96B91B14046012112F02FFD3068446814F00F04C0F866
:2002600004A0EFD0296BAB6B686B491E2963401E6863EBB905F18800012116F079FB13E0D1
:20028000306844680022202904F00F044260CCBF4FF0200A8A464046514612F00BFDCAF160
:2002A00020008145C8BF81464946404613F00AF9EC77404610F02EFB706A18B1024621468B
:2002C00040469047B80910D3AF6A77B14046394612F060FDA862AD6A3DB996F82000054965
:2002E000095C4046C9190FF037F9BDE8F087C0465C88020068880200F8B50546A869837804
:2003000000242746002B2CD0FE2B2ADC427800784B494C4E00EB022009783288264682421E
:200320000DD031F0010306D115F0D7FB00280CBF8126892616E0022908BF802612E01846E6
:2003400015F074FA50B18268002A04BF4068846804D00120194690470127044604B98326BB
:2003600000E08226384801685EB954B1227BE0790223801810FB03F00C30C3B2502B01DD35
:2003800058E0042301F8016BA869007801F8010BA8694078042B01F8010B42DD181F01F8BF
:2003A000010B207801F8010BA07801F8010B6088001201F8010B207901F8010BA0880012A0
:2003C00001F8010BA07900F00F0001F8010BE07901F8010BE67916B10020864214DC207B04
:2003E0000870267BFEB1491C002086421BDD26694200965D0E702669925B12124A70267BB3
:20040000401CC0B2891CF0E7A6684200965D0E70A668925B12124A70E679401CC0B2891C26
:20042000DBE70020087005F11100A91C48F204020DF032FE1FB114B1204611F01BFBF8BD62
:20044000E5040120E00301202C040120FEB5524C60692589A689E169806D2A4689190831C4
:2004600008F054FD6269916D49199165E2697619B0B212180832127801A90A70444EE169E8
:20048000401C80B20918097A721C401C117081B2E269A18152180832126868460260091DCB
:2004A000A181042115F016F863690090054615F04FFED863284615F0F1F9A3F84000EA206C
:2004C00012F030FF02213548324D017068684069007830B1307810B97078FF2801D0042014
:2004E000E0706769E078397C084338749DF9040016F05EFA87F8460007F17406BE653989C4
:200500009DF904007B6887F84800B7F85C000026401AC0187860B88987F84760800A0AD38E
:200520002868D0F80813384688476769786E10B1B7F8680010B397F8600050B12868D0F862
:200540000C13384688476769F86C10B1B7F85000A0B12968B8310A68107838B1936C2BB1B2
:2005600019463846884767692968B831D1F8A01138468847666115F0F3F9FEBD2868D0F8F3
:20058000541204F11400884766610DF0EDFDFEBD2C1A002014010020B41801206F1B012081
:2005A0002DE9F84F8146D9F80040D9F8047094F82360B4F814A0D4F810B090460D465EB18E
:2005C000A168434815F066FE002818BF6FF001007BD1012084F8260084F8218000262560E8
:2005E0004A463C483C49E66114F005FD3978272016F0A8F951465846062205F081F8002883
:2006000057D13749091F086820F00200086094F82000042806D133484C380068406901461A
:20062000272088472D4F4FF0020B4FF0805AC7F8FCB2DAF8FC0140680146062088470AF5A4
:20064000FE7A38BB584613F029F9B8F1020F4FF0010005D0B8F1040F18BFB8F1060F01D17A
:20066000314600E00421C7F84C11E968C7F85011C7F8546184F82400DAF80000AA68E96828
:20068000036968681C460B46A04748460DF0FCFABDE8F88F4020386080253D6094F82600EB
:2006A00020B10B4816F05CF984F82660C7F8FC6207E094F8260020B1054816F051F984F819
:2006C00026604FF0FF30E061E069BDE8F88FC0464C160120AC19012061D501000444024040
:2006E00088470240FC0100102DE9F04F00214FF00209C41CADF1540D8DF84A1081788DF8E0
:2007000048902046139115F08BFFA41CADF84000204615F085FF0A34804614F8010B149014
:20072000204615F07DFFA41C14F8015B8246102D0BDA6DB12F466E46204615F071FFA41CDE
:200740007F1E26F8020BF7D102E080208DF84A002678102E5DDA5EB1641C37460DF1200B70
:20076000204615F05DFFA41C7F1E2BF8020BF7D19DF84A0000284FD12C4F381D0468AB1936
:2007800013FB09F00F305FFA80FBBBF1500F3EDC15F016FF404538D184F800804FEA2820F5
:2007A000607015F0CBF9A41C0146204616F0A8F804461498207084F801A04FEA2A23A37051
:2007C000E570241D65B16846A41E017804F8021F30F8021B6D1E4FEA21216170F5D1A41CC5
:2007E00026705EB1641E08A8017804F8021F30F8021B761E4FEA21216170F5D1384610A96A
:2008000020225B460DF048FC04E0484602E0102000E080208DF84A001399652001220DF18F
:200820004A0311F0F5FD15B0BDE8F08F280401202DE9FE4F8246DAF8180090F800900021F4
:200840006A469D2005F034FD9DF80000814531DA9DF80000A0EB0900C4B20A2CC8BF0A2415
:20086000E00009F0ADFB5FEA000821D0054624B300262746B34606EB09018B202A4605F0FC
:2008800017FD6879401E0AD0401E06D0401E02D00320687105E00220FBE70120F9E785F864
:2008A00005B07F1E05F1080506F10106E3D104E0002402E04FF0000844469AF811000AF1D8
:2008C000020A8DF801000527CDF804A014FB07F0001DC0B20646401C09F072FB4546071CA0
:2008E00040D0791C0022084602709DF80020BA7087F803903C712CB3491C083D15F8082F06
:2009000001F8032F2A8812124A706A7902F0070201F8022FAA7912F0180F0BD0D3082CBF27
:2009200006230223520928BF43F001030A7842EAC3020A70AA784A706A88641E4FEA222236
:200940008A70DBD10B4D2C1D514648F23202334620600DF101000DF09FFB384611F08AF8BB
:2009600009346C60B8F1000F02D0404611F082F8BDE8FE8F280401202DE9F0470646880F34
:20098000C0F08E8000200EF0FDF8464815F014FD454C40F60A09A4F8009000256580207B37
:2009A00005F00F0120F00F00014321736560607B4FF0010808F00F0720F00F0047EA0001F4
:2009C0003046617306F06EFBD6F808A04A462146D01F574600F1010C00E027467C6834B161
:2009E00023889A4203D0984218BF9C45F5D179607A7B2E4C05F00F0322F00F0213437B738F
:200A0000D4F8983033B1DA681288904223D06046904220D0338FF3B1F56306F13802558091
:200A200096F8440005F00F0320F00F00034386F8443096F8450008F00F0320F00F00034344
:200A400086F845304A60487B05F00F0620F00F0046EA00054D7315F021FB1548A06294F80C
:200A6000310080B91348006801684046884701280FD0787B08F00F0120F00F000143797339
:200A80000D4EA66205E011F035F80028FBD010F051FA504615F090FC5146404614F0DEF884
:200AA000BDE8F08701010E04601A012068F20020855C0000E001001035FE0100F8B53C4DB5
:200AC000002428703B4E85F84A4040F20110308040F60C4009F074FA706028B17068214606
:200AE00040F60C420BF07AF933483449344B364EC161344A03627778426237F0010718D159
:200B0000317D012915D13149314F8162F3780761590802D2406B58B90BE02E4F47632E49ED
:200B2000C1622E4B43612E4AC2602E4B836138468047AC602C48046013F030F8707830F022
:200B400001002FD115F0F0FB28494FF6FE70642721F8080F48800C714C717F1E8C71F7D161
:200B60002349C82748804C704C607F1E01F8084BF8D120490827A1F1CA02508014727F1E4F
:200B800002F10A02F9D12A781E277F1E21F8080BFBD1194901200870104610214FF47A725F
:200BA00015F087FE03F0DCFF14480460F8BDC04650010120DC0A0120E40201203D3802006B
:200BC000C156020029DE0100E4040120ADA40100614B02001951020079D10100B9BF0100BB
:200BE0001D0102007D670100E40A0120C4060020EC09002044020020650F0120000A0120BC
:200C0000F0B5064631684889ADF1440D4008C0F092804A894FF6FE70104048810868036A04
:200C2000C57F5978187800EB0120694611F0DDFAD878997801EB0021ADF80A105A791879EB
:200C400000EB0220ADF80C0098799DF807708DF81200D879002F8DF8130008BF082403D044
:200C600003F10800102405909DF808701FB1181908340690E4B28DF801409DF8057037B181
:200C8000185D641C8DF80500E4B28DF801409DF806C02A480027BCF1000F06D190F82F201B
:200CA00052B1428F8A4206D106E090F82F201AB99DF8022002B90127A7B9BCF1000F05D1A1
:200CC0001B190A932D1B8DF81C500CE090F830001B190E330A9314F0A9FF2D1B281A0E38D8
:200CE0008DF81C000A9B37BB1878042823D10DA800210E220BF072F8BDF80A000A9FADF894
:200D000034007978880924BF01208DF83F0031F07F001CBF01208DF83E00C80934BF069993
:200D200005990DF1360015F0EBFD30798DF840000DA80FF03BFE11B0F0BDC04650010120B3
:200D40002DE9FF4105466E68AF680C4615F0F2FD3178012903D115F06DFF002080E0012105
:200D6000317015F067FF207870706078B07060687060A068B060E068F06020693061207DF8
:200D80003075607D7075A07DB075A069B061207F3077607F4FF0000843467077A07F3363FF
:200DA000C6F82080B0771C4674627463B462B46386F82C4086F82D4086F8A84186F8A941CE
:200DC000786806F0E7FA284606F040FB28460CF00BFD684615F0D0FA3A7B06F16C00B96895
:200DE0000192214A00956B4611F0A2F9684615F003FB396902911D49009506F188006A4603
:200E00000FF096F8B07830B906F1C400214613F0BFF817483061707830B906F58A7021463B
:200E200013F0B6F81348F060684615F0A0FC01948DF8004006F5B2700F4902950A226B46C4
:200E400010F038FDB969FA6906F13C0015F019FA0A4A06F1580004212B4613F0C1FC284626
:200E60000090BDE8FF81C046A501010043E901007F6802002D6802004D120200A9640200F3
:200E80002DE9F84F80460D462868DFF824A1D8F80040D8F804700689D0F804B0E168914631
:200EA000504615F0F7F90028CDF8009018BF6FF0010074D148464FF0000960723A496561BD
:200EC00042464B46C4F804903648A37014F093F83978272015F036FD31465846062204F028
:200EE0000FFCA8B9334E4C3E306840690146272088472E4F4FF0020BC7F8FCB2F06C4068A3
:200F000001460620884750B14020386080263E60504615F025FD4FF0FF30BDE8F88F584663
:200F200012F0BCFCF06C95F82010C26928699047F26CDDF800C095F8200095F82110136872
:200F4000BCF1010F4A4608BF01229847E869C7F85001C7F85491A869C7F85801A96959B131
:200F6000F06C076968684A461346B847F06C806901461148401E8847207A042804D03068A9
:200F80000069014627208847F06C0369E969EA68A8681C460B46A04740460DF0B5F9BDE89F
:200FA000F88FC046AC190120A5E90100044402404C160120FC01001003000080F0B50E4699
:200FC0000746002406F10805ADF1240D28468DF81C4014F070FA18B9384629460CF062FBF9
:200FE000284607A96A460AF07BFE414D01466878A127012818BF022812D19DF81C30BBB9D1
:2010000005A8214608220AF0E9FE05A807A96A460AF066FE01464FF6FF70884204D16878CC
:201020009DF81C5025B907E001208DF81C0068784FF6FF728A4207D1002855D115F02CFB74
:20104000002851D127463AE02A4B9DF810205D782746002A3BD0521E2DD0521E0AD0FB3A22
:2010600008D0921E40D1012812BF0228012086F8260024E08A0002EBC102B169D218383242
:2010800053688B4215D8491C012851601CD002281AD038B9748240F20110B0829DF8125049
:2010A00086F8285006F11E0002A9082214F076FD1AE0A22718E0012806D0022804D040F2EF
:2010C00003107482B0820FE04FF48170F9E705209DF81330708203F07F00B08205B1012464
:2010E00086F8264086F82740384609B0F0BDC046E4040120CCE800202DE9FC4706467568DE
:20110000D6F808802F780FB1AF6B1FB14FF0FF30BDE8FC8729630024EC77171C6C631BD092
:2011200005F13C0915F006FC82466946484610F061FD002820D4504615F07CFD9DF8000045
:20114000296B0870686B296B7F1E00F10100686301F101012963E5D169786A6B286B012919
:20116000A0EB0200286305D1E868296B0346304698476A6B144659E0AF63D8F80010086B32
:2011800040F400700863D8F80010886B40F4FA608863504615F04EFD05F5D47014F04CF987
:2011A000687805F5D47768BB15F0C4FB95F82D1069B1696B59B1A96B49B1AC6315F03AFD08
:2011C00005F5D47014F028F9686BBDE8FC8715F031FD696805F58A76304615F05BF80028BD
:2011E000F2D0AC633046214615F054F80028EBD0384614F011F91022696B286BEA77401A2D
:201200002863E1E715F096FB95F82D1061B1696B51B1A96B41B1AC6315F00CFD05F1880092
:20122000012115F0A5FB01E015F004FD2046BDE8FC8770472DE9F04F05468846ADF1140D8E
:201240001C46D5F808B00E990092DBF80400019108EB0401884238BF6FF003047BD3404E0A
:2012600030684FF0FF3115F015F83E48019F01684FF0000978081CD23846CDF80C908008A9
:2012800027D334B33046DBF800200099066823464244491E521E11F8010F12F8015F05406F
:2012A00085421CBF6FF00604301C52D15B1EF2D10FE034EA010701EA040202D02A480068C6
:2012C000121801EA080128460DF0D6FF002803903CD1DBF800500FF0E1FE27464544DDF81C
:2012E00000A0029002E0BF1BB244AD1997B1082F8CBF08263E1C15F01DFB0490294632465A
:20130000504614F07BF98146049815F093FCB9F1000FE8D0029813F053FBB9F1000F12D1D0
:201320000198C00812D38CB1DBF8000000994044491E401E10F8012F11F8013F9A4202D145
:20134000641EF7D102E04FF0FF3003900448039C006815F005FB204605B0BDE8F08FC046C3
:20136000001B0120081B0120041B01202DE9FE4F0CAF1D468B465FEA02083E78009014BFEF
:201380004FF0804A4FF0005A15F0D4FA0324DFF804910190BBF1FF3F14D1D9F8A8100098C4
:2013A00015F012F858B9D9F8AC10009815F00CF800280CBFD9F89870D9F8AC7008E0D9F86D
:2013C000A87005E000985946002211F0B7F80746002F59D097F8330030F07F0053D04C464C
:2013E000D4F8A800B84219D0D4F8AC00B84215D000982A463346394608F0AAFB002842D068
:2014000094F8240001283CD094F82400042838D0214904F1E00015F0ABFA32E0D4F8A80094
:201420005346002211F0A8F8D4F8AC005346002211F0A2F8B8F1000F14BF1848184813F034
:20144000D7FBB6B1D4F8A80000224FF0807311F093F8D4F8AC0000224FF0807311F08CF8AE
:201460003869C4F8D80094F8DC0040F0010084F8DC0035B1D4F8981000982A46334608F073
:2014800067FB832400E00424019815F0D3FB2046BDE8FE8F68F20020020000400100020474
:2014A000010001042DE9F04FADF1140D02921D460191DDF83CB00E9C009015F03BFA464AC4
:2014C0006FF001084FF00109002392F840A2039009FA03F616EA0A0F6FD0B5F1FF3F18BF2A
:2014E000AB426AD1D8B214F0F7FD002865D0877A002F62D192F84012B14382F840124F4651
:201500008772009D437292F842120560491C82F84212019E06722E4F4760017A07460129DD
:201520001ED0022924D140F20361018290F90930C17C5B1D21F00F0103F00F030B43C37462
:201540006379817C63F3C7018174C17CA37963F34611C174C17CE37963F30411C17407E044
:201560000A20388297F90900401DB874A0687861BBF1000F08BF002012D09BF801009BF8D9
:20158000001097F90960134C4FF6FC75800040EA4110711D40EA012005EA000144EA01003A
:2015A000B861029800B17860506808B9386850600CF0E4F897F9098002E05B1C032B87D354
:2015C000039815F037FB404605B0BDE8F08FC046734A01000100040668F200202DE9F0414A
:2015E00004464A480078ADF1280D18B9E17A15F0F5F808B9012085E06846002124220AF050
:20160000EDFB208B00F0010100F00C00084301D1207A08B9B62075E00F288DF808004FF0A3
:20162000000613D002284FF003050DD0032806D0012812D126884FF6FF700F2508E068463A
:20164000214615F05DF908E0208804E020880B2502218DF80810ADF8000005F00C07B7F167
:201660000C080CBF03200120678A801DC1B27818C0B28DF81F0008F0A3FC071C40D0089737
:20168000B81CB8F1000F00F8015B04D100F8016B311200F8011BA17B00F8011BE189091225
:2016A00000F8011B217C00F8011B218A091200F8011B628A616914F071FA14F07BFF0326BF
:2016C0003A46810041F0030102F8011B80111070A0898DF80C60A37EADF80A0015F00C0FA3
:2016E0008DF80D300CBF012000200021ADF80E00684607F0A9F80446384610F0BBF900E0A6
:201700001024E0B20AB0BDE8F081C046C60A01202DE9F84306464FF6FC751C46174688465C
:20172000B54200F0848000210FF028FCDFF804910646B9F83A00B04201D1E00977D3214679
:2017400030460BF04BF9C0B9A81C00210BF046F998B914F0180F0DD0374B0020997911F02E
:20176000180F03D1642805DA184606E0401C08336428F3DB0220BDE8F883AD1C06804545B3
:2017800018BFA0F802808471610824BF44F004048471012F0CD04179012913D0817911F018
:2017A000180F0CBF99F83710FF210171477109E001214171817911F0180F0CBF99F8381092
:2017C000FF210171012F32D1B9F8481040460FF0EBFF60BB194C1A4F00204101A1EB800174
:2017E000C919B1F87C6307F2AC52002364215588AE4205D0491E02F1080203F10103F6D11B
:20180000642B04D0401C1C341428E6DB0FE0204600211C220AF0E2FAA4F80080B9F848001D
:201820006081AA27A77401266674062525740020BDE8F88350010120CC0600209C040020B2
:20184000200100202DE9F0479646464A88461E23002401460125204697782FB15B1E02F12D
:20186000080204F10104F7D11E2C79D03E4C3F4F814633264FF6FF7C82F8069037F824AFFF
:20188000D04510D0638F53450DD03B7933F0040A06D0012B07D14B899C4508BF284302E064
:2018A00093795B1C9371761E4FEA4505E6D1304D1426ACF1010C35F81C3F98450DD09C454F
:2018C0000BD0B4F848306F89BB4206D16F7C27B1AF7C17B193795B1C9371761EEBD19779A0
:2018E000082F01DC17B909E0082393718B7C012B04D094F826305B1C137101E082F8049019
:2019000094F82B30937094F82570D7708E891680CD7C82F805E0D571B8B116491E2201F1E0
:201920003B030D46494613F8017F37B1BE4504D0521E01F10101F6D107E01E2905DA83F88A
:2019400000E005EB8105C5F8AC002078402110F071F820B920784021642214F0AAFF012040
:20196000BDE8F08744020020500101200810002080040020200100202DE9F84F8346DBF85D
:201980001800057800216A46A3200EF06DFEBDF800004FF00009854224DABDF80000401BE3
:2019A00084B2042C01DA0CB91DE00324E00000EB041008F005FB5FEA00090FD007464FF069
:2019C00000088CB146467119A2203A460EF04CFE761C1837F6B2B442F5DC05E04FF0B508F1
:2019E000002401E04C46C8469BF81100E1B215278DF8020011FB07F0001DC0B2401C08F062
:201A0000DFFA4E460BF1020B071C45D0781C82468AF800809DF80010E3B2B970FD700425C1
:201A20003C7143B3001DE4B2314614F069FF317A00F8011BB17A00F8011B7189091200F862
:201A4000011B317D00F8011B317D032906D0317B00F8011BB1890E35091205E006F10C01B7
:201A600014F04EFFB17D1535641EEDB200F8011B06F11806D8D10C4E2B460DF10200594640
:201A800048F23302341DC4F800A00CF005FB38460FF0F0FF09347460B9F1000F02D0484698
:201AA0000FF0E8FFBDE8F88F2804012030B54B4C0546E079ADF12C0D012840F0878014F06C
:201AC00023FC002840F08280688800287ED1404905A8122207F01AFA20784FF480510DF008
:201AE00021F8A96911F8010B0C784A788DF8140004EB0220ADF816009DF81400C8BB881C2B
:201B00009DF8181010F8012B10F8015B10F8014B01F0E00102F01F020A438DF8182010F825
:201B2000013B8DF8195010F8012B10F8015B8DF81A4010F8014B8DF81B3010F8013B8DF817
:201B40001C2042788DF81D5005788DF81E4005EB02218DF81F30841CADF8201014F8010BC9
:201B60008DF8220014F8013B8DF8233025788DF82450BDF82000B0F5285F23D2154800684D
:201B80000DF126016A460AF0ABF80446C82C11DA9DF8100010B1FD208DF8100021461422F5
:201BA0006B46042011F074FC0B4AA000012100EBC4001154002014F07BFD01200146F5F7C4
:201BC000DBFC03E00120022111F044FB0BB030BDA6860200EC0601200DE900206806012039
:201BE0002DE9F84FD0F8E8200023083A002AC8BF0123D0F8C0C0D0F8D020E346DBF8004042
:201C000094420CD8DBF81470002FBC4678D001228CF81020D0F8C0B04FF0000E00E0964622
:201C2000DCF80020A2EB0E02B2F5806F88BF4FF48062D0F8D8702FB9C0F8D820D1F81C8004
:201C40008E6904E0C0F8DC20D1F824800E6ADCF804402CB92B4C9F00E55900F1F6040AE0EA
:201C6000294D9F00ED5903F1010A02FA03F90EFB0A444C44641EB56034600C6804F1080986
:201C8000C6F80490B56843F6F07A1401103C0AEA04042543B560DCF8086026B9194BDD59A3
:201CA00000F1F40308E0194DED595F1C02FA03F30EFB07669B195B1EC8F80850C8F804308C
:201CC000C8F80090D8F80830E34544EA0304C8F8084004D1D0F8D0309B18C0F8D03090F8B7
:201CE000FE706FB90B685A6A42F003025A62D0F8CC004F6943680A69196847EA020088621C
:201D0000BDE8F88F24880200348802002C8802002DE9F04306467568B7680C46ADF1140DD3
:201D200014F008FE95F8FD1021B96169102901D8042903D214F07EFF00206FE04FF001090E
:201D400085F8FD9014F076FF2069C5F8E4006069C5F8E800207B85F8F900207885F8F8004A
:201D60000020616885F8FC008046C5F8C080C5F8C480C5F8C8802B4AC5F8EC10217E12F861
:201D8000211085F8FA10F989A5F8F610237B002B0CBF1021494685F8FE00C5F8F010387B27
:201DA00005F0F8FA30460DF095FA97F83B0085F8FB00304609F090FA684614F0DDFA787985
:201DC00000966B463979184A0190284610F0B0F9684614F011FBB96802911449009605F1A5
:201DE00030006A460EF0A4F80EF0BAFD014633460F4AC5F8CC1005F11C00042112F0F0FCDD
:201E000095F8F80030B905F16C00414612F0C0F8084800E0A068C5F8BC00304605B0BDE830
:201E2000F083C046E8850200F9C300003118020035670200776802002DE9F04FADF1140D20
:201E400002A913F049FA5FEA000940F08380434F029C3E69218856B1B61F0322002036F83D
:201E6000063F994205D0521E00F10100F7D1C82601E080460026182008F0A2F8051C0ED0BF
:201E80000021182209F0AAFF608818212A4614F04BFC4FF6FF70608028460FF0EBFD4FF63B
:201EA000FE7A4FF0000BA4F800A0002E84F804B050D13869444668B3142008F081F85FEA71
:201EC000000827D04C205946022203AB14F068F902255E463869B44207D0A9B24C20062299
:201EE0006B4614F05DF9694603E0610001EB84010918A8B20622404413F050FE761CAD1D9F
:201F0000032EE7DB4C201421424614F00DFC40460FF0B0FD4C205946022203AB14F040F94C
:201F2000C0B93F695FB1610001EB8401BDF80C007A5A5646964204D138B1401E03E0BDF8E1
:201F40000C00401C80B2ADF80C004C20022103AA14F0EAFB484605B0BDE8F08FCCE80020D6
:201F6000F0B5ADF13C0D11F0A5FF454E96F84A00082807D0332086F8290086F827000127F7
:201F80007765B76568460021242209F027FF3D4D2878012804D0012000278DF80A0002E035
:201FA00000278DF80A700F2446208DF837400DF13701B4700FF0FEFE6D1E8DF82470A8794C
:201FC0008DF8250014F0F6FA8DF826008DF827708DF8287096F85C008DF82A700F28A8BFD8
:201FE000201C06F15D018DF829000DF12B0014F087FC0DF13300FF21032209F0EFFE96F808
:2020000096008DF8360009A80CF0D6FB06F1140145200FF0CFFE08F0CBFE8DF80C708DF86D
:20202000207096F850008DF8157096F851508DF80800B6F848308DF8095096F85320ADF8C2
:20204000043096F83C408DF80B2006F13A018DF8064053200FF0AEFE06F13E014B200FF0D7
:20206000A9FE96F82B203078642111FB02F2082114F022FC684605F0D1F80FB0F0BDC0468A
:2020800050010120E5040120FEB505462B7A33F001000BD0288804460FF08CFC30B9032B8A
:2020A00006D1284601A911F009FB18B90220FEBDADF80440688A443007F082FF071C08BFCD
:2020C00010206ED00021442209F088FEA87A0DF1060112F05DFF9DF8060087F83A009DF81E
:2020E0000700012187F83900384612F061FA242207F11000294613F051FD07F1440038643E
:20210000688AB88769696A8A386C13F047FDBDF804002449B8808878F8718878401C8870C2
:2021200014F08CFD044614F027FA97F839604FF47A71FF236043B0FBF1F0388003FA06F051
:2021400087F83700002487F83600288B8DF80040400834BF201C01208DF80100287A8DF833
:20216000020068460EF052FF801EC1B2BE8FBD8F87F8341097F8342095FBF1F0C0B2387283
:2021800096FBF2F15143761A1CBF401C3872064E388D40F008003885307801210CF058FF9B
:2021A0002046FEBDE0060120800A0120F0B50646B16948780D7805EB002543480088ADF136
:2021C000140DA84271D1414C708802A90BF06AFAB71C241D01281DD19DF80F00042807D150
:2021E0009DF80E00CF2803D19DF80D008C280BD09DF80F0054280DD19DF80E00EF2809D1AE
:202200009DF80D00442805D15F201123E0700020237102E00020E07020712A490A6802F861
:20222000010B02F8015B2B1202F8013B2078C11001F0020300F0070001F00101194340EAFA
:20224000C10002F8010B607800F0F80100F00700084302F8010BA07802F8010BE07802F83E
:20226000010B207902F8010B607902F8010BA07902F8010BE07902F8010B207A02F8010BB6
:202280002089001202F8010BA07A02F8010BE07A02F8010B207B10233946107048F20202F2
:2022A00006F111000BF0F8FE0AE048F202000090307C0190707CB11C80222B4611F0C0FEA7
:2022C00005B0F0BD2C040120E00301204C1A0120F8B5474C054620684030816F0F780023A3
:2022E000B7B395F8987097B92521297501680968C98AC90939BFD0F8940090F82500D0F8E3
:20230000940090F84E0085F86A00801C0EE01521297501680968C98AC90939BFD0F89400BB
:2023200090F82500D0F8940090F84E0085F86A00042085F8693005F1900185F86B000A68BC
:2023400005F170073A604E687E600889388101E001202875B5F89E0095F8A07095F82C2038
:20236000E88295F8A160EF760F2A2E770CD02068B5F8A870D0F8046305F12C011A4607B987
:2023800001222846B047034673B995F83C00FF2801D1A86D38B12068D0F8FC2205F13C01DF
:2023A0002846904703460BB11F461FE020680027D0F87463009795F89C10B5F89A3005F1E4
:2023C00090022846B047071C10D1216801F5807108682A89C0899042A8BFD1F8781103DABE
:2023E000E5206870D1F86C1128468847F8B2F8BD140100202DE9FF47444D0C460646904688
:20240000600831D230460EF0B9FD698F814205D03046022122460BF002FC08B9002072E06A
:2024200030464FF6FE7102222346FFF771F9002868D124F02004E0091ED2304602A912F0F0
:20244000E6FA70B9B5F84810304611F02DFF071C12D0B81C13F02FF870B1B91C02A814F024
:202460004FFA44F0200407E04FF6FC76A00834BF44F0080444F0100425486B8F90F800907B
:20248000012509F101010022C9B20170491E00951846C9B20AF016FBA0BB4FEA641AA00971
:2024A00034BF06200E208DF8050001A812F0D4FD071C25D0BD7713F041FB78623869057054
:2024C00004F07804447080F802903112C670002301715FEA5A01437103D3801D02A914F046
:2024E0000FFA4FF6FC70B8F1000F788004D0B8F10F0FB8BF87F81A803846F7F7A9FE02E052
:20250000102000E0C7200090BDE8FF8750010120640F01202DE9F041454C05462078002820
:2025200000F08280B4F9B600B4F9B41088421DD004F1980128460E4611F035FC70B9D4F8A7
:20254000A810284613F040FF28B906F10801284611F029FC01E0D4F8A80038B1B0F9301077
:202560000A224FF0E043284603F0A6F914F0E2F9804604F1B8000168A94219BF0026466083
:20258000002606602078401EC0B2207000283BD194F82400656002280ED1082010F0A4FD3C
:2025A000404614F047FB05F150004FF0FF3113F071FE14F0BFF9804604F1E00014F0D2F902
:2025C00004F1600014F0B4F904F58E7014F0CAF904F17C0014F0ACF904F5AC7014F09AF971
:2025E00004F5CE7014F096F9E16911B104F14800884704F1340012F0BFFD0C48007801281D
:2026000002D10E2004F02EFC606805F15007854208BF6660404614F00DFB384614F09EF987
:2026200005F1B80014F076F9BDE8F0818687020068F200202DE9F843434D444C3E4EDFF806
:20264000FC80DFF800910746012F44D139480068006801460120884701283CD096F8380180
:20266000002838D108342068C0F38140C8B940460068B0B154F8080C000834BF4FF48050B3
:202680004FF440502E4908600A2014F02DF94846006901460120884706F1940014F042F93C
:2026A00001E012F093FA0121206886F83811C0F3814010B94046006848B913F0C3FF8009BF
:2026C00005D28020A860286840F080002860032011F0E4F82BE057BB0BF03EFBA068C0F3A7
:2026E0008140A8B94046006890B106F1940014F01BF92068000834BF4FF482514FF4415178
:20270000134A48461160006910B101460020884796F8380158B12868802720F080002860DE
:202720000320AF6011F0A2F8002086F838010020BDE8F883E0010010501800204086020074
:20274000A8A00C403086020090220840AC4F005028A10C402DE9F04105460024ADF1500D22
:2027600028888DF84C400FF025F9002879D13E480078A0B9A87804280FD113F0C5FD60B9A8
:20278000686813A901AA09F0ABFA80469DF84C0000280CBFAD26261C02E0B62600E0B3263E
:2027A0001E2012F0D3FB074666BB03209DF816108DF84D000FAA03A80CF030FD0DF14D0015
:2027C00008210FAA0BAB0CF02DFBA8680BA9102212F0B2FCA8B106A80090414622461423DA
:2027E000042010F013F89DF82B0030F07F0003D00DF12B0011F092FA022006AB8DF8280042
:2028000012E0AD269DF84C00012812D102949DF81700019430F07F0003D101208DF8150001
:20282000FF248DF8144001AB04204146142210F02FFEB7B10920387028887880A8787E77EC
:20284000387169680822781D13F0A8F9A96807F10D00102213F0A2F90448007839460DF075
:20286000C1FF14B0BDE8F081E5040120CB03012044492DE9F04105464C310868002877D149
:202880003E4CA7683E1C0BD068883988884203D12979BA78914218D03E46BF69002FF4D1EC
:2028A0001C2007F08DFBD4F80880071C63D000211C2209F093FA4FF6FE70FF233881B8F197
:2028C000000FFB720CBFA760B761687AB871287A78712879B87068883880287B3875287A99
:2028E000012806D107F10C00FF21082209F076FA05E007F10C0005F10D0114F001F8A97A14
:20290000062938DD6879012803D013F0CBFE002831D0B87A00231E46884202DAEA7A102AA4
:2029200005DB884204D1F87AE97A884200DD01231348007830F0010203D0022808BFEE7957
:2029400000E0AE791EB9E08F2988884206D12BB128883881A87AB872E87AF872E87908B161
:2029600001203871A87908B10120F870BDE8F081096828468847BDE8F081C04650010120D8
:20298000E5040120C40301202DE9F04F002788460646ADF1140D039713F0CCFF3A4D04906D
:2029A0006868384CC36C2069052103AA9847684613F06AFBDFF8E490CDF80880DFF8D0B054
:2029C000DFF8D4A0DFF8CC80009629F0010926F00106B1451BD02D4820F00100B0420ED17B
:2029E0009BF900106B68206911F1020F24D059469A6B91F90010904781281BD015E04046AC
:202A00000068D0F84C0580476FF001071AE09AF900106B68206911F1020F0DD051469A6B82
:202A200091F900109047812804D040460068D0F84C0580476B682069DB6A69463A4698472B
:202A4000071C04D540460068D0F84C058047B14507D00E4820F00100B04204BF58460770AE
:202A600001E05046077001206F6803902069FB6C052103AA9847049814F0DCF805B0BDE86D
:202A8000F08FC046A4060120D4050120B51E0200B10A012014010020B00A0120E9970100AA
:202AA0002DE9F0413C4F3B4C3C4D38696168ADF1300D58B921B92868D0F84C0580476168CB
:202AC000096A07F11C0088473548B8636069016929B12868D0F8D40090F853008847286895
:202AE000D0F8D40090F942000CF0DCF8B0F1FF3F0A9008D00290000834BFBDF808004FF6BF
:202B0000FF7028490880DFF8A0800026A8F87E60C8F8806098F8890020F00F0040F00100A9
:202B200088F8890098F88810012363F3C71188F888102868D0F8C403804730B91B49102097
:202B40006B680870596814230B703869454650B9606804687968164805F17C0207F11C0384
:202B6000A047386113E0304610F02AFC6068416E02A88847334660680593066D08228DE86B
:202B80000C0038697C35294602AAB047A5600CB0BDE8F081D4050120A406012014010020F4
:202BA00054F10080E600012058000120D8000020680F0120BCB505460020E860012428616E
:202BC000A978287501F0030348081DD2C80801F00C0201D3042A04D1022B01D1480900D239
:202BE00002240C2A04BFA41CE4B2022B01D148090AD2241D32F00807E4B203D00C2A18BF4C
:202C0000042A01D1641CE4B231F07F070BD0E878641C10F0030FE4B205D0641C8808E4B219
:202C200024BF641CE4B213F0CBFC2A88641CE4B290420BD0880909D32148016828468847E0
:202C4000286918B9A87800F0DF00A870287D002834D150202F6969792B798DF800008DF8A1
:202C600002101819C0B227B17A7F397F89180918C8B28DF8010068460FF098FAC8B12988EB
:202C8000012747764180A97880F83810E97880F839102979036980F842101919416480F864
:202CA00048402F691FB13A7F416C89184164E860BCBD284613F056FD10202875BCBDC046A7
:202CC000B80801202DE9F0410F463E4C3E4904EBC00409782668D4F80480ADF1280D8142BE
:202CE0006BDD07B9394F96F85200002865D198F80100022826D1022086F852000EF0DEFB8B
:202D0000684613F0A3F900258DF800508DF808503968039598F80000019169460EF0CAFEBF
:202D200070607068002848D013F044FDF87998B13A68B979706864235143B1FBF3F113F053
:202D400034FD09E002F06EF8012198F8000086F85210002586F8540006A813F008FD8DF83D
:202D6000185008941A480795294606AA0EF0C2FDB060B068E8B138683060B87986F8530082
:202D8000F87988B1401E09D0401E10D1B8884FF6FF72411020460CF0FAFE08E096F8531099
:202DA000204610F065F802E020460FF0F5FA204604E0706808B113F0F3FC00200AB0BDE8CE
:202DC000F081C046F88602006A83020004880200E3220200F0B50446A178606840182178B7
:202DE000ADF1440D0546F9B9217F0D2914BF00230123227C617841EAC20141EA431100F81B
:202E0000011BA16912F0BEFE0646012B04D104F1080113F075FD0836207C04F1080101280D
:202E200004BFA07D307005E0297860780843287004F10801A7692E7804A813F061FD06A862
:202E4000394612F09FFE0670A078237F8DF80000E7788DF8013066788DF80270608A8DF846
:202E6000036060B9A18A40F201128A4207D194F8281004F11E000CAA0CF0D0F903E0A18A62
:202E80000CAA09F093FE0CA8FF270390207C8DF84070022803D003280CD1022000E000208D
:202EA0008DF8400008210CAA08AB10A80BF0BAFF08A8039020786368694604AA00F028FA3A
:202EC000044628780021102200F0F800287008A808F084FF0CA80021102208F07FFF204627
:202EE00011B0F0BD70B53248304E4FF08055B067D5F8D8012F4C036801210A46ADF1280D4B
:202F000020469847D5F8D801426801212046904713F056F8284906F124040822204612F04A
:202F20003DFE26490822204611F04CFF20B924492046082212F032FE2248A060224DE560E5
:202F4000224B2361224A62612249A161224DE561224B2362224A62622249A16200252563F2
:202F60006563E562204BA363204AE26320492164F06A10B1F16A2846884706F02BFA0DF069
:202F8000E5FB684629462422082313F02BFE06F108048DF8185029466A46204613F01EFE03
:202FA000746013F017FE28460AB070BDE8010120E368020000400340C87F0500EC87020035
:202FC000F0120050517B0100CD000200B9AE0100DD90010045A60100F1BA0100FD7B01001C
:202FE0000DC8010019F70100555B020009D10100C1DD01002DE9F04104460D461646104628
:203000000021342208F0EAFE082D5CDB61782078357000EB012031460FF0E7F800280CBF83
:2030200001270027E178A078A2792379657900EB0120B274E179708103EB0520F174F579D8
:20304000B081002D08BF082103D004F1080010217061357A084625B160180831B061C9B240
:203060000846002386F82030757973622DB17070605C491C7071C9B20846757FFDB1481CBF
:20308000C2B2605C7270511C86F82000C9B27170A25C86F821208242A8BF737710DA0C28C7
:2030A000C8BF0C20DFF85080450009192A46404612F074FD7078C6F824804019C1B27070F0
:2030C0003078814202DD0020BDE8F081B379401A6418C5B2002B08BFB46209D007480E3D7C
:2030E0000E34EDB2B4620078357712F09FFD2D1A35773846BDE8F081440100208001012089
:20310000B0B5C16891F838300A6903F0030535F0020702F8013B40D1D90803F00C0401D395
:20312000042C08D1022D01D1590904D2C16891F83B1002F8011B0C2C09D1C16891F83C102A
:2031400002F8011BC168898F091202F8011B022D01D1590921D2C16891F83E1002F8011B7B
:20316000C168C98F091202F8011BC16891F8401002F8011BC168B1F8401034F008074FEAF7
:20318000212102F8011B03D00C2C18BF042C04D1C16891F83A1002F8011BC46894F83910DD
:2031A00003F0020701F003010F430DD1618D090A0AD2144DA97884F84910A97802F8011B83
:2031C000A978491CA97003E094F8491002F8011B33F07F0714D0C16891F839101170C16840
:2031E00091F8394014F0030F0AD091F84B1002F8011F990804D3C06890F84C0002F8010F61
:20320000B0BDC046E00601202DE9F04307464FF6FE754FF00008ADF11C0D391DBD8101A89B
:203220008DF8008013F056F968460AF061FD07F10409444601280BD1BDF80C00BDF8021015
:203240007E88B8818E4218BF6E4602D1012441E046468DF80E807888ADF810000DF10E005B
:2032600008F0F6FD012808BF0DF10E043046012618BB74B97888854206D1484612F01BF984
:20328000012818BF404602D138460CF0EDF906461FE0A089B881201D12F00DF9012807D083
:2032A000484612F008F9012813D103213C460DE038460CF0D9F9064606E080893146B881A6
:2032C00038460DF03BFD24B16580022120460DF035FD34463E78A6B1384611F0B9F90128E8
:2032E0000FD10A48BD89001D0168AA0002EBC502501889180A78164203D116430E7013F0E1
:203300002EF9204607B0BDE8F083C046DC0A01202DE9F04F0C46834661782078D4F80C90FB
:203320004018C6B2E0781D469246ADF13C0D0428A8BFA77803DAA07800278019C6B211F063
:2033400069FC0E90E07812F071FC0D9049461022F01900EB050809A813F0CAF84FF0000986
:203360000146BBF1000F25D1E078042847DB002946D1684613F05FFA09A8069621780797E1
:20338000637800900D240D9E01951A46CDF810A0204FCDF8148058188DF8204052188DF86F
:2033A000216040195219039069463868029213F06EFA23E0E078042821DB09BB684613F0EF
:2033C0003AFA09A8069621780797637800900D240D9E01951A46CDF810A00E4FCDF81480CD
:2033E00058188DF8204052188DF8216040195219039069463868029212F05FFB014609B171
:203400005FFA81F90E9812F090FD48460FB0BDE8F08FC0460CDC00202DE9F04780463D498C
:20342000D8F80460C86CD1F808A07F2500220124A946ADF1200DB0438446C86404FA02F035
:203440001CEA000F10D05FEA0A074FF0000007D0BB789A4204BF401CC0B2BF69002FF7D148
:203460008542C4BF051C9146521C1B2AE6DB002E0D4637D1284C5FEA0A0726D02168B5F813
:2034800048004FF6FF72254B3E88B0421AD1BE78B14517D103F130063688B24208D113F04F
:2034A0001DFAA5F848003E88B0420ED057460AE0002485F84A4009B1C4208847204611F0F4
:2034C000F3F924E0BF69002FDED185F83C90FEF747FDE0B10020216885F84A00B9B1C42025
:2034E000884714E0EE64684600211C2208F076FC8DF8044000268DF80760D8F80400009001
:2035000095F852708DF80570684608F009FE08B0BDE8F087500101200C0A0120E40401202F
:20352000FEB53F4C074694F84A00032803D0012818BF092870D13B4D7878384E69780028B3
:2035400050D17888B91C608753200EF033FC94F84A00092801D011F0F7F90127422002A9F0
:203560008DF808700EF026FC0420694684F84A004A2011F085F904F14000694613F0C0F90C
:2035800030780B2805D0B4F84800002107F020FE01E006203070687830F0010008D1E08F61
:2035A0004FF6FE71814203D06946002200F0ACFD94F83200000934BF0020381C02A98DF8F9
:2035C000080052200EF0F6FB6878022822D194F83200000934BF381C4FF400403946FCF782
:2035E000DDF917E002290CD130780B2804BF0A2030700020E87020784FF480410BF092FAF3
:203600007878B4F848200146104607F0E1FD002084F84A0011F0F0FEFEBDC046C4030120B6
:2036200050010120E40401202DE9F04391460A68D9F800401678804600271D463846ADF172
:20364000140D242E02F101020A6058D11678521C4C2E0A600ED1AA68E41C24F00304241D41
:2036600054F8040C414613F0B1FA2968EF600127091A2960462E1AD1E41C24F00304241D4A
:2036800054F8040CE41C029024F00304241D54F8040C002741460390AA68ADF8047001A86F
:2036A00013F090FA2968EF600127091A2960532E25D1E41C24F00304241D54F8040CE86151
:2036C000C9F80040288B0090A968EA69D8F800004B4613F073FAD8F80040002744B1A96834
:2036E0008142D8BF481ED8F800100918C8F80010D9F800402968EF600127091A2960662EE0
:203700000BD1298B012904D0E41D24F00704083403E0E41C24F00304241D1FB9E9690E70D8
:203720000127EF60C9F8004005B0BDE8F08370472DE9F04105463E48401C0078ADF1280DCE
:2037400030F0010169D1374C04F13A0109880026A94228D0284613F076F8071C59D03879E4
:20376000012818BF022854D18DF818607888ADF8240006A80CF05AFC00284AD038882849C1
:2037800008800DF10B0007A913F0BAF812F024FE8DF81660ADF8140039790222684606F0E1
:2037A00083FBFE6039E0002D33D030F001004FF001062ED10CF068FBADF82600BDF8260079
:2037C0000DF12601608753200EF0F4FA1648BDF8264007680EF0AEFA1448007810210BF0F0
:2037E00037FCA7B14FF0D6087868007860B1042011F0ACFB011C07D081F800804C80786853
:20380000406800780CF0EEFF3F68002FECD10CF04DFD16B9284611F0ABF80AB0BDE8F08115
:20382000EA02012050010120C00A0120CB030120E40401203F482DE9F04F001FADF1140D6C
:2038400000F1A80100F1980B8046029100F1AC0103914FF4804012F0EFFBE8B14FF0045094
:20386000D0F89813D8F8046090F88503C3F38857C1F31501C0F38002C1F31501B805014332
:20388000B06841EAC2716A4602F040FCD8F804008168012011F0E2F9002702260DF10409C0
:2038A000234D049759F8044F236883B32068806912F0C2FB82462068002352460EF05CFE05
:2038C0001AF00A0F08D1BAF1000F20D0206847F48047C8F8B0001AE020681449AB6880696D
:2038E000014023EA0100A8602068C1692A6822EA010028602168102011F0B0F921680BF1B0
:20390000080011F097F8049847F002072060761EC8D127B108F1E000394613F029F804F03E
:20392000B9FCF9F74BF805B0BDE8F08FFDBFFFFF0C1004406CF200202DE9F8430446A06A89
:203940000D464778C178807800EB0129207F042866D136480378DFF8DC80354901263846BE
:20396000022829D9C01E072846D90838012819D9801E02D0401E3FD03DE033F001033BD167
:20398000414691F83200800836D391F84A00082802D14846FFF7CCFE48460CF077FDC52845
:2039A0002AD122E033F0010026D108460078800822D30DF0A5FD1FE033F001001CD10846AF
:2039C0000078800818D34846002109F007F870B1817911F0180F0AD0A18900910288438828
:2039E0006189104600220CF0C1FB002604E0484612F090FA00E00025608939464A4610F08C
:203A00006DFD60890DF0D6FF50B1A07C022807DBA18940463A300088884201D0012E02D01A
:203A20000020BDE8F8832846BDE8F883E504012082010120500101202DE9F04FDFF8E4A0E8
:203A4000DFF8E88000244FF001096FF001064FF6FF7B2546ADF1240D01A80090294622464B
:203A6000102303200EF0D2FE00284BD1BDF804109DF80970A80000EB45102AF80010504459
:203A800047719DF80A3083719DF80820027180F809900482BDF80610C4729DF80B70418012
:203AA0000623C771049A0372AA278772B2F1FF3FC46015D1037983B11B4A1778032B0CDA25
:203AC0002FB958F82720C26158F8272009E058F827309A01A2EB830202E0C661866103E09D
:203AE000C261826180F820408B450BD08DF81490ADF8201005A80CF099FA18B1BDF8040081
:203B000010F036FF6D1C332DA6DB2046042110F0C7FD3328A4BF0648047007F049F909B045
:203B2000BDE8F08F2C100020E804012098800200FD0901202DE9F8433A4C364D8146241D55
:203B400054F8040C800807D254F8080C05F14D01000C40F0F000087033484FF001214FF045
:203B600080531838DFF8A880C0F804140088D3F8F0012668016803F5F87730468847B00EAE
:203B800003D2700E24BF02202870386842683146484690470FF0CAFE38B12068810C2CBF5F
:203BA000002040F307200EF0D9FB2048BC300068C0F3053188F80010410A39BF402185F863
:203BC00023104021E974800900F0380040F46050A8F85C0038688168304688470E490F4AE5
:203BE0000AE0105C9478131D844299BF184410F8010C18444078086008684B689842FCD15E
:203C00000228EED1064901200860BDE8F883C0460EB00C400962084000600C40DC870200EF
:203C200094046042B04F005018A00C4050130050394AF8B52120742112F070FD0A2814BFCA
:203C4000002501250C2006F0BBF9071C14D0FF210C2208F0C3F8314E002407E02146012029
:203C60000C223B460BF0E4FE641CA4B23088A042F4DC38460DF0FEFE294E707830F0010081
:203C800015D1102006F09CF9071C10D0FF21102208F0A4F800240320214610223B460BF03E
:203CA000C7FE641C332CF6DB38460DF0E3FE1D48006820B180470A2808BF45F008050FF094
:203CC0000DF90A2808BF45F01005142006F078F9071C1CD00021142208F080F84C20142189
:203CE0003A4612F01BFD0446092C04D14C2014213A4612F019FD38460DF0BCFE06F1480227
:203D00007120082112F00AFD04430A2C01D145F020052846F8BDC04674010120DC0A012071
:203D2000E4040120300901202DE9F0413A4D04462868ADF1200D18B90FF0BCF9286840B3A5
:203D400030490978A14224DD4FF0FF3112F0A2FA2D490C2014FB00146768A66838780128FD
:203D60002ED0B268511EC843B86028683368844619420BD17068824208D8B96801408142CC
:203D800004D1706930BB308B042804DB604612F0E7FD002431E0DFF8748058F82030A3B93C
:203DA000684612F0A3F900208DF80C00F1698DF80000307E049169460DF03CFF031C01D10C
:203DC000002417E0308B48F82030114A815C491C815400E003687B601048318C0D4B016017
:203DE0007A681A60204611F087F90120387020460FF04AFA286812F0B3FD204608B0BDE809
:203E0000F081C0465C830200A0850200B01A0120401B01200C1B0120141B0120101B0120D8
:203E20002DE9F8431D463B4B089C1B68C3F340689B0E15D20388A3F6020343B141F21E06BF
:203E40009B1B04D000F11A030B60C06903E000F112030B604069106000202860206056E06B
:203E60000388A3F60203F3B141F21E069B1B17D041F6E6769B1B05D0876AC36A90F8246039
:203E8000BC4603E0D0F820C0436A002600F11A070F60C1691160C5F800C02360007E0DE03B
:203EA000466A836A01E08669C36900F112070F60416911602E602360C67B007C00F0070709
:203EC000286888B140F203714FF6FF72052310F04BFC8146B9F1050F06DA3046394609F0FB
:203EE000DBF8296841F82900206880B140F203714FF6FF72052310F037FC0546052D06DA2F
:203F00003046FF2109F0C8F8216841F825004046BDE8F88394120050F0B5014688890425A9
:203F2000ADF1240DADF8140000248DF81F504A888DF81E40354EADF81C20081D897B069009
:203F4000022923D10DF121016A4607F0C9FE07469DF82100012856D19DF81000022852D16F
:203F600068462146142207F039FFFF20BB008DF81000142203EBC700345031184C606B4643
:203F80004C72284639460FF083FA3CE051B3032925D008A96A4607F0A3FE01469DF82000C4
:203FA00001281AD19DF81000022816D1FF209DF812708DF810008A000194781C00946B4674
:203FC00000F00F008DF8120002EBC100345082195460284614220FF05BFA012408E0102095
:203FE000214601E0082001218DF81F008DF81E1005A800F04FFC30B9012C04D1BDF81C0034
:20400000069906F0AFF809B0F0BDC04604E9002038B505461446480817D2880872D31C200F
:20402000002112F0A1F91D20002112F09DF91E20002112F099F91C20002110F081FB0021E0
:204040001D2010F07DFB002159E01C20002112F08BF91D20002112F087F91E20002112F02D
:2040600083F9284606F032FB21460090C20F0888A0F6020068B141F21E03C01A09D041F6EC
:20408000E773C01A09D191F8240010F07F0F04D019E0C87B10F07F0F15D1012A0DD01C200F
:2040A000002110F04DFB1D20002110F049FB1E20002110F045FB1C2014E01C202F2110F09A
:2040C0003FFB3221BCE7012A10D01C20002110F037FB1D20002110F033FB1E20002110F02B
:2040E0002FFB1E20012112F03FF938BD1C20002110F026FB1D20322110F022FB2F211E204E
:2041000010F01EFB38BD7047F0B50E1C14460546ADF1140D04D0084612F0C2FB071C1ED1B4
:20412000324F33203979FF2905D0401E07F12407F8D100274BE001208DF80000ADF80250C3
:20414000314601A812F0C6F96846FFF75DF8BDF80C00002678802846BE7110F009FC0020E4
:204160000122014614B1052CB8BF04213D803C71797106263E727A72AA25BD723882F87106
:20418000F8728023F86087F82130E4B118480678032C18DA17483EB900EB8601096B00EB2F
:2041A0008600F961006B0AE000EB8600036B9901A1EB8301F961016B8801A0EB8100B861CD
:2041C00087F8202003E06FF00100F861B8610020042110F065FA332802DB074900200870A7
:2041E00006F0E6FD384605B0F0BDC0462C100020E804012068800200FD0901202DE9F0433D
:2042000081463848384C07AFADF1240DADF81E300578ADF81C1094F84A009046042814BF62
:204220000828C2205BD0BDF81E004FF6FE71814208BFC32053D0684600211C2207F0CEFD5B
:20424000032007A984F84A0050200DF0B3FD4B200DF11E010DF0AEFD84F83C80BDF81C006F
:20426000BDF81E6084F832504946A4F8480004F15D00E68712F044FB1C4805F0CE0646F037
:20428000800504F1240600788DF81A5030F0010003D13878401C84F85C0002208DF816007D
:2042A0000F258DF80B80002284F85150BDF81E708DF80820BDF81C30ADF80E7006F12D0142
:2042C000ADF8183054200DF075FD06F12C01472084F850500DF06EFD684603F031FB09B079
:2042E000BDE8F083521A012050010120E5040120F0B5364D384C0028ADF1140D6978207297
:204300005ED129B9207818B9082011F0CBFC697831F0010051D168460021102207F05EFDBB
:2043200011F0F2FF002848D0294D05F1240006463930074610F04EFE20B9284938461C3158
:2043400012F0DEFA06F1160153200DF033FD95F83200000934BF0020012004A98DF8100097
:2043600052200DF027FD082085F84A0006F020FD07F05EFE1A49486808B901204860E0795F
:204380004FF440710AF064FE68460FF02FFB684600210FF01FFD95F8650010B9002004F03D
:2043A00003FA68460021102207F018FD09480078012802D0012010F077FA01200FF046FB3C
:2043C000E07902210AF044FE05B0F0BDE4040120500101209A060120C403012000DC0020A3
:2043E000100A01202DE9F84F06467068B6F80A80447800F1020B042C10D0012C07D0062CC9
:2044000005D090F81A9000F1120500270AE090F8129000F1130700F11B0503E000F1120749
:2044200000F11A054FF0010A5FB1384611F043F8012806D111F082FB0146384611F09EFA7C
:204440008246BAF1010F20D0204C607830F0010039D1B8F1000F36D1384669460FF02EF968
:20446000012830D100217172BDF80000708194F8260020B170680078052808BF01213173DB
:2044800030460BF0C5F8BDE8F88F202010F05EFD071C18D004203870A7F80280594610225E
:2044A0003C71B81D87F8059011F078FB07F11600294612F00FF887F81E900548FC77007807
:2044C00039460CF08FF9BDE8F88FC046E4040120CB030120DFF8E8C02DE9F04300260D466E
:2044E00080464FF0B3094FF00E0E3746ADF11C0D01E07F1CFFB2002F5ED1002422462346DC
:2045000001E05B1CDBB263B913FB0EF01CF80010FF29F6D011464A1C8F42D2B2F1D100EBBD
:204520000C04002CE5D061798919CEB2B045E0DA28460021182207F051FC6179A8EB06005F
:204540004018C0B204EB4000C088688111F0F6FA0146284612F0D4F96078012822D06088E1
:20456000ADF80C0004218DF8001068460BF05EFDE0B103208DF8160001A90DF10E0012F0C5
:20458000BFF99DF816709DF81600032F287518BFBDF80E0009D105F10C000DF10E0112F049
:2045A000AFF903E0012028756088A8812078287220794FF00009A875484607B0BDE8F08314
:2045C000220100202DE9F043374C0346354A2668364C108E2578012B9146ADF11C0D0746A2
:2045E00018BF4FF000080CD14FF6F87402E012F0D2F801468C42FADD0029F8D08846B9F805
:2046000030002B4CE6644FF6FF7184F852500F2684F85060B94284F851604FF0000584F88D
:20462000535004D1814201D112F0B5F80746A4F8487009F1500010F0CDFC09F15007012890
:2046400004D104F15D00394612F05AF904F15D00074610F0BFFC18B9E220394610F010F9AA
:20466000A4F83A8084F85060E58784F85160052084F85C5029461C2284F84A00684607F0BA
:20468000ADFB8DF804508DF80750E06C009094F852708DF80570684607F042FD07B0BDE859
:2046A000F083C046E4040120D0030120990601205001012070B5324C0D46A80850D2E8089A
:2046C0005DD30125042065700FF0E8F82D480068006B8047A060606804F198060146306863
:2046E00070B10069064649B18E4207D0B16AC90803D3436A0421002298477576314661608B
:20470000486821490078086002200FF0C7F8112002F040FE1D48007884F8245010B90E209A
:2047200002F038FE60684168886808B9C86810B1174811F041FE174907200026086016492B
:20474000174B0E60154D4E600A68A36245EA020008601A2012F0F2F8192012F0EFF870BDF4
:20476000FBF776FC204600F1A001096811B909F005F870BDE03045F0020112F0F9F870BD17
:2047800068F200208C010010D021084086870200510007060000046014100440024000400E
:2047A000790901002DE9F04781461E46924688460846ADF1180DFDF73FFB404610F04CF84F
:2047C000324807684FB103208DF8080041460822684611F0E3F96846B8472D4C607830F0E6
:2047E000010047D1ADF80290CDF8048002208DF808000025ADF80050404612F051F82EBB9D
:2048000028B9484641460BF069FEAA281ED111F07BFDD8B9AB20294603AA0BF025FF4046E9
:2048200005A92A4607F05CFA94F82700012807D19DF8140020B98DF80950684607F08AFECC
:2048400001208DF80900684607F084FE404612F027F878B1007968B105280BDABAF1010F53
:2048600003D0012818BF022801D112F075F840460AF026FF4846002110F002FA484610F01C
:2048800077F810F091FE06B0BDE8F0872C090120E40401202DE970410546DFF8D880A87A86
:2048A0000024ADF11C0D60B9E87A400909D230480078012804D1404615300078012800D044
:2048C000C824002C4DD12888696805AA0FF0CEFBA87A00282DD14046E97A00784A0902D2DA
